:1000000000560020B16C0000116C0000216C000053
:10001000396C0000516C0000696C000000000000A9
:10002000000000000000000000000000816C0000E3
:10003000916C000000000000A16C0000996D0000B0
:10004000F96B00000000000000000000D51801005E
:1000500011180100811801000000000000000000DC
:10006000954C000059F9000039F900004D190100C4
:100070000000000000000000000000006D190100F9
:100080002DE9F843054689464FF00108154E164CF8
:10009000164F12E0236943F00403236187F832808E
:1000A000BFF34F8F00BF30BF87F83200236923F0C2
:1000B00004032361BFF34F8F62B600F01DF872B6E0
:1000C000735D33B900F014F80028E3D000BF30BFEF
:1000D000F2E700237355B9F1000F00D0C84762B6AC
:1000E000BDE8F8838422002000ED00E000001050FD
:1000F0005FF800F0C54B00005FF800F0B9FC0000AD
:10010000FFFFFFFFFFFFFFFFFFFFFFFFFFFFFFFFFF
:10011000FFFFFFFFFFFFFFFFFFFFFFFFFFFFFFFFEF
:10012000FFFFFFFFFFFFFFFFFFFFFFFFFFFFFFFFDF
:10013000FFFFFFFFFFFFFFFFFFFFFFFFFFFFFFFFCF
:10014000FFFFFFFFFFFFFFFFFFFFFFFFFFFFFFFFBF
:10015000FFFFFFFFFFFFFFFFFFFFFFFFFFFFFFFFAF
:10016000FFFFFFFFFFFFFFFFFFFFFFFFFFFFFFFF9F
:10017000FFFFFFFFFFFFFFFFFFFFFFFFFFFFFFFF8F
:10018000FFFFFFFFFFFFFFFFFFFFFFFFFFFFFFFF7F
:10019000FFFFFFFFFFFFFFFFFFFFFFFFFFFFFFFF6F
:1001A000FFFFFFFFFFFFFFFFFFFFFFFFFFFFFFFF5F
:1001B000FFFFFFFFFFFFFFFFFFFFFFFFFFFFFFFF4F
:1001C000FFFFFFFFFFFFFFFFFFFFFFFFFFFFFFFF3F
:1001D000FFFFFFFFFFFFFFFFFFFFFFFFFFFFFFFF2F
:1001E000FFFFFFFFFFFFFFFFFFFFFFFFFFFFFFFF1F
:1001F000FFFFFFFFFFFFFFFFFFFFFFFFFFFFFFFF0F
:10020000FFFFFFFFFFFFFFFFFFFFFFFFFFFFFFFFFE
:10021000FFFFFFFFFFFFFFFFFFFFFFFFFFFFFFFFEE
:10022000FFFFFFFFFFFFFFFFFFFFFFFFFFFFFFFFDE
:10023000FFFFFFFFFFFFFFFFFFFFFFFFFFFFFFFFCE
:10024000FFFFFFFFFFFFFFFFFFFFFFFFFFFFFFFFBE
:10025000FFFFFFFFFFFFFFFFFFFFFFFFFFFFFFFFAE
:10026000FFFFFFFFFFFFFFFFFFFFFFFFFFFFFFFF9E
:10027000FFFFFFFFFFFFFFFFFFFFFFFFFFFFFFFF8E
:10028000704700BF034613F8012B002AFBD1181A50
:10029000013870470048704720D50100332070476F
:1002A0000220704708B506F025FC08BD08B506F029
:1002B0009FFC43690148984708BD00BF20D5010055
:1002C00010B50C4611461A46012807D010B1022875
:1002D0000BD010BDE0B200F041F8FAE7BDF80830ED
:1002E000C9B2E0B200F07CF8F3E7E0B200F02AF91E
:1002F000EFE700BF044B00229A80DA805A819A818E
:10030000B4221A81704700BF88230020014B18785F
:10031000704700BF8823002010B40446034B0FCB66
:1003200084E80F00204610BC704700BF8C230020DB
:1003300082B0094B5B690020DAB262F30700C3F3B5
:10034000072262F30F20C3F3074262F317401B0E2C
:1003500063F31F6002B070478823002010B5044685
:100360001D4B1B7813F0030F02D010F00C0F15D1AA
:1003700014F0030F1CD113F0080F02D014F0040F77
:1003800022D113F0040F15D014F0080F12D0124B25
:1003900000229A80DA80B4221A810BE006F0AAFBD0
:1003A00002690D4B1A61FFF7A5FF00F001F901E0AA
:1003B000FFF7A0FF084B1C70084C204600F05AFEC7
:1003C000204600F023FB10BD034B00229A80DA8008
:1003D000B4221A81EEE700BF8823002028D501004F
:1003E00010B5044600F06EFF042C00D010BDFFF7DE
:1003F0008DFF10F00C0F05D000F075FF4368984793
:1004000000F0E0F84B4C204600F082FE204600F061
:10041000A3FB494B1A78042A37D0082A4AD0464B06
:100420005B89B3F5616F05D3434B002159819989ED
:1004300001319981404B99894EF66023994251D000
:100440003D4BD9884EF6602399424FD03A4B99885C
:100450004EF6602399424DD012F0080FC6D000F03E
:1004600042FF4368984703689847002846D1324BBB
:100470001B7813F0080FB9D02E4800F083FE002837
:1004800048D02D4BB4221A81B0E72B49CB880133D9
:100490009BB2CB802949A1FB0301490901EB8101F2
:1004A000A3EBC1039BB2002BB9D123494B89013384
:1004B0004B81B4E720490B89013B0B818B880133C9
:1004C0009BB28B801E49A1FB03014909C1EB0111BD
:1004D000A3EB81039BB2002BA1D117494B890133B8
:1004E0004B819CE7144B00219981A9E7124B002115
:1004F000D980ABE7104B00219980ADE700F0F3FE07
:100500004368984700F08FFD0128B0D10A4BB42210
:100510001A81ACE7084B1B7813F0080F3FF466AF65
:10052000054B1B89002B7FF461AF06F061FB03686C
:1005300098475BE728D5010088230020CDCCCCCCA0
:100540008988888810B5062819D8DFE800F01904D2
:100550001D201823260006F0CDFA044606F048FBBD
:10056000C3684FF48062002120469847FFF7C2FE1F
:100570000D4800F07FFD04F1F00000F034FA10BDEA
:10058000094800F09BFDFAE7084B1975F7E7074BA0
:100590005975F4E7054B9975F1E7044BD975024895
:1005A00000F068FDEBE700BF28D50100882300209C
:1005B00008B588220021024819F0DDF808BD00BF07
:1005C000A02300202DE9F04F85B0824600229249F9
:1005D00011F832306FF3C71301F8323001EBC20368
:1005E00058786FF3C710587098786FF3C7109870E9
:1005F000D8786FF3C710D87018796FF3C7101871D7
:1006000058796FF3C710587198796FF3C7109871C4
:10061000D8796FF3C710D8710132112AD8D1DAF81E
:100620000030984703900023029345E04FF0010803
:100630004FF0140CB5423AD801974FF04C093346AD
:10064000464698462BE04FF001084FF0140CF1E7B6
:10065000425C42F08002425402F07F0202EB0C0B3B
:10066000BBF14C0F0FDD425C69F3060242540133CB
:100670009BB29C420FD319461EF80320D209E7D043
:10068000002EF4D0E4E7624410F801B062F3060BE8
:1006900000F801B0EBE70135ADB2A84507D3A7429A
:1006A000F9D8019B5C4A02EBC50E7046E3E7029B5A
:1006B000013302930A2B66D09DF80880DAF82830BF
:1006C00040469847012805D0DAF828304046984738
:1006D0000228ECD1DAF80C30404698478146DAF827
:1006E000103040469847834600EB00134B4A82FB8C
:1006F0000312DE17C6EB22264FEAC903484A82FBE3
:1007000003271F44DB17C3EBA727DAF8183040464E
:100710009847DAF8083040469847002814BF11245B
:100720000424B6B2351B25EAE575ADB22644102E79
:10073000A8BF1026B6B2BBB21F1B27EAE777BFB22D
:100740001C44072CA8BF0724A4B2DAF8083040469E
:100750009847A9F141091FFA89F940F2B633994542
:100760003FF664AFBBF1B90F7FF66DAF002814BF41
:100770004FF0140C4FF0010C002814BF4FF001088B
:100780004FF0000856E70026234F1FE0043AE55CCF
:1007900062F30605E55404E0013AE55C62F3060500
:1007A000E5540133082B0ED0C25CD209F9D1C25CEA
:1007B00002F07F02122AEFD8032AE7D8E25C6FF337
:1007C0000602E254EDE70136112E04D0002307EBB8
:1007D000C6000446E8E7039B1BB1002421460E4DEA
:1007E00005E0FFF7E5FEF8E70134112C0DD00023FA
:1007F00005EBC400C25C02F07F02092A84BF01310C
:1008000089B20133082BF5D1EEE7034BA3F888102A
:1008100005B0BDE8F08F00BFA0230020B5814E1BBE
:1008200049D6B9F22DE9F04F83B00646019114463E
:100830000368984770B13E4A92F88A30013382F8D3
:100840008A30A146002C5ED00027B8469346DFF8D8
:10085000E8A037E0FFF7ACFE4FF00008019B83F8FB
:10086000008055E0F3682046984740B3336920463E
:10087000984720B3F36820469847054633692046D9
:10088000984700EB00108AFB0023C017C0EB232021
:1008900080B2ED00274B83FB05232B44ED17C5EBFE
:1008A000A325ADB20BEBC000435D03F07F03122B19
:1008B00005D808F101085FFA88F8019B1C70013720
:1008C0004F4510D0FCB2B36A204698470128C9D0E2
:1008D000B36A204698470228C4D0B36A2046984796
:1008E0000328ECD1BEE7B8F1000F0CD0104BB3F8E1
:1008F0008830442B10D8B8F1010F09D012D9002349
:10090000019A137004E04FF00008019B83F8008007
:10091000404603B0BDE8F08F4FF00008019B83F81C
:100920000080F5E74FF00008019B83F80080EFE7B7
:10093000A023002049D6B9F2B5814E1B431E9BB2BD
:100940004FF6FD7293421BD84B1E9BB2934219D8AF
:1009500001EB01110C4B83FB0131090AC0000B4B69
:1009600083FB00231844C0F38F20094B03EBC10124
:10097000085C00F07F0013288CBF00200120704726
:100980000120704701207047B5814E1B49D6B9F24E
:10099000A0230020F8B506460F4C2568238903EBF9
:1009A00083035B00F4336B8006F022F9043523895E
:1009B00003EB830307690A22314605EB4300B8477E
:1009C000238901339BB22381226852789A4201D84D
:1009D00000222281F8BD00BF2C240020704708B5FA
:1009E000FFF7D8FF08BD10B5044606F001F9C3684B
:1009F0004FF44472002120469847034B1C60462365
:100A000063700A23237010BD2C24002030B5A5B0DC
:100A10000446436898474F4B1B7913F0030F09D0E6
:100A2000A368984710F0080F21D1A368984710F0E9
:100A3000040F1CD1474B1B7913F00C0F09D0A3688E
:100A4000984710F0020F41D1A368984710F0010FAA
:100A50003CD1A36898473F4D2871E36804A89847A4
:100A6000BDF81830EB8000236B8125B030BD002528
:100A700001950295ADF80C5006F0BAF8C3680A2249
:100A8000294601A898479DF80430022262F3020328
:100A90008DF80430E36810A89847BDF80430BDF81D
:100AA000462062F30F13ADF80430E3680CA89847B2
:100AB000BDF83E30ADF80630E36808A898470B9BB8
:100AC000ADF8083001A8FFF765FFB3E700250195F1
:100AD0000295ADF80C5006F08BF8C3680A2229463F
:100AE00001A898479DF80430032262F302038DF8B1
:100AF000043063689847BDF80430028862F30B1332
:100B0000ADF80430134A52891209C3F3072362F384
:100B100007138DF80530E36820A89847BDF88230A8
:100B2000ADF80630E3681CA89847BDF87030ADF802
:100B30000830E36818A89847BDF86E30ADF80A3061
:100B4000E36814A89847179BADF80C3001A8FFF78D
:100B500021FF7EE72C2400202DE9F04FA9B00546A7
:100B600043689847AB68984710F0080F04D1AB680A
:100B7000984710F0040F39D02B689847436898477E
:100B8000044600F050FA80B12B68984743689847B4
:100B90008146002705970697ADF81C7002460A218A
:100BA00005A800F02CFAB846D3E0204600F03FFA42
:100BB0000028E9D16B689847B0F86030002B40F00E
:100BC0005781AA4BDC880134EB6818A89847BDF818
:100BD00068309C4200F0BB81EB680FA89847A34B9C
:100BE000BDF84420DA805A8901325A8129B0BDE823
:100BF000F08FF368204698473369204698472B6862
:100C0000984743689847834600F019FAB0F1000A04
:100C1000C0F228816B689847C388ADF80C306B68C8
:100C200098470389ADF80E306B6898474388BDF844
:100C30000C201344ADF810306B6898478388BDF8DA
:100C40000E201344ADF812305FFA8AFADBF80C304C
:100C5000504698470190DBF810305046984703AA59
:100C60000146019800F0A4F9002840F0FD804FF4FF
:100C7000C973ADF80C3040F66A03ADF80E3040F29F
:100C8000A623ADF8103040F62413ADF81230DBF88F
:100C90000C30504698470190DBF81030504698478A
:100CA00003AA0146019800F083F9003018BF012023
:100CB0009DF8263060F345138DF826306B68984711
:100CC00090F86330C3F302039DF8282063F3020217
:100CD0008DF828206B68984790F86230C3F30203C0
:100CE000BDF8282063F38812ADF82820B3682046A9
:100CF00098479DF8293060F382038DF82930B36955
:100D0000204698471F2828BF1F20BDF8263060F3D3
:100D10008A13ADF82630F369204698471F2828BF6C
:100D20001F209DF8273060F3C7038DF82730336A02
:100D300020469847C0F38F001F2828BF1F209DF82A
:100D4000293060F3C7038DF8293008A8FFF722FE89
:100D50000137D9F800309847FBB28342BFF42AAF7D
:100D6000FBB228AA134413F88C4CCDF82080CDF8A0
:100D70002480ADF82880D9F82830204698470128EB
:100D800005D0D9F82830204698470328E0D12B68B1
:100D90009847436898470646EB680BA89847BDF804
:100DA00030A005F025FFC3680A22414608A89847ED
:100DB0009DF820306FF302038DF82030B36A20468F
:100DC0009847012814BF002001209DF8203060F3CF
:100DD000C3038DF82030BDF82030BDF8322062F317
:100DE0000F13ADF820304FEA1A129DF8223062F34B
:100DF00003038DF822309DF824306AF303038DF845
:100E00002430F36820469847BDF8223060F30F1372
:100E1000ADF82230336920469847BDF8243060F39E
:100E20000F13ADF824302B69984713909DF82630A6
:100E3000C0B260F301038DF82630736A20469847EC
:100E40009DF8263060F383038DF8263003F00C0301
:100E50000C2B7FF4CEAE9DF8263043F00C038DF8BA
:100E60002630C6E6404623E7012021E72C24002057
:100E700000230B930C93ADF834302B6898474368EC
:100E80009847064600F0DBF8041E4FDB05F0B0FE85
:100E9000C3680A2200210BA898479DF82C30012234
:100EA00062F302038DF82C30EB6814A89847BDF864
:100EB0002C30BDF8562062F30F13ADF82C306B6860
:100EC000984790F8603013F0020F3AD16B6898475A
:100ED00090F8603013F0040F35D16B68984790F8A4
:100EE000603013F0080F30D16B68984790F860308D
:100EF00013F0100F14BF062200229DF82E3062F36B
:100F000003038DF82E30E4B2F36820469847BDF80D
:100F10002E3060F30F13ADF82E303369204698471A
:100F2000BDF8303060F30F13ADF830300BA8FFF789
:100F300031FD6B6898470023A0F860301B4A53814D
:100F40003FE60122D9E70422D7E70522D5E70024AE
:100F50000B940C94ADF8344005F04AFEC3680A22A5
:100F600021460BA898479DF82C30042262F3020317
:100F70008DF82C30EB6824A89847BDF82C30BDF8CC
:100F8000962062F30F13ADF82C30EB6820A8984739
:100F9000BDF88E30ADF82E30EB681CA898471F9B2B
:100FA000ADF830300BA8FFF7F5FC15E62C24002037
:100FB000134672B1128882420DD89A8882420CD3AD
:100FC000DA888A420BD3588888428CBF00200120DF
:100FD00070470020704700207047002070470020B5
:100FE000704710B50446084611460023224600F01B
:100FF000BBF90021204600F0E4F9C0B210BD08B5ED
:10100000002300F0B1F908BD08B500F0ADF908BD46
:1010100008B5002100F0D5F9C0B208BD08B500F050
:10102000D0F9C0B208BD08B500F076F908BD08B522
:1010300000F086F908BD08B500F05AF908BD08B5FA
:1010400000F0E6F908BD000010B543689847048831
:10105000003418BF012405F0CBFD8368224603212C
:101060000220984705F0C4FD83682246032104202E
:10107000984710BDF8B507460F4B1B68BBB100245D
:1010800025460D4E56F8253053B156F82530984771
:1010900003682BB156F825309847036838469847BF
:1010A0000134E4B2254656F82430002BEAD1384604
:1010B000FFF7CAFFF8BD00BFC00F0020F8B5074614
:1010C000124B1B68F3B100242546104E56F825300C
:1010D0008BB156F82530984743683846984750B149
:1010E00056F825309847C3682BB156F825309847F5
:1010F000C368384698470134E4B2254656F8243090
:10110000002BE3D13846FFF79FFFF8BDC00F00204A
:101110002DE9F04107461A4B1B68002B2DD0002407
:101120002646174D05E00134E4B2264655F8243032
:101130001BB355F82630002BF5D055F826309847CC
:101140004368384698470028EDD055F82630984730
:1011500090F81480BB68984718EA000FE3D055F860
:10116000263098478368002BDDD055F82630984705
:101170008368384698470028D5D0BDE8F08100BF85
:10118000C00F00202DE9F04107461C4B1B68002BC7
:1011900032D000242646194D05E00134E4B226463B
:1011A00055F824302BB355F82630002BF5D055F8E0
:1011B000263098474368384698470028EDD055F8C0
:1011C0002630984790F81480BB68984718EA000FBB
:1011D000E3D055F8263098470369002BDDD055F849
:1011E000263098470369384698470028D5D0012013
:1011F00000E00020BDE8F0810020FBE7C00F0020E8
:1012000008B5436898470078C0F3400008BD7047B0
:1012100030B587B00446036898474368984702464C
:101220001F4903A800F0CFFE9DF8153013F0020F00
:101230002ED0BDF80C30CD3B9BB240F29D229342A4
:1012400029D8BDF80E2040F6B7039A4225D99DF85B
:101250001430043BDBB2382B01D9002019E0002305
:10126000019302934FF00203012565F387138DF874
:10127000043005F0BDFC436801A8984763689847AF
:1012800090F8603043F0020380F86030284600E0B8
:10129000002007B030BD0020FBE70020F9E700BFC9
:1012A0003824002008B540F2371354223E2102486A
:1012B00000F074FE08BD00BF3824002000487047CD
:1012C0003CD5010010B51446012802D0022805D0F3
:1012D00010BD1A46204601F043F8F9E719461046BA
:1012E00000F0FCFFF4E70148704700BF54D501004F
:1012F00038B505460368984748B10024AB68E0B2AA
:101300009847034630B901340A2CF7D100E0002396
:10131000184638BD0123FBE738B5054603689847F2
:1013200050B10024AB6AE0B29847012806D00134DE
:101330000A2CF7D1002000E0002038BD0120FCE796
:1013400038B505460368984750B10024AB6AE0B24F
:101350009847032806D001340A2CF7D1002000E07A
:10136000002038BD0120FCE72DE9F84F8246894670
:101370001646984600252F4609E07B1CDBB20AF88A
:1013800007404B451BD01F4601350A2D17D0ECB244
:10139000B36A204698470028F6D0F368204698475D
:1013A0008346336920469847B8F1000FE5D042469E
:1013B00001465846FFF7FCFD0028DED1E4E7BDE812
:1013C000F88F2DE9F843074688460024264604E0B6
:1013D0000136F6B201340A2C17D0E5B2BB6A2846B2
:1013E00098470028F6D0FB682846984781463B6915
:1013F00028469847B8F1000FEAD0424601464846D1
:10140000FFF7D6FD0028E3D1E4E770B2BDE8F8832A
:1014100038B505460368984760B10024AB6AE0B26E
:10142000984728B901340A2CF8D14FF0FF3038BD65
:1014300060B2FCE74FF0FF30F9E7000008B5436801
:1014400098470078C0F3C00008BD064B41221A80BF
:10145000BA225A8040F2F7329A8040F6A602DA8029
:10146000704700BF54240020F0B585B005460368DE
:101470009847436898470246204902A800F063FC59
:101480009DF80830022B03D00024204605B0F0BDA3
:10149000BDF80A70BDF80C60194A31463846FFF7AE
:1014A00087FD04460028F0D00023009301934FF0FD
:1014B0000203042262F38503012464F387138DF889
:1014C000003047FA02F38DF8023046FA02F38DF845
:1014D000033006F00F0646EA07168DF8046005F0A3
:1014E00087FB4368684698476B68984790F8603078
:1014F00043F0080380F86030C7E700BF5C24002099
:101500005424002010B584B00D4C0E2303935D23AA
:1015100002931E230193022200921223012104F15F
:10152000080000F0E9FB41232380BA23638040F2E6
:10153000F733A38040F6A603E38004B010BD00BFDC
:1015400054240020004870475CD5010008B543686A
:101550009847037813F0240F14BF0120002008BD22
:1015600038B543689847C5880489418829448288EA
:101570002244034B5D809C80D9801A8138BD00BF16
:10158000882400202DE9F04784B0804643689847BE
:101590000378C3F38009C3F34017D8F800309847A5
:1015A000436898473C4E024606F1140102A800F039
:1015B000CAFB9DF808A0BDF80A50BDF80C40B21C4B
:1015C00021462846FFF7F4FC30BB06F10A0221460B
:1015D0002846FFF7EDFC034600285AD1184604B010
:1015E000BDE8F0872C4B1A700023F7E71FB32A4B96
:1015F0001B78012B1FD00023F0E7D8F80430984760
:1016000090F8603043F0040380F860300123E5E790
:101610000023E3E70023E1E70022BAF1010FE1D064
:10162000BAF1020FF4D1B9F1000FDFD01FB91A4B94
:101630001B78002BEED1002301934FF0020301220F
:1016400062F3850362F387138DF80030124E33780E
:101650008DF801302B118DF8023023118DF80330F5
:1016600004F00F0444EA05158DF8045005F0C0FAA3
:101670004368684698473378002BBED0D8F80430CA
:10168000984790F8603043F0200380F860300123E1
:10169000A4E70122C1E700BF8824002030B587B04D
:1016A0000546036998470590030E1FD1254C0A2370
:1016B00003935D23029324230193052300931223B4
:1016C0000222114604F1140000F016FB6B689847E3
:1016D000C588018942882A4483880B446580A1809B
:1016E000E2802381BA2140F6A6021FE0154C0A23AE
:1016F0000393662302932423019307230093122369
:101700000322022104F1140000F0F6FA6B689847F6
:10171000C588018942882A4483880B446580A1805A
:10172000E280238140F2864140F69E02054B412033
:101730005881998140F2F731D9811A8200221A70BA
:1017400007B030BD882400200048704774D50100E0
:1017500070B50646002425467368984720444576B0
:1017600001341C2CF8D170BDF8B503689847436864
:10177000984705460C4CC368A07A984706462B69E3
:10178000A07A98470746AB6AA07A9847022801D00A
:101790000020F8BD04F1140239463046FFF708FC7A
:1017A000003018BF0120F4E7C824002038B50446F3
:1017B00043689847037D012B0CBF01210321244876
:1017C00000F0CBFC63689847B0F84B4040F2A91397
:1017D000002C18BF23461E4A9382B0F84D1040F2E9
:1017E000E173002918BF0B46D382B0F84F2040F2B6
:1017F0008F23002A18BF1346154D2B83B0F85130A4
:1018000040F6C700002B18BF184668839CB14E3CB9
:10181000A4B20F48848389B14E3989B20C48C18380
:101820007AB14E3292B20A490A846BB14E339BB2FE
:10183000074A538438BD40F25B14EAE740F29371E3
:10184000ECE740F2DD22EEE740F61513F0E700BFCB
:10185000C82400202DE9F04F8DB006460368984754
:10186000436898470446924901F11403024609A8C7
:1018700000F082FCBDF824300093BDF826A09DF84E
:101880002D509DF82EB0BBF1010F13D0884B93F86B
:101890002430012B40F00981A36A28469847032889
:1018A0000DD060B102283DD0BBF1010F00F0C18026
:1018B000002433E07E4B012283F82420ECE77C4BAC
:1018C000002483F8244083F825403046FFF740FF8A
:1018D0000394022343F00C02012464F387128DF871
:1018E00008208DF80930009A13118DF80A304FEA5C
:1018F0002A138DF80B300AF00F0A4AEA021A8DF803
:101900000CA005F075F9436802A8984773689847DA
:1019100090F8603043F0100380F8603020460DB03E
:10192000BDE8F08F624B93F82530002BBCD1E36803
:101930002846984707462369284698475D4A014646
:101940003846FFF735FB60BB0121594B83F8251062
:10195000002303934FF00203032262F3850361F334
:1019600087138DF808308DF80920009A13118DF82F
:101970000A304FEA2A138DF80B300AF00F0343EABE
:1019800002138DF80C3005F033F9436802A898472C
:101990007368984790F8603043F0100380F8603027
:1019A00082E7002702970397049705970697079702
:1019B000089714234FF00109CDF804A09A4624E0BB
:1019C0000135102D19D07C19A4B2336898470368EB
:1019D0000320984703684146E8B298477D28EFDD29
:1019E0000CAB03EBD40304F0070409FA04F413F876
:1019F000282C144303F8284CE2E71037BFB20AF151
:101A0000010A1FFA8AFAE02F03D000255FFA8AF84C
:101A1000D9E7DDF804A002AF0DF124083C46E51B30
:101A20007368984714F8013B28444376A045F6D1E3
:101A30003AE7214ABDF82A10BDF82800FFF7B8FAA6
:101A4000044600283FF46AAF73689847027D012A74
:101A500014BF00220122002303934FF0020303214D
:101A600061F38503012464F387138DF808308DF842
:101A70000920009A13118DF80A304FEA2A138DF8C5
:101A80000B300AF00F0343EA02138DF80C3005F017
:101A9000AFF8436802A898477368984790F8603099
:101AA00043F0100380F8603038E7002436E700BFC9
:101AB000C8240020E4240020DC24002010B5436862
:101AC00098470478C4F300140CB9204610BD05F003
:101AD0008FF883680122032110469847F5E770B517
:101AE000044643689847037D012B114E4FF04E0387
:101AF0000CBF012203221946304600F030FB0025BE
:101B000086F8245086F825502046FFF721FE6368AA
:101B1000984710234375636898470E23837563685D
:101B200098471C23C37563689847057670BD00BF4E
:101B3000C8240020004870478CD5010010B5044629
:101B4000C28A038A9A4202D901234375837494F8A6
:101B50002530012B0FD0227D0A4B53F8223020462E
:101B6000984701280CD0022814BF00200220638D62
:101B70000133638510BD042363750123A374EAE771
:101B80000120F4E7D40F0020C289B0F91830B0F971
:101B900020105B1A002BB8BF5B42934218DCB0F9EF
:101BA0001A30B0F922105B1A002BB8BF5B429A4280
:101BB00010DBB0F9262043889A4207DCB0F92A30BE
:101BC00040898342CCBF002001207047002070472D
:101BD000002070470020704770B5044690F82450EC
:101BE000012D05D9AB1EDBB2012B08D9002070BD39
:101BF000012383740020207503236375F7E7C68CE7
:101C0000013636B2C684FFF7BFFF08B90123A374BB
:101C1000032D01D00020EAE723889E42BCBF0123A8
:101C2000A37463889E42C4BF0123A3740023237559
:101C3000E27C237B9A4201D00020D8E7B4F9283017
:101C4000A2889342BCBF0122A274E2889342C4BF1F
:101C50000123A374B4F92A3022899342BCBF012224
:101C6000A27462899342C4BF0123A3740023238515
:101C7000A37C4BB10020A0746685A38B2383E38BE8
:101C800063830123E374B2E70023E3740220AEE729
:101C900010B5044690F8243023B9038D0133038531
:101CA000002010BD012B25D1FFF76EFF18B90223CC
:101CB00063750123A3740122E284E37C1344DBB245
:101CC000E3742275B4F92010A183B4F92220E283D1
:101CD0003BB1A37C2BB9E07C012814BF002001207C
:101CE000DFE70020A07401236385208521836283C0
:101CF000E374F0E70020D4E730B4BDF80850BDF835
:101D00000C400280438001FB02F292B2AB1A838046
:101D1000A21AC280058144810173BDF81030C381CD
:101D2000BDF81430038200238374C3740385438594
:101D3000C38443754FF6FF72028342838283C2835A
:101D4000037530BC7047F0B585B005460C461646A5
:101D5000002301930293ADF80C30498B208BFEF7E2
:101D6000EDFDD0B10A2201A93046FEF75BFD012846
:101D700022D90023A374E37423856385E384637508
:101D80004FF6FF7222836283A283E28323752B7056
:101D90006B80AB80284605B0F0BD0023A374E374CC
:101DA00023856385E38463754FF6FF722283628324
:101DB000A283E2832375D5E79DF8047000B3F3682E
:101DC0003846984720843369384698476084B36A18
:101DD0003846984784F82400B36938469847E0822B
:101DE0003046FFF728F9A0B9002384F825302046B3
:101DF000FFF7A4FE228B638B28706A80AB80C9E753
:101E00004FF6FF7323846384002384F82430E38235
:101E1000E6E7012384F82530E9E700BF70B5044602
:101E20000E4615788B6A28469847012801D0012074
:101E300070BD002323806380A380E38023816381BE
:101E4000A381E38123746374227E02F0F80263F3BA
:101E5000C3022276F36828469847A0813369284652
:101E60009847E081237C01332374E0E72DE9F041BA
:101E700004460F461678CB683046984780463B6943
:101E8000304698470546BB6A30469847032841D0FC
:101E9000A389A8EB03031BB22380B4F902209A4262
:101EA000B8BF1A4616466280B4F904709F42A8BFB4
:101EB0001F46A780E089281A00B2E080B4F9082004
:101EC0008242B8BF02462281B4F90A108142A8BFFB
:101ED00001466181B4F9125001EB050C604553DAFB
:101EE000491B884250DD521B904203DC227E42F0A7
:101EF00002022276EA1993424BDA7F1BBB4248DD8D
:101F0000721B9342DEBF237E43F008032376012039
:101F1000BDE8F08100232374B4F90020E38A9A42DB
:101F200022DB217E01F00801002914BF00201020CF
:101F300059428A4206DC227E12F0040F04BF40F0B0
:101F40000800C0B2B4F9062093420FDC237E13F0E0
:101F5000020F0BD140F00400C0B29142D8DB237EC7
:101F600013F0010F08D0D3E70020E1E7914207DB2F
:101F7000237E13F0010F03D140F00200C0B2C7E787
:101F8000002808BF0120C3E7217E41F0010121762E
:101F9000A9E7227E42F004022276B1E741828282E2
:101FA000C3820023038043808380C38003814381F5
:101FB0008381C38103744374027E02F0F80263F3E9
:101FC000C302027670472DE9F04186B004460D4603
:101FD000164600238DF81730314903AA03C982E859
:101FE000030000930193ADF808300A226946304699
:101FF000FEF7F7FF80469DF800708DF81770B36A02
:1020000038469847002831D0B8F1010F2ED1B36976
:1020100038469847AB8A834228D3B36838469847F6
:1020200020BBF3689DF817009847804633699DF8F8
:102030001700984707462B7C06AA02EB830353F848
:102040000C3C0DF11702314628469847A989EA89C8
:102050006B7C5E1C6E7421806280A4F80480E78033
:1020600023726072204606B0BDE8F08100232B8009
:102070006B80AB80EB802B816B81AB81EB812B7410
:102080006B742A7E02F0F80263F3C3022A7623807F
:102090006380A380E380237201236372E2E700BFC1
:1020A000A4D5010070B504460E4615468B6A10464D
:1020B0009847012801D0002070BD0023237223809F
:1020C0006380A380E3806372A372E372F36828469F
:1020D000984720803369284698476080A572637AC4
:1020E00001336372E7E7F8B504460E4615468B6A7E
:1020F000104698470746F36828469847A0803369FA
:1021000028469847E080238A9BB9A289B4F9003019
:10211000B4F904105B1A002BB8BF5B42934213DC86
:10212000B4F9023000B2181A0028B8BF4042824207
:102130000ADB227AE3899A4209D300236372E07AA8
:10214000B0FA80F04009F8BD0123E372F1E7032FF4
:102150004FF0000008BF6072F5E7C18170478181D0
:10216000C281038200230372038043808380C38083
:1021700043728372C37270472DE9F04186B0044602
:102180000D4617461E460023036043608360039399
:102190000493ADF814300B8A3288D21AADF80420BB
:1021A0007288D21AADF80620B2881A44ADF8082019
:1021B000F2881344ADF80A3001A93846FEF72EFF25
:1021C000804631463846FEF729FFB8F1010F0DD0A1
:1021D000AA7A00236B7223806380A380E38023723A
:1021E0006272A372204606B0BDE8F08108B90023F0
:1021F0002B7201AB3A460A2103A8FEF705FF6A7A63
:102200000D4B53F822309DF80C203946284698474C
:10221000B5F800C06F88AE88E9882B7AAA7A03F1F6
:10222000010E85F808E0A4F800C06780A680E18070
:1022300023726272A072D5E7DC0F0020014B188870
:10224000704700BFF02400200A207047024B5B68F3
:1022500003EB0010807B7047F0240020024B5B688A
:102260000001185C704700BFF0240020024B5B683F
:1022700003EB001040887047F0240020024B5B689D
:1022800003EB001080887047F0240020024B5B684D
:1022900003EB0010C0887047F0240020024B5B68FD
:1022A00003EB001000897047F0240020024B5B68AC
:1022B00003EB001040897047F0240020024B5B685C
:1022C00003EB001080897047F0240020024B5B680C
:1022D00003EB001040787047F0240020014B198078
:1022E00058607047F024002000487047ACD50100CA
:1022F000C0F10F0000EB001001EB4000024B1B6827
:1023000033F91000704700BFF8240020C0F10F001F
:1023100000EB001001EB4000024B5B6833F910004A
:10232000704700BFF8240020C0F10F0000EB001040
:1023300001EB4000024B9B6833F91000704700BF6F
:10234000F8240020C0F10F0000EB001001EB40006A
:10235000024BDB6833F91000704700BFF8240020FF
:10236000014B43F821007047F8240020014B03EB98
:1023700080007047D8D50100E22230B50E4B83B003
:1023800000921A680D490E4B632000F0BDFC0D4C05
:1023900004F1140554F8043B1B699847AC42F9D189
:1023A000E522094B00921A680449054B632000F0AE
:1023B000ABFC03B030BD00BF04040020F099010065
:1023C000F89901001400002008040020DA2330B539
:1023D0000E4A0F4D0F4C83B02146126863200093C4
:1023E0002B4600F091FC0C4A0C4B127853F822302B
:1023F000DB689847DC200A4A2B4612682146009089
:10240000632000F081FC03B030BD00BF0404002055
:10241000F8990100E4990100E40F00201400002065
:1024200008040020932330B50E4A0F4D0F4C83B0A3
:1024300012682146009363202B4600F065FC0021C2
:102440000B4B0C4A1B6811705B68984796200A4A30
:102450002B46126821460090632000F055FC03B023
:1024600030BD00BF04040020F8990100D899010094
:1024700014000020E40F0020080400207E2230B564
:10248000114B83B000921A681049114B632000F081
:102490003BFC00220F4B104C1A7004F1140554F849
:1024A000043B1B689847AC42F9D18D2300250B4CA7
:1024B0000B4A0649126863200093054B257000F013
:1024C00023FC03B030BD00BF04040020CC99010000
:1024D000F8990100E50F002014000020E40F00200F
:1024E00008040020002370B5454C8CB003A801936C
:1024F00007F0F6FE2378002B61D0424A424B127857
:1025000053F822309B689847237801909DF81B2050
:102510009A4252D09DF81B30DBB2002B23700CBFC7
:10252000022301239DF8242012B101228DF80420FA
:102530009DF825201AB10121344A82F82210012B7E
:1025400034D0022B15D09DF80420002A3CD1002065
:10255000019BDAB262F30700C3F3072262F30F2094
:10256000C3F3074262F317401B0E63F31F600CB006
:1025700070BD0723234C8DF80430237804259D4239
:10258000E5D0214E56F82330DB6898472A4621785B
:1025900002200DF0F9FF2A46217802200DF09EFF5F
:1025A00056F8253025705B689847D0E70623154C10
:1025B0008DF8043023780325E1E70023B2E79DF886
:1025C0001B20002AA2D198E70E4C013A2378062A54
:1025D000BDD801A151F822F0FD250000F925000029
:1025E0004F250000F52500004F250000B72500000D
:1025F0007D2500000225C2E70125C0E70025BEE7D2
:10260000E50F0020E40F0020140000208C0D0020B6
:1026100030B4184D0022D5F8014001322346186825
:1026200002EBC201294480B1586898B19868B0B1F2
:10263000D868C8B1042A1BD0D1F80130013218681B
:1026400002EBC20129440028EED1206818605868C6
:102650000028EBD16068586098680028E8D1A0682D
:102660009860D8680028E5D1E068042AD860E3D1F2
:1026700030BC7047A403002030B4184D0022D5F8B8
:10268000014001322346186802EBC201294480B19F
:10269000586898B19868B0B1D868C8B1042A1BD0FE
:1026A000D1F801300132186802EBC2012944002838
:1026B000EED12068186058680028EBD16068586037
:1026C00098680028E8D1A0689860D8680028E5D10B
:1026D000E068042AD860E3D130BC7047D4030020FE
:1026E00010B502F0CDF8094B1B689847084B1B68E2
:1026F0009847084B1B689847BDE81040064A074BAF
:10270000127853F822305B68184700BF00000020A1
:102710005C0D0020240D0020E70F0020C4A1010063
:1027200070B500249AB010AE2146304628220BAD79
:10273000CDE90B44CDE90D440F9417F01CF808AB1C
:10274000CDE90333CDE90544CDE9005606480293AF
:1027500008940994ADF828402B4604682A46294677
:102760000A20A0471AB070BD282600200B4A08B5E1
:1027700012780B4B53F82230DB689847FFF7D0FFF5
:10278000084B1B699847084B1B699847074B1B6907
:102790009847BDE8084002F00FB800BFE70F0020DF
:1027A000C4A10100000000205C0D0020240D0020C9
:1027B00070B58AB0054608F01BF80128044606D01B
:1027C0002DB1012D38D0032D14BF044602241E4D17
:1027D0002B78A34221D001A807F082FD2246297858
:1027E00001200DF0D1FE2246297801200DF076FE61
:1027F0002B78012B13D0012C20D0144E56F8233007
:10280000DB68984756F824302C705B689847287826
:102810000AB0BDE8704007F0F1BF0AB070BD002CEF
:10282000E9D1FFF7A3FF2C70FFF75AFF28780AB011
:10283000BDE8704007F0E2BF0024C8E79DF8132010
:10284000002ADAD1EDE700BFE70F0020C4A10100A4
:102850002DE9F04F93B007F02BFD09A807F040FDDC
:1028600009A80DF07DFE5B4A5B4B12785B4D53F877
:1028700022309B6898470890C0F3072AC0F30744AA
:1028800004F022F907F0C4FF2A789DF82A30834625
:102890009A4206D09DF82A0006F042F89DF82A30A8
:1028A0002B704F4B0125986805F028FB0026CB23A1
:1028B000DFF850814B48DFF844914B4F05932A468F
:1028C00029464346CDE90309CDE901660095642018
:1028D00000F0C8F93B6898F800209978914213D02D
:1028E000D121CDE901662E46404A0233059103927B
:1028F000CDF8109000952A462946642000F0B2F9E0
:102900003B689B7888F800300DF0DCFA3B688DF866
:102910001F00DB7883421BD1BBF1000F2CD15EBBC3
:1029200074B39DF83D30002B9DF83C3018BF002457
:1029300053B3002007F062FF4FF0010A012C2DD0A5
:1029400074BB5046FFF734FF012013B0BDE8F08F91
:102950000122E02100232648CDE90491CDE901338D
:1029600003900DF11F0364200092114600F07AF9E4
:102970003B68D8780DF092FA002007F04FFF022450
:102980009DF83C30002BD4D19DF83330002BD5D0AE
:1029900007F02EFF0228CCD0012CD1D10FF064F922
:1029A0007E22144B00921A681349144B632000F0E6
:1029B000ABF9FFF7DBFEFFF793FE8322104B00928B
:1029C0001A680D490D4B632000F09EF9012013B0E9
:1029D000BDE8F08FE70F0020C4A10100E60F002042
:1029E000D805002090A101000C0600209CA1010048
:1029F000B8A10100040400206CA1010080A1010025
:102A000008040020380400202DE9F0479CB004465B
:102A100003A8884607F064FC00235B4E9DF8232042
:102A2000C6E90033C6E902333382002A58D094F84D
:102A30002B0094F82AA094F82990504594F828E0A7
:102A40003AD8A0F11D01A0F11007821EC9B2FFB251
:102A5000D2B2F14526D84B4614E0A3F10B04022C68
:102A600041D803EB031400EB440438F9145000245C
:102A700036F914C0AC45B8BF26F814500133DBB2A8
:102A80009E450FD3022AE8D9022F37D8A3F10B04B1
:102A9000022C47D803EB031400EB440438F914501C
:102AA0000324E5E70130C0B201310137013282452C
:102AB000C9B2FFB2D2B2CCD23E2200210DF1320017
:102AC00016F059FE002340F60115822400961A469E
:102AD0000CA91E20ADF830508DF8354008F048F8AC
:102AE0001CB0BDE8F087DC1F022C29D803EB0314CF
:102AF00000EB440438F914500124B9E70229BDD889
:102B0000A3F10B04022C26D9DC1F022C33D99C1E06
:102B1000022CB3D803EB031400EB440438F914502F
:102B20000824A5E7DC1F022C1DD99C1E022CA5D869
:102B300003EB031400EB440438F91450052497E721
:102B40009C1E022C9AD803EB031400EB440438F9C2
:102B5000145002248CE703EB031400EB440438F90F
:102B60001450062484E703EB031500EB4505042409
:102B700038F915507CE703EB031400EB440438F9F3
:102B80001450072474E700BFE80F0020F0B5204E72
:102B900083B0054601F1200014461F467160FDF721
:102BA00071FB1C4B1C4A9968213037604860946067
:102BB00060782278E37802FB00F203F07F0303FBE6
:102BC00002F3164C22790B60D3B2012B01D003B073
:102BD000F0BD7721FF221E46114F397022712379F3
:102BE000FF2B10D120222946684616F095FD009B48
:102BF000032B04EB830206DC019BD2F8052006FAC6
:102C000003F31342EBD105233B7003B0F0BD00BFCB
:102C1000F41900203006002014080020DC1B0020DE
:102C2000E006002070B504460E461546049A194683
:102C300020F8022B20341E2216F05CFE204631467E
:102C4000DF2216F057FE45B13046FDF71BFB294643
:102C5000C0F1DF02204416F04DFE2046BDE8704072
:102C6000FDF710BB2DE9F041C4B004460E461546F1
:102C70000146202204A81F4616F04EFD049B032B9C
:102C80000EDC01221F48059900EB8303D3F805C031
:102C900002FA01F313EA0C0F02D00379934202D037
:102CA00044B0BDE8F0814FF000084FF48072414617
:102CB00004A816F060FD4F9B424600934D994E9B31
:102CC00004A8CDE90288FFF7ADFF9DF80BC04A9B31
:102CD0004B9A8DF80F0063F3060C20464C9C62F370
:102CE000C71C3B4604A902AA8DF808608DF809505C
:102CF0008DF80C808DF80E408DF80BC0FFF746FF65
:102D0000CEE700BFDC1B00202DE9F041C4B0044633
:102D10000D4616460146202204A81F4616F0FCFC6C
:102D2000049B032B0EDC01221948059900EB830359
:102D3000D3F805C002FA01F313EA0C0F02D00379AD
:102D4000934202D044B0BDE8F0814FF000084FF448
:102D50008072414604A816F00EFD4A9B324600934D
:102D600029463B4604A8CDE90288FFF75BFF4346AE
:102D70008DF80F0002AA04A92046ADF808808DF84E
:102D80000B808DF80C808DF80E80FFF7FFFED9E7E1
:102D9000DC1B0020F0B587B0654601F0F5FE01F0C0
:102DA00019FF0021084601F0F5FBD5E90121044691
:102DB00004204FF4457C002701260090074D084869
:102DC0002346CDE90305CDF814C0CDE90167722093
:102DD000FFF748FF204607B0F0BD00BF80A3010009
:102DE00090A301002DE9F04790F815C082B0BCF126
:102DF000000F2BD01C4600254FEA4C0606EB8C0634
:102E000003EB0616216294F8247084F8245094F899
:102E1000257084F8255094F8267084F8265094F88C
:102E2000277084F8275094F8287084F8285094F874
:102E3000297084F8295094F82A7084F82A5094F85C
:102E40002B7084F82B503034A642DBD1BCF1000F3C
:102E50002FD098469146824600269AF814301BB32C
:102E600000257700DAF8003006225C5D68466110C4
:102E7000013116F051FC9AF8142004F0010406FB0D
:102E80000291009B3C449B0004EB440403EB0414BC
:102E900001984B5D4444216A00EB8000834001357A
:102EA0000B43AA422362DDDC9AF815300136B342A7
:102EB000D3DC02B0BDE8F0872DE9F04100241962AF
:102EC000196593F8241083F8244093F8251083F8AB
:102ED000254093F8261083F8264093F8271083F8AE
:102EE000274093F8541083F8544093F8551083F812
:102EF000554093F8561083F8564093F8571083F8CE
:102F0000574093F8281083F8284093F8291083F845
:102F1000294093F82A1083F82A4093F82B1083F85D
:102F20002B4093F8581083F8584093F8591083F8C1
:102F3000594093F85A1083F85A4093F85B1083F87D
:102F40005B40017D82B019B306461D46571E3368AB
:102F5000062213F8048068464FEA6801013116F032
:102F6000DBFB08F0010800994FEA480290448A0010
:102F700002EB081201992A4417F8013F106A01EB8D
:102F800081018B4003431362337D0134A342DEDCB5
:102F900002B0BDE8F08100BF2DE9F04F97B006AF59
:102FA000D1F8016004463863022100203E6101F03F
:102FB000F1FA0021F861084601F0ECFA01F032FC68
:102FC000EC4694F81490647D804604FB09F2D01D11
:102FD000C008ACEBC000854695002B46EC460A3392
:102FE000DB08ACEBC30306A89D46002106AB7B6261
:102FF000FC62FD60786116F0BEFB2A46FF21786A0C
:1030000016F0B9FB07F140031A46042302F8043D09
:10301000114601207A6001F02FFDB2684FEA890362
:103020009178BB61D37812785B1A01339A4240F3EE
:103030005D810A234E46BB626300BB60BB6AB24936
:103040001F2B40F340811A4601FB03F103EB4313AE
:1030500002EB431303EBC33301F1404103F140435F
:103060002031AA4A013341F01F01A9489362C2E905
:10307000081330328242F8D14FF4807300240122C9
:103080004FF004090593A34B01920493A24BCDF892
:103090000090CDE90243BD6A11467B686420FD6360
:1030A000FFF7E0FDFD69FA682146284616F063FB4C
:1030B000FB6A002B00F0F5807D634FF0405B2546F6
:1030C0003C624FF0000A4FF001094FF4FA743B6A7A
:1030D0003A695344137701F057FD01F07BFD8BF8FB
:1030E000F390D6B1D7E90C3C186806EB000E10F847
:1030F000013B03F0010252450BD15B1008EBC313F7
:10310000B3F840201988DCF80030521A1344CCF888
:10311000003070450CF1040CE9D1013C8BF8F35000
:10312000D9D1BAF1000F02D14FF0010ACDE77A6B85
:10313000B9693B6A0A447A63BA68023393423B62D4
:10314000BFD140F2191204237249059204917349C8
:103150000093CDE902410194FD6932462B46F96A9C
:103160006420FFF77FFDD7E9059A7B6AD7F828B07E
:10317000A5F1040EA3F1040C86B16246704600234B
:1031800050F8041F52F8045FA94238BF09F803B091
:1031900003F1010338BF11609E42F1D1FB6A013493
:1031A000A342D644D444B144E6D100244FF49172F2
:1031B0000123CDE9014457495948049103900592F0
:1031C0000093D7F82C907B69324649466420FFF77C
:1031D00049FD40F223120423BD6A4E490135BD6208
:1031E0005048CDE9014404910390059200937B6A15
:1031F000324649466420FFF735FD3E2D7FF41EAF71
:10320000FB6AB146B3B17B6A474D1A1F5EB11046E7
:10321000002150F8043F0131A5FB03C38E424FEA61
:1032200053130360F5D1BB6901341A44FB6AA3420E
:10323000ECD1B1464FF4967200240092354B002237
:103240003A496420FFF760FD40F22D110122314E12
:10325000334B049603937B69CDE9014405910092B9
:10326000D7F82C804A4641466420FFF7FBFC40F229
:103270002F13224600932E4933466420FFF744FD66
:103280004FF498750420CDE90144264B049603932E
:103290007B6A4A460090414605956420FFF7E2FCB0
:1032A0002DE040F219131B4A642004921B4A03923A
:1032B000F96ACDF80090CDE901110593FB6932461A
:1032C000FFF7D0FC71E7BB6A1A4601FB03F103EB81
:1032D000431302EB43130D4A03EBC3330C489362D1
:1032E000C2E9081330328242F8D1C5E64FF49A722F
:1032F000084B00920F4900226420FFF705FD443778
:10330000BD46BDE8F08F00BF208410029800046025
:103310009806046080A30100B8A20100C4A20100C5
:10332000D8A20100E4A20100D34D6210F0A2010076
:1033300004A3010014A301002DE9F043437D864658
:10334000007DF3B1002601F1FF3C0F494FEA43082D
:1033500098B16446DEF80020871812F8019B14F833
:10336000015F09F00103334403EB430301EB031353
:1033700003EB59039742DD73EFD10236464584448F
:10338000E6D1BDE8F08300BF98000460F0B5DCF83A
:10339000000087B064460F46FFF7CEFFD4E9012155
:1033A000002040F21D360125CDE90100054C0648FC
:1033B0003B46CDE90304059600956420FFF752FCD7
:1033C00007B0F0BD80A3010084A20100427D02B3DA
:1033D000F0B40026037DDFF83CC0ABB100247700D9
:1033E000056806FB03122D5D05F001033B4403EB6A
:1033F00043030CEB031303EB5503DB7B1355037DF6
:103400000134A342ECDC427D0136B242E5DCF0BC83
:1034100070477047980004602DE9F04F8046A3B0D4
:103420000391602200210AA816F0A5F94FF4C062AA
:103430000021894816F09FF998F814309E4643B34E
:10344000D8F8000001241D1807E056F85C3C8542BE
:1034500043EA070346F85C3C1BD010F8013B03F03D
:1034600001014E000E441F2B22A904FA03F701EBC1
:103470000616EADD16F8582C203B114604FA03F331
:10348000C2F30102134363F30101854206F8581C9D
:10349000E3D198F81550002D00F04A820021012454
:1034A000D8F80420A81812F8013B04FA03F390425C
:1034B00041EA0301F7D1C1F3130200234FF0405C4E
:1034C0009DF83600039E9DF86670140CD6F80490A3
:1034D00092B220F00F002043ADF83420ADF8642004
:1034E0009DF8292027F00F078DF8360099F8000085
:1034F0003C436FF3C3028DF866408DF85700BDF86A
:1035000030408DF887008DF829209DF832009DF815
:1035100056209DF8597004F0030420F03F0022F07B
:103520001F02ADF830408DF83200BDF860409DF8C4
:1035300062008DF856209DF8862063F3C3078DF84E
:10354000597022F01F0204F0030420F03F008DF8B0
:103550008620ADF854308DF83330ADF884308DF8D6
:103560006330ADF860408DF862003269CCF84810E5
:10357000002D00F0CE81CDE900329A46364B4FF057
:10358000010B0293774641F4801349460993D8F81A
:1035900004C02AF003031A4605931CF80A304FF0C2
:1035A000000E0BFA03F9C9F31309C9F30D039B00CD
:1035B0000793CDF810904FEA993389460432029C64
:1035C0000692089326464FEA4E0522AB754403EB5C
:1035D0000515603D0FCD0FC60FCD0FC695E80F0046
:1035E00086E80F00009A238862F309032380002FE6
:1035F00000F08D8101996FF000420B460F4413F8E3
:10360000011B8A42A8BF0A469F42F8D1D2B2E27299
:1036100099F80630002B40F05A812368049A62F32F
:103620001F33236094F82E3099F8052023F01F03F0
:1036300098F8151084F82E304FF00003501EA38523
:10364000062800F27881DFE810F01B010801E20093
:10365000E000DE00DC000900980004600B1F534509
:1036600040F364810CEB0A031D7994F82E300BFAB9
:1036700005F5C5F3044023F01F030343A58584F833
:103680002E30C5F31405BAF1030F12DD0CEB0A035B
:1036900013F8040C94F82E300BFA00F00543C5F330
:1036A000044023F01F030343A58584F82E30C5F39F
:1036B0001405CB1E534511DD0CEB0A03D87894F8A2
:1036C0002E300BFA00F00543C5F3044023F01F032E
:1036D0000343A58584F82E30C5F31405BAF1020F13
:1036E00012DD0CEB0A0313F8030C94F82E300BFADE
:1036F00000F00543C5F3044023F01F030343A585F1
:1037000084F82E30C5F314058B1E534511DD0CEBE8
:103710000A03987894F82E300BFA00F00543C5F3AD
:10372000044023F01F030343A58584F82E30C5F31E
:103730001405BAF1010F08DD0CEB0A0313F8023C83
:103740000BFA03F31D43C5F31405236894F82E0008
:1037500045EA133545F48015C5F3140320F01F0026
:10376000013940EA13405145A58584F82E000FDD4C
:103770000CEB0A035B78C1B20BFA03F32B43C3F3E0
:10378000140321F01F0141EA1341A38584F82E1090
:10379000BAF1000F07D0D4441CF8011C0BFA01F158
:1037A0000B43C3F3140383F4FF13099883F4FF530B
:1037B00094F82E1083F01F030340C3F3044021F05C
:1037C0001F010143012AA38584F82E100BD0DB438F
:1037D000E268A17BC2F31302134021F00F0242EA18
:1037E0001342A381A2733034BEF1000F57D1039B63
:1037F000D8F804C0D3F8049098F814704FF0010E74
:10380000E0E6002555E700257EE700259DE7013924
:10381000514540F381800CEB0A035B7894F82E103D
:103820000BFA03F3C3F3044221F01F011143A385F4
:10383000C3F3140284F82E10BAF1000F70D0D444F0
:103840001CF8013C0BFA03F31343099AC3F3140366
:103850001340C3F31401DB4308E0394A236882EACA
:103860001333099A1340C3F31401DB4394F82E2059
:10387000A18522F01F0242EA114284F82E20A7E718
:103880004FF0000294F82E30A28523F01F0343F07E
:10389000100384F82E303034BEF1000FA7D0009A08
:1038A00098F815302232C2F309020092029A0AF106
:1038B000010A60320292019A534502F122020192FA
:1038C00027DD039B98F814705B6819465FE6059B3B
:1038D0000CEB0301069B0CEB030511F8013B206880
:1038E0000BFA03F3226843EA103363F31F328D426D
:1038F0002260F2D12389079A03F003031343238143
:10390000A37A089A23F03F031343A3728AE6FF22A7
:103910007DE623B0BDE8F08F0022BAF1000F8ED112
:10392000099B1340C3F31401DB439FE70025AAE67C
:103930002A462946C1E54FF0FF33002196E700BF34
:10394000FFFF0F00002900F0A3802DE9F04FD1F810
:103950000120ADF5137D0CCA93F8009093F801B0E7
:103960001278884609EB0B070AA9064607929D784C
:1039700093F804A0DC78FFF729FD464BF9B2481C08
:1039800083F8290009F1010C09F1FF3083F82210B6
:1039900083F824C083F82500079A002A73D1A9F17F
:1039A0000A0983F827904FF000093A4B4A469E4691
:1039B0000AF03F0C05F01F0004F00F0183F8289077
:1039C00002F114030EEB43039C7801326CF30504FF
:1039D0009C705C88112A60F38A14C4F3072561F394
:1039E000C6055C80DD70EBD14FF04050002280F8BE
:1039F000A720347DBCB14FF0010C3168254D013951
:103A000011F8013F1C2BEA5402F1010209DD90F884
:103A1000A7E01D3B0CFA03F343EA0E03DBB280F888
:103A2000A730A242ECD1D8F801103046FFF7F4FCE1
:103A30000AA93046FFF780FCD8F8013030465968B3
:103A4000DA68C979144BFFF7CDF949F640435E2196
:103A500001370124002504207F0093FBF7F705912F
:103A60000E4A0F49CDE9000404920391029509AB77
:103A70002246214664200997FFF7F4F820460DF509
:103A8000137DBDE8F08F0BF1010B83F827B08AE7B7
:103A900008467047000004609800046080A301009D
:103AA00070A30100F0B50C4699B0602200210746D2
:103AB000684615F060FE30220021544815F05BFE88
:103AC0004FF408709DF80130626843F008038DF8E8
:103AD0000130BDF80010537960F30901013BADF8E6
:103AE0000010032B03D8DFE803F07F6D02024FF0D4
:103AF000FF344FF0405100209DF82E30ADF82C409F
:103B000043F01F038DF82E30C1F830014FF0013320
:103B100000216D461278CDF813308DF82F20CDF8A6
:103B20001730CDF81B308DF81F30CDF80F308DF8E1
:103B30000B100CAC0FCD0FC40FCD0FC495E80F00C8
:103B400084E80F003D7D3DB33C680126254407E035
:103B500052F85C3CA54243EA070342F85C3C1BD0A8
:103B600014F8013B03F00100420002441F2B18A887
:103B700006FA03F700EB0212EADD12F8581C203BAC
:103B8000084606FA03F3C1F301010B4363F3010096
:103B9000A54202F8580CE3D16C461C4F0FCC0FC75E
:103BA0000FCC0FC794E80F0087E80F00184E0CAD3C
:103BB0000FCD0FC60FCD0FC695E80F0086E80F009A
:103BC00019B0F0BD4FF0FF344FF0405100209DF888
:103BD0002E30ADF82C4023F01F0343F00F038DF877
:103BE0002E30C1F8300191E700204FF040519DF890
:103BF0002E30ADF82C0023F01F03064843F01003CD
:103C00008DF82E30C1F8300180E700BF98060460BF
:103C1000C8060460FFFF0F00002900F086802DE930
:103C2000F84FD1F80160424AD6E900531C7893F866
:103C3000018095F800A004EB0805EDB204F101093C
:103C400093F802C093F804E0DF7805F1010B5FFA06
:103C500089F9631E82F829B082F8225082F8253053
:103C600082F82490BAF1000F5AD10A3C82F827401A
:103C700000242F4B224698460EF03F0E0CF01F0CEE
:103C800007F00F0783F8284002F1140308EB430301
:103C90009C7801326EF305049C705C88112A6CF3E9
:103CA0008A14C4F3072567F3C6055C80DD70EBD189
:103CB0004FF0405500221F4C1F4B85F8A72084F879
:103CC0002F9083F82F90077DCFB14FF0010E04683D
:103CD000DFF85CC0013C14F8013F1C2B0CF80320FA
:103CE00002F1010209DD95F8A7801D3B0EFA03F3EE
:103CF00043EA0803DBB285F8A730BA42EBD10D46A0
:103D000004463146FFF7CEFED5F80130204659680B
:103D1000DA68C979074BFFF7CFF80120BDE8F88FC3
:103D200008F1010882F82780A2E70846704700BF23
:103D30004C00046098060460C8060460F0B40025D6
:103D40004FF040530326D0F8011001248A684D74C7
:103D50001778042083F82C7157784FF4C07C83F8CF
:103D60002D71977983F82A71177A83F82B719778D8
:103D700083F82E71D27883F82F21D1E900211778AA
:103D800083F8257183F88E60C9780F27491B18BF07
:103D9000012183F8841083F8814083F8805083F8F0
:103DA000AE0083F8AF00557893F8891085EA0406D1
:103DB00066F30511022683F8891093F8A11065F3C4
:103DC000041183F8A11083F88D0083F8B04083F8C4
:103DD000C570A3F8C8C083F8CC60507A517983F8D5
:103DE0000001907883F80501D07883F80A0183F800
:103DF0000D11117983F81011117A83F8DA10D27944
:103E000083F8A020F0BC00F019BE00BF012138B536
:103E10004FF04053D0F80140084693F8415100F06C
:103E2000B9FB637C074903EB0313EDB200EBC3005E
:103E300001EB0541882215F093FC637C0133637428
:103E400038BD00BF80080160D0F801305B689B7905
:103E50004BB3F0B44FF0C04784B0DFF84CC004AEB1
:103E6000002568466A463B46002153F825408833C2
:103E700042F8044B96422144F7D13C4650F8043BAB
:103E8000A1EB43035B10904244F8253004F1880411
:103E9000F4D10135222DE4D107F508776745DFD14C
:103EA00004B0F0BC70477047800800604FF040538A
:103EB000F0B503260025D0F801400127A2680420B0
:103EC00011784FF00F0C83F8E010517883F8E1106F
:103ED000917883F8E210D17883F8E310917983F830
:103EE000E610127A83F8E720626883F88E60D27851
:103EF000521B18BF012283F8842083F8817083F855
:103F0000805083F8AE0083F8AF00226893F88910E0
:103F1000547884EA070E6EF305114FF0200E83F8F3
:103F2000891093F8A11064F3041183F8A11083F8A9
:103F30008D0083F8B07083F8C5C083F88760A3F85C
:103F4000C85083F8CCE0517A83F80011917883F857
:103F50000511D17883F80A11117983F81011117ABB
:103F600083F8DA10D27983F8A020BDE8F04000F0A1
:103F700065BD00BF4FF04053F0B403264FF0000C76
:103F8000D0F8010001258268017F147801EB41011E
:103F900083F8E040547883F8E14097788C0083F808
:103FA000E270D178042783F8E310917983F8E61062
:103FB000127A83F8E720426883F88E60D278B2EBF9
:103FC0000C0218BF012283F8842083F8815083F803
:103FD00080C0026893F88910507880EA050C6CF371
:103FE00005114FF00F0C83F8891093F8A11060F3BE
:103FF000041183F8A11083F88D7083F8B05083F812
:10400000C5C083F88760A3F8C84083F8CC50517AC4
:1040100083F80011917883F80511D17883F80A119B
:10402000117983F81011117A83F8DA10D27983F8B4
:10403000A020F0BC704700BF2DE9F04F95B006AF4F
:1040400007F138056A4CDFF8B8C145F8300D07F1C3
:10405000240607F1140894E80F0088E80F0007F120
:10406000600340463146C8E9025C7B63FCF708F90F
:1040700094E80F005F4C86E80F00304607F13401EA
:10408000C6E90254FCF7FCF8012000F045FD0028C9
:1040900000F0A7800021E9460A46BB6805461C7D62
:1040A000D0F8010093F815E0D0F804C00368C7E920
:1040B000034E04FB0EFA9CF802403C605C78597099
:1040C0007C604D4C02F1140304EB43035988013228
:1040D00041F4F861112A5980F4D16A460AF10703C4
:1040E000DB08A2EBC3039D4606AC0169524620469D
:1040F0009CF801B015F034FBBAF1000F09D023464B
:1041000004EB0A0113F8012B04328B4203F8012C53
:10411000F8D148F0010346F00106CDE900635246AC
:1041200059462346012002F007FFD7E903214FF04B
:10413000000A40F222300123DFF8C8802F4E05909C
:104140000093CDE901AACDE9036823466420FEF778
:1041500089FDD7F810B0D34547DDD646D7E9020A26
:10416000BAF1000F0EDD0022037DD5F801100EFB21
:104170000323496914F803C0895C01326144524544
:10418000E154F1D10EF1010EDE45E9D12146FFF7F0
:10419000D3F8D7E9032140F22D3C4FF0000A01206B
:1041A0002346CDE9000ACDE9048C6420CDE902A6BE
:1041B000FEF758FD3B68104803F01F010AF1140395
:1041C00000EB43035A880AF1010A61F38A12BAF13B
:1041D000110F5A80F2D1D5F801303A791B685A7024
:1041E000CD463C37BD46BDE8F08FB868CEE700BF8E
:1041F000489901008D3300000000046084A2010092
:10420000952D000080A301002DE9F04FADF5177D3D
:1042100006AF786001200C4600F07EFC0026D0F846
:104220000130D4F801201B6854685A78B8605E7079
:10423000FA6001214FF4087207F1200094F801B0F0
:1042400015F099FAADF6880D06AB184631464FF4D5
:10425000086215F090FABBF1010F40F38E80012443
:10426000DFF83081031FC7F81080A1469846444DFF
:104270007E61DFF824A15046112221460AF1300A5E
:1042800015F079FAAA45F6D1012240F252334FF0E7
:10429000040A3C493E69039179696420CDE90191A2
:1042A0000593114607F11C030496CDF800A0FC61AC
:1042B000FEF7D8FC00F068FC00F08CFC40F25633AE
:1042C0007969314ACDE901910392059322224FF099
:1042D000C0431021CDF800A004967220FEF7C2FC66
:1042E00041464FF0C043DFF8B4E007F12002186800
:1042F00051F8046F04338642BCBF147008607345E4
:1043000002F10102F3D14FF459733A690593049213
:104310001E4ACDF8009003927A690134CDE901225A
:1043200007F12003222210216420FEF79BFCA34505
:104330009FD1D7F81080786807F12001FEF7FCFFC5
:1043400040F2693400220120BB683E7BD3F80110A3
:1043500007F120030D680E496E70CDE9012200902F
:104360000391CDE90484222210216420FEF77AFC17
:1043700007F51177BD46BDE8F08FDFF81880DAE762
:10438000A706046090A20100C0CA010084A2010037
:10439000A0A2010080A30100A700046080080060C3
:1043A00008B500F017FCBDE808400021084600F001
:1043B000F1B800BF012170B50446084600F0EAF8E4
:1043C00000210546012000F0E5F8D4F801202B1F5C
:1043D000147C011F05F1840653F8042F02FB04F23C
:1043E000B3424FEAE21241F8042FF5D100F1840103
:1043F00005F5867053F8042F02FB04F298424FEA49
:10440000E21241F8042FF5D170BD00BF704700BF24
:1044100010B572B60C4A1468A4B90C490C4B086864
:104420001160027803EBC2035B6898470422094BD2
:104430001A75BFF34F8F4FF04053012206490C729B
:104440001A709A7062B610BDFC0F00202410002074
:104450003C04002000001050842200204FF0405304
:1044600093F84121002082F0010283F8412193F862
:10447000432182F0010283F8432170474FF04053FB
:1044800010B593F82430CBB172B60E4A14689CB9BB
:104490000D490E4B08681160027803EBC2035B689C
:1044A000984701230A4A1375BFF34F8F4FF04052CC
:1044B00008490C721370937062B610BD0BF0B6FD14
:1044C000E2E700BFFC0F0020241000203C04002085
:1044D0000000105084220020002230B5264B87B007
:1044E00004461A7200292ED101A80BF053FF022CAA
:1044F0009DF804300AD1012B29D0022B04D11F4B87
:104500001F49204A0B60136007B030BD012B0CD04F
:10451000022BF9D11C4B002CF2D11C4A1C49116012
:104520001749184A0B601360EEE70023174D144833
:10453000144A15492B6003601160ACB107B0BDE8A7
:104540003040FFF79BBF08460BF01EFFCCE700236F
:104550000E4C0B480B4A094923600360116007B0F9
:10456000BDE83040FFF754BF02980CF0BBF907B02C
:10457000BDE83040FFF782BF8422002011440000D4
:1045800048100020441000207D44000094100020BA
:104590000509010001290CD007D3022903D1074BDB
:1045A00053F82000704700207047054B53F8200057
:1045B0007047044B53F82000704700BF4C10002098
:1045C000641000207C1000204FF0C04370B5584CA0
:1045D000584E594D594962682360336029601AB1B9
:1045E0005749201D08F01AF873681BB15549564801
:1045F00008F014F86B681BB15449554808F00EF8E0
:104600004F4A4FF48871534807F07CFF4D4A4FF4EE
:1046100088714D4807F076FF4C4A4FF488714C483A
:1046200007F070FFA3681BB14B494C4807F0F6FF39
:10463000B3681BB14A494B4807F0F0FFAB681BB1A8
:1046400049494A4807F0EAFF434A8821434807F0AE
:1046500059FF434A8821434807F054FF424A8821C2
:10466000424807F04FFFE3681BB14149414807F05A
:10467000D5FFF3681BB14049404807F0CFFFEB6816
:104680001BB13F493F4807F0C9FF394A502139481B
:1046900007F038FF384A5021384807F033FF384ACE
:1046A0005021384807F02EFF23691BB1364937489F
:1046B00007F0B4FF33691BB13549364807F0AEFF48
:1046C0002B691BB13449354807F0A8FF2E4A8821D1
:1046D0002E4807F017FF2E4A88212E4807F012FFB8
:1046E0002D4A88212D4807F00DFF63691BB12C4925
:1046F0002C4807F093FF73691BB12B492B4807F037
:104700008DFF6B691BB12A492A4807F087FF244AAD
:104710005021244807F0F6FE234A5021234807F091
:10472000F1FEBDE87040224A5021224807F0EABE5F
:10473000641000207C1000204C10002000008560D8
:10474000E4A30100F8A301008010002014A40100DC
:10475000501000206810002030A401006C100020D0
:104760004CA40100841000206CA40100541000200F
:104770008CA4010070100020A8A401008810002063
:10478000C8A4010058100020E8A401007410002003
:1047900004A501008C10002024A501005C1000205D
:1047A00044A501007810002060A5010090100020B1
:1047B00080A50100601000202DE9F047114C124E39
:1047C000124DDFF84CA0DFF84C90DFF84C8004F17C
:1047D000140754F8043F1BB15146204607F01EFF52
:1047E00055F8043F1BB14946284607F017FF56F815
:1047F000043F1BB14146304607F010FFBC42E8D1F0
:10480000BDE8F087641000204C1000207C100020D0
:10481000A4A30100B4A30100CCA301000048704789
:10482000000084600048704700000230F8B516466A
:104830001D4604460F46FFF785F808B10F4B1F6071
:1048400031462046FFF7E8F908B10C4B5E60069A46
:104850002946204601F0E6FC18B1084B069AC3E948
:104860000225DDE90712204601F0F6FC20B1034BDA
:10487000089A1A61079A5A610120F8BD04100020B5
:104880002DE9F04F8DB004AF0AF0D2FF02240546A7
:10489000B860982200215F4814F06DFF5E4B2A7DBE
:1048A0002968D3F8010000945C4B00F0E3FC5C4BFA
:1048B0006A7D6968D3F801005A4B009400F0DAFC75
:1048C000242200215848C7F804D014F054FF0AF0FD
:1048D000AFFF437D544D1A467B612B46073202F4ED
:1048E000FC72ADEB020D4268067D3A61046804AAD1
:1048F000FA60A5F124011A7F093B42F00A0283F80D
:1049000025208B42F7D17B69002B77D03869F96875
:1049100002460139184412F8013BC3F121038242D7
:1049200001F8013FF7D100F09DFC814600F09EFCAC
:104930008246002E6BD0A3194FF0010B984607F169
:104940001806C7F800A014F801AB08224FEA4A0184
:10495000304614F0E1FE19F90A30B96903EBC303DC
:104960002B44FA69585C0BFA02F20243A0455A54F0
:10497000E9D17B69D7F800A013B34FF0010B7B6935
:10498000FC6823447B613B6903F1FF3814F8011B89
:1049900018F8019F49000822304614F0BDFE1AF9AC
:1049A0000930B969023303EBC303FA692B44585C3D
:1049B00001320BFA02F202435A547B69A342E5D159
:1049C000D7F804D00FF028F80FF070F80EF0DEFFE3
:1049D000FDF71EFEFDF750FE1149144A144B0091DD
:1049E000B8681449CDE901320B4B134AFFF71EFF9B
:1049F000FFF7EAFD2437BD46BDE8F08F00F032FC3A
:104A0000814600F033FC8246002ED9D093E707F1AF
:104A10001806B2E700000460A40300204C2F002019
:104A2000D4030020B42600207C270020C8030020E7
:104A3000D0010020540A0020980A002008B50BF08D
:104A400027FA054B1B78984204D01846BDE8084069
:104A50000BF000BA08BD00BF3804002010B50BF001
:104A600017FA04460BF008FA844203D0BDE8104060
:104A70000BF0F0B910BD00BF2DE9F04100248046D5
:104A8000104B0E46202221460F481C6014F073FE86
:104A9000A04514DD2146013E0C4D0B4F06EB080CE2
:104AA00016F8014F0A4B53F8042F1078A04204BFA8
:104AB00047F821200131AB42F5D16645F0D1BDE880
:104AC000F08100BFFC0F00202410002020100020E7
:104AD0000010002070B50E4D2C68B4B1206803782A
:104AE0000A2B12D80B4E56F833309847636863B1DF
:104AF0002B682268191D29603AB15868037806EBC3
:104B0000C30673689847012070BD0020286070BDFF
:104B1000FC0F00203C040020074B10B403F12004DC
:104B200053F8042F1178814202D0A342F8D1002219
:104B3000104610BC704700BF00100020044B11B19C
:104B400043F820107047034A43F82020704700BF05
:104B50000C0400200D44000070B5094C094E04F10E
:104B6000200554F8040F03785A1E092A02D856F873
:104B700023309847AC42F4D1BDE87040FFF76EBFD8
:104B8000201000200C04002000210120FFF7A4BC0D
:104B900000210220FFF7A0BC01460020FFF79CBCCB
:104BA00008B50BF0BFFE002303480449044A036024
:104BB0000B60136008BD00BF4810002044100020A7
:104BC00094100020024B1868003018BF0120704775
:104BD000FC0F002008B5084908200BF03DF8FFF74E
:104BE000BBFF0BF09FFE002304480549054A036004
:104BF0000B60136008BD00BF5D440000481000203A
:104C0000441000209410002038B572B60BF08AFED4
:104C100000200E490E4A0F4B08601060186062B603
:104C20000D4B1C6884B10D4BA3F1200553F80429EA
:104C30002168914218BF5860AB42F7D1BDE83840B7
:104C4000074908200BF008B838BD00BF4810002005
:104C50004410002094100020FC0F00204010002081
:104C60005D44000008B5044908200AF0F5FFBDE8DE
:104C70000840FFF771BF00BF5D44000008B504495C
:104C8000082014F05DFEBDE80840FFF765BF00BFD7
:104C90005D440000082270B5304C314D23682A6015
:104CA000B3B118680278022A31D05A6882B1FFF78E
:104CB00011FF00283FD001232A4A1375BFF34F8FFD
:104CC0004FF040520020284908721370937012E090
:104CD00001260020244A23491672244A08751268C6
:104CE0000AB1904723681868214B027853F8323094
:104CF00098470023236010221E4B2A60D3F800211E
:104D000012071CD44FF0405300225A7070BDD0F8E7
:104D10000120567C002EC8D1154B1B6998470123F2
:104D2000104A1375BFF34F8F4FF040520E490E7269
:104D300013709370DFE701220B4B1A72DBE700223E
:104D400008240D480D49C3F8804102704FF04053CC
:104D5000C1F8402100225A7070BD00BFFC0F002036
:104D6000580900200000105084220020A4220020B6
:104D70003C04002000E100E0570900200000025040
:104D8000F0B5012A83B0164605460C461F462DDCB9
:104D90000146684614F0C0FC36B3009B3F2B1D460D
:104DA000A8BF3F25019A002B134405F03F05B8BF6B
:104DB00000253F2B1A46A8BF3F22002B4FF00001D1
:104DC00002F03F03B8BF002304F1100207EB420CCE
:104DD00009B30A19103207EB4202907965F3050016
:104DE00090710131B142F3DB03B0F0BD104607F022
:104DF00053FB044106FB04F40F2C294606DD012277
:104E0000684614F089FC0126009BC7E732466846D5
:104E100014F082FCC1E79CF8062063F305028CF8CD
:104E20000620DEE7F0B5012A83B0154604460E469B
:104E30001F462DDC0146684614F06EFC009B2DB326
:104E40003F2B1C46A8BF3F24019A002B134404F0BB
:104E50003F04B8BF00243F2B1A46A8BF3F22002BB7
:104E60004FF0000102F03F03B8BF002306F110022B
:104E700007EB420CF1B18A19103207EB420290792C
:104E800064F30500907101318D42F3D103B0F0BDA0
:104E9000104607F001FBF30744BF06416E4321466D
:104EA0002A46684654BF06F1FF36013614F034FC3A
:104EB000009BC5E79CF8062063F305028CF80620EA
:104EC000E1E700BF70B5DCF8103086B0644600251D
:104ED0009847FFF77FFED4E902320121042040F217
:104EE00097260295CDE90001054D06480596CDE9C6
:104EF00003057220FDF7B6FEA06806B070BD00BFC6
:104F0000BCA50100C8A5010070B5DCF8103086B062
:104F1000644600259847FFF75DFED4E9023201217F
:104F2000042040F2CD260295CDE90001054D06484A
:104F30000596CDE903057220FDF794FEA06806B042
:104F400070BD00BFBCA50100C8A5010030B5DCF8EC
:104F50000C3087B064469847FFF73CFE40F2634050
:104F6000002201210425A368059002920648074A01
:104F7000CDE90051CDE9032014227220FDF772FE25
:104F8000A06807B030BD00BFBCA50100C8A50100E6
:104F900030B5DCF80C3087B064469847FFF71AFE4E
:104FA0004FF49360002201210425A368059002922A
:104FB0000648074ACDE90051CDE9032014227220AA
:104FC000FDF750FEA06807B030BD00BFBCA50100D2
:104FD000C8A501002DE9F04F0D46CC1D890087B012
:104FE00024F007040A3121F0070106AFADEB040DF0
:104FF0000DF11808ADEB010D9B4606AEBC6A9DB1E4
:105000000023013800EB050E10F8011F1AB112F849
:1050100001C008F803C01CB154F8211046F8231051
:10502000704503F10103EFD112B340F21A424FF081
:10503000010A4FF00009344B0592344A5146CDE93C
:105040000332CDE9019943462A46CDF800A06420F9
:10505000FDF708FEFB6AFA6AD3F801301178D3E94C
:10506000002312780A299B7952441BD0062939D093
:10507000A4B140F23A404FF0000E01214FF0040C71
:10508000224C059022483346CDE903042A46CDE957
:10509000011ECDF800C06420FDF7E4FD0437BD46D5
:1050A000BDE8F08F009340F64A30CDE9036BCDE9BF
:1050B00001584FF4D7734FF4487102F0C1F840F231
:1050C0002A4C0420134A114B009004930392CDE91B
:1050D00001995B465146CDF814C02A466420FDF77D
:1050E000C1FDC5E7009340F64A30CDE9036BCDE939
:1050F000015882234FF4487102F0A2F840F2364C76
:105100000420054ADFE700BF44A60100BCA501005A
:1051100060A601004CA6010058A601002DE9F04F41
:105120000D46CC1D890087B024F007040A3121F018
:10513000070106AFADEB040D0DF11808002DADEB26
:10514000010D9B4606AEBC6A13DD0023013800EB5F
:10515000050E10F8011F1AB112F801C008F803C0BB
:105160001CB154F8211046F82310704503F10103D7
:10517000EFD112B340F261224FF0010A4FF0000963
:10518000334B0592334A5146CDE90332CDE90199BB
:1051900043462A46CDF800A06420FDF763FDFB6A74
:1051A000FA6AD3F801301178D3E90023127809297B
:1051B0009B7952441BD0052939D0A4B14FF42070FB
:1051C0004FF0000E01214FF0040C224C05902248B4
:1051D0003346CDE903042A46CDE9011ECDF800C0CF
:1051E0006420FDF73FFD0437BD46BDE8F08F009316
:1051F00040F64A30CDE9036BCDE901584FF4D7733F
:105200004FF4487102F01CF84FF41C7C0420134A40
:10521000104B009004930392CDE901995B465146EF
:10522000CDF814C02A466420FDF71CFDC5E70093A5
:1052300040F64A30CDE9036BCDE9015882234FF4A3
:10524000487101F0FDFF4FF41F7C0420044ADFE7A2
:105250001CA60100BCA5010038A6010024A601007F
:1052600030A60100004870474C2F002000487047CE
:10527000B42600202DE9F04F87B0406806AFD7F87C
:1052800028904578D01D20F0070009FB05F5ADEB0F
:10529000000D0DF1180A0E465046002190461C469E
:1052A00014F069FAA94541DB4FF0000B08F1FF3912
:1052B00022224FF0FF31204614F05DFA33784FFA86
:1052C0008BF0B8F1010FE0542DDD4FF0000E6FEAC6
:1052D000060C711C11F8012BA356B3F1FF3F05D149
:1052E000431CAB42ACBF00235BB2A35498421AD01C
:1052F00092FBF5F005FB1020012814BF01204FF0B0
:10530000FF30204482569A420DD00CEB01029145A9
:10531000A1EB060200F09580904501DD1846D9E723
:10532000BEF1000F4CD1BBF1000F46D0C623DFF811
:105330002CB1009300225B4645496420FDF7E4FC54
:10534000B8F1000F6CDD013EB14606EB080119F81B
:10535000013F93FBF5F205FB12324945E254F6D1C9
:105360000121CC2000223B4BCDE904B0CDE9011254
:1053700003930091234642466420FDF773FC0AF133
:10538000FF3316F8012FA256B14503F8012FF8D1CB
:1053900001210024D0253048CDF810B003905346A9
:1053A000642042460595CDE901140091FDF75AFCB1
:1053B00020460437BD46BDE8F08F4FF0010B77E77C
:1053C0000121BC200022234BDFF890B0CDE901126F
:1053D00005900091CDE9033B424623466420013EFF
:1053E000FDF740FC06EB08010AF1FF3316F8012F28
:1053F000A256B14203F8012FF8D101240021C025A3
:105400001548CDE901410390CDF810B06420534612
:105410004246059500942146FDF724FC2046C8E746
:105420000121CC2500200B4ACDE901100392CDF8D3
:1054300010B023460595009142466420FDF712FC0A
:10544000A6E79045BCDD4FF0010E184642E700BFCD
:10545000E4A5010008A60100D4A50100BCA5010037
:105460002DE9F047D2F8017006467A680D46527869
:105470009846012A19D9002815DD00244FF04C095F
:105480004D1E01E07B685A78510094FBF1F301FB5B
:10549000134315F8010F611009FB03830134FFF773
:1054A0006FFCA642EED1BDE8F0870028FBDD0024AA
:1054B0004FF04C0ADFF8249019F904306110002BEA
:1054C00006DB7A680AFB03835278285DFFF758FCF5
:1054D0000134A642F0D1BDE8F08700BF4C2F002078
:1054E00070B5644686B0DCF804200B4BFFF7B8FFBC
:1054F0004FF42876012100202368E268074D084C0C
:10550000CDE9010005960091CDE903457220FDF734
:10551000A9FB06B070BD00BF90070460BCA50100E8
:10552000B0A5010070B5644686B0DCF804200B4BD2
:10553000FFF796FF40F2D626012100202368E2689B
:10554000074D084CCDE9010005960091CDE90345D2
:105550007220FDF787FB06B070BD00BFC008046075
:10556000BCA50100B0A501002DE9F047D2F801600B
:105570001F4672685278012A1ED900281ADD4D1E76
:1055800021244FF04C0805EB000901E073685A78BC
:10559000510094FBF1F301FB134315F8010F04EBE9
:1055A000D47108FB03734910FFF73CFCA94504F1D3
:1055B000FF34EBD1BDE8F0870028FBDD0D464FF04E
:1055C0004C0A0D4C01EB000904F1220814F9013BCF
:1055D000A8EB040101EBD171002B4FEA610106DB5E
:1055E00072680AFB037352782878FFF71BFC0135B9
:1055F0004D45EBD1BDE8F087B426002030B56446B8
:1056000087B0DCF804200B4BFFF7AEFF40F26C458F
:105610000121002223680848084CCDE90122CDE988
:1056200003040595009114227220FDF71BFB07B0BF
:1056300030BD00BFF8060460B0A50100BCA50100A4
:1056400030B5644687B0DCF804200B4BFFF78CFFC5
:1056500040F2A2450121002223680848084CCDE908
:105660000122CDE903040595009114227220FDF773
:10567000F9FA07B030BD00BF28080460B0A50100EA
:10568000BCA50100F0B403268C68012527784FF0F3
:10569000060C80F8E8706778002B80F8E970A7782E
:1056A000B8BF033380F8EA70E778C3F38F0380F85C
:1056B000EB70A779D2B280F8EE70247A072780F8D1
:1056C000EF4080F88E60002690F88940096844F029
:1056D000300480F8894090F8A1406FF3041480F8FA
:1056E000A1400C7880F8A94080F8985090F88B4041
:1056F0006FF3000480F88B4080F88D7080F8B05014
:1057000080F8C56080F8815080F8805080F8AEC085
:1057100080F8AF7080F884604C7A80F89F408C7A73
:1057200080F89E4080F89C60A0F8CA3080F8CD20B8
:105730004B7BF0BC80F800318B7880F80531CB785A
:1057400080F80A310B7980F810310B7B80F8DA3061
:1057500090F8A330CA7962F3061380F8A33090F86A
:10576000A3300A7A62F3020380F8A330CB7A80F880
:10577000A0307047D0F8011008B54A684FF4F263C2
:1057800052784FF040505200FFF77CFFBDE80840D0
:10579000FFF764B9D0F8011008B54A684FF40C63FC
:1057A00052784FF040505200FFF76CFFBDE80840C0
:1057B000FFF754B949F6404301441144033149000D
:1057C00093FBF1F140F2E91070B5012200260425A7
:1057D00088B008AB43F8041D064C05900648CDE997
:1057E0000126CDE90304114600956420FDF73AFA3D
:1057F00008B070BDBCA50100A0A501002DE9F04FC7
:1058000098464C230D4603FB08F1CB1D83B023F0D3
:10581000070300AFADEB030D7960064614466846FA
:105820000A468946002113F0A6FFB8F1000F694629
:105830005FFA85FC57DD6B465C250DEB09005A7855
:105840001D7002F0EC0242F002025A704C338342A7
:10585000F5D1636893F80190BCF1000F29D00024C2
:105860004FF04C0B0123DFF88CA0013E05E04269AC
:1058700001342A436445426118DA16F8012F1AF9F7
:1058800002001F2A03FA02F50BFB0010EFDD057E74
:10589000203AAE4603FA02F2C5F30105154301347E
:1058A00065F3010E644580F818E0E6DBB8F1000FFF
:1058B00010DD00234C255524B9F1020F07D105FB5B
:1058C0000312D07C547420F001009474D07401331E
:1058D0009845F1DC7A68386B13F042FF386B0C376F
:1058E000BD46BDE8F08FBCF1000FF3D0636893F8BC
:1058F0000190B4E74C2F00202DE9F04F85B01546FC
:10590000D0F801800A7DD8F8044002AF66780868B4
:1059100003FB06F603EBC30A1146334600954246E5
:10592000FFF76CFF0AF10703D8F8044023F00703E0
:10593000C7F804D0ADEB030D94F805B00DF10809DC
:10594000484652460021647813F015FFBBF1020F60
:1059500000F0CC80BBF1040F00F0B180BBF1010F6F
:1059600000F0838052460021484613F004FF002EC9
:1059700040F3DD802C464FF0000C4A460023E1182E
:1059800012F8010B0133092B0872F8D10CF1010C4C
:10599000664509F1090904F14C04EEDC4FF0000EF4
:1059A0002846F146D8F80480D7F804D098F8064085
:1059B00004F01F0404F0030C4FEA8C1CA40800211F
:1059C00001F1100300EB430393F806A0DA790AF023
:1059D0003F0A22F0070201314AEA0C0A2243112948
:1059E00083F806A0DA71EBD190F84A300EF1010E7F
:1059F00023F01F03764580F8489080F8499080F89E
:105A00004A3000F14C00DADC002398F8049098F852
:105A100003A098F802B0504649465A4698460124D9
:105A200009EB0A0E0BEB090CAEF10A0E0CF1010C9E
:105A30005FFA8EFE5FFA8CFC01339E4285F802A06D
:105A40002C7185F803C085F8059085F806B085F8B7
:105A500007E085F81980AC7605F14C05ECDCFFF722
:105A6000A9FE0C37BD46BDE8F08F002E5FDDCB46AA
:105A70004FF0000EDFF8E0A05946DFF8D4C0002355
:105A8000022C03D0012C03D1012B01DC9E4506D052
:105A900003EBC30208781CF8022002430A700133AA
:105AA000042BEDD10CF1010CE24501F10101E6D12D
:105AB0000EF1010E76450BF1090BDDD15AE7002EF0
:105AC00035DDCC4606EBC60E1F4CCE4461461F4B5F
:105AD00013F8012F587AA34242EA000201F8012B81
:105AE000F6D10CF1090CF445F0D143E7002E1EDD90
:105AF0004C46174806EBC60C90F801E0837ACC447C
:105B00004EEA030E08300EF0F50E2146114B13F845
:105B1000012F93F809A0834242EA0A0201F8012BFF
:105B2000F5D184F801E009346445EED122E7D8F8D4
:105B30000430D7F804D0D87819799A78FFF73AFE6C
:105B40000C37BD46BDE8F08F962700208D2700203A
:105B50007C2700207B270020852700202DE9F047A7
:105B600092B0DFF8F0C002AFDFF8ECA007F12C0430
:105B700007F11C0907F1080605468846BA619AE84C
:105B80000F0089E80F00214607F16003C9E9026CA4
:105B90004846FB63FAF774FB9AE80F00DFF8BCC0D5
:105BA00084E80F00C4E9026C204607F13C01FAF7D3
:105BB00067FB0520FEF7B0FF034600210220D3F863
:105BC0000160FB60FEF7E6FC0523AA7E07F14001B9
:105BD00001F83C3DD31D03F4FC73ADEB030D02ABA8
:105BE000386101207A61BB60FEF746FFBB699847C8
:105BF000FEF7F0FF736844F001045878800106F066
:105C00004BFCB26849F001065189BB68CDE90046FA
:105C10007A6901F04DFA796928688B000A3323F01C
:105C20000703ADEB030D02ADD7E90343BA68CDE935
:105C300000342B46FFF772FAB8F1000F05D07A69ED
:105C400029464046920013F08BFD4037BD46BDE823
:105C5000F08700BFC54E000058990100E1540000D4
:105C60002DE9F04792B0DFF8F0C002AFDFF8ECA00A
:105C700007F12C0407F11C0907F1080605468846C0
:105C8000BA619AE80F0089E80F00214607F1600326
:105C9000C9E9026C4846FB63FAF7F2FA9AE80F008A
:105CA000DFF8BCC084E80F00C4E9026C204607F1AD
:105CB0003C01FAF7E5FA0920FEF72EFF0346002122
:105CC0000420D3F80160FB60FEF764FC0923AA7E80
:105CD00007F1400101F83C3DD31D03F4FC73ADEB2B
:105CE000030D02AB386101207A61BB60FEF7C4FE90
:105CF000BB699847FEF76EFF736844F0010458785B
:105D0000800106F0C9FBB26849F001065189BB6801
:105D1000CDE900467A6901F0CBF9796928688B00F2
:105D20000A3323F00703ADEB030D02ADD7E90343BC
:105D3000BA68CDE900342B46FFF7F0F9B8F1000F4F
:105D400005D07A6929464046920013F009FD403794
:105D5000BD46BDE8F08700BF094F0000589901001B
:105D600025550000F8B59B0003F10A0424F0070450
:105D700000AF002AADEB040DEC460CDDBC69ACF1C4
:105D80000405013C224414F8016F51F82660944246
:105D900045F8046FF7D11A46614613F0E1FCBD46A1
:105DA000F8BD00BF70B582B009F042FD0121044684
:105DB0000220FEF7EFFB002106460220FEF7EAFB79
:105DC0000546A27E3146920013F0CAFC2168A37EEC
:105DD000227D284600912946FFF7C4FF02B070BD1E
:105DE00038B509F025FD012105460220FEF7D2FB5A
:105DF000044600210220FEF7CDFBAA7E2146BDE825
:105E00003840920013F0ACBC70B582B009F010FDC0
:105E1000012104460420FEF7BDFB002106460420B4
:105E2000FEF7B8FB0546A27E3146920013F098FCBF
:105E30002168A37E227D284600912946FFF792FF24
:105E400002B070BD38B509F0F3FC0121054604200D
:105E5000FEF7A0FB044600210420FEF79BFBAA7E70
:105E60002146BDE83840920013F07ABCD0F801100A
:105E700008B54A684FF4DF6352784FF04050520043
:105E8000FFF700FCBDE80840FEF7E8BDD0F80110C0
:105E900008B54A6840F6280352784FF04050520047
:105EA000FFF7F0FBBDE80840FEF7D8BD2DE9F04F45
:105EB0001E464C2303FB06F5EB1D83B023F00703BE
:105EC00000AFADEB030D04468846914668462A466E
:105ED00000217D6013F04FFC002EAA466D465FDD69
:105EE0006B4642200DEB0A015A78187002F0EC0262
:105EF00042F012025A704C338B42F5D1D9F804307B
:105F0000B8F1000F93F801E02EDD00204FF04C0AAD
:105F10004FF0010CDFF89890631E07E04A690130EA
:105F200042EA0B0B8045C1F814B01BDD13F8012FBA
:105F3000C2F1210419F902101F2C0CFA04FB0AFB10
:105F40000151EBDD0C7EC2F10102A3460CFA02F214
:105F5000C4F301041443013064F3010B804581F85C
:105F600018B0E3DC002E11DD00234C246FF0550047
:105F7000BEF1020F07D104FB0352D17C507421F013
:105F800001019074D17401339E42F1DC7A68294694
:105F9000386B13F0E5FB386B0C37BD46BDE8F08F6E
:105FA000B8F1000FF2DDD9F8043093F801E0ACE766
:105FB000B42600202DE9F04F87B01C4694460B46CE
:105FC000D0F8016002AFFA607268497D5578586870
:105FD00004FB05F5CDF800C02B463246FFF766FFFF
:105FE00004EBC402D31D746823F00703C7F808D07C
:105FF000ADEB030D94F805900DF108084046002123
:10600000647813F0B8FBB9F1020F00F0D480B9F155
:10601000040F00F0B980B9F1010F7ED0002D40F3DC
:10602000EB804FF0000CFC6842460023E11812F8A8
:10603000010B0133092B0872F8D10CF1010C6545F5
:1060400008F1090804F14C04EEDC4FF0000ED7F81B
:106050000CC0F1466046D6F80480D7F808D098F80E
:10606000064004F01F0404F00306B601A408002152
:1060700001F1100300EB430393F806A0DA790AF06C
:106080003F0A22F0070201314AEA060A2243112997
:1060900083F806A0DA71EBD190F84A300EF1010EC8
:1060A00023F01F03754580F8489080F8499080F8E8
:1060B0004A3000F14C00DADC002398F8049098F89C
:1060C00003A098F802B0504649465A469846012423
:1060D00009EB0A0E0BEB0906AEF10A0E01365FFA68
:1060E0008EFEF6B201339D428CF802A08CF804407B
:1060F0008CF803608CF805908CF806B08CF807E0FB
:106100008CF819808CF81A400CF14C0CEADCFFF783
:1061100051FB1437BD46BDE8F08F002D6CDDAB1C84
:106120007D60C3464FF0020EA4461D46DFF8F09096
:106130005846374CAEF1020A0023BCF1020F20D0C2
:10614000BCF1010F07D1012B05DD022B0CBF002292
:106150000122524505D003EBC3020178A25C0A4339
:1061600002700133042BE8D10134A14500F1010094
:10617000E2D10EF1010EAE450BF1090BD8D17D68CD
:106180004FE79E45E7D1ECE7002D35DDC44605EB32
:10619000C50E204CC64461461F4B13F8012F587A98
:1061A000A34242EA000201F8012BF6D10CF1090CDE
:1061B000F445F0D135E7002D1EDD4446144805EBCB
:1061C000C50C90F801E0837AC4444EEA030E08300F
:1061D0000EF0F50E2146114B13F8012F93F809909C
:1061E000834242EA090201F8012BF5D184F801E06B
:1061F00009346445EED114E77368D7F808D0D8782D
:1062000019799A78FFF7D6FA1437BD46BDE8F08FB2
:106210007C270020962700208D2700207B27002048
:106220008527002089B182B138B505461446084655
:1062300002232946064AFFF75FFB20462946022330
:10624000044AFFF7B7FE012038BD0020704700BFA9
:1062500090070460F806046089B182B138B505463C
:106260001446084602232946064AFFF745FB204606
:1062700029460223044AFFF79DFE012038BD002075
:10628000704700BFC0080460280804602DE9F04F83
:1062900091B0DFF8F0A002AFDFF8ECC007F1240402
:1062A00007F114053E1D804689463A619AE80F00C1
:1062B00085E80F00C5E9026C2846214607F1600316
:1062C0007B63F9F7DDFF9AE80F00DFF8C0C084E8D0
:1062D0000F00C4E9026C204607F13401F9F7D0FF42
:1062E0000620FEF719FC034600210320D3F801B075
:1062F000BB60FEF74FF9062398F819A007F13801A3
:1063000001F8383D0AF1070303F4FC73ADEB030D0C
:1063100002ABF86001207B60FEF7AEFBDBF80430D7
:1063200045F00105587844F00104800106F0B4F806
:10633000DBF808207B6851894FEA8A06CDE90045E1
:10634000524600F0B5FE06F10A0303F4FF63ADEB1D
:10635000030D02ACD7E9025398F81510D8F80400E1
:106360007A68CDE900352346FEF734FEB9F1000F17
:1063700004D032462146484613F0F2F93C37BD4678
:10638000BDE8F08F589901004D4F0000FD55000009
:106390002DE9F04F91B0DFF8F0A002AFDFF8ECC0CC
:1063A00007F1240407F114053E1D804689463A6131
:1063B0009AE80F0085E80F00C5E9026C28462146DF
:1063C00007F160037B63F9F75BFF9AE80F00DFF8E2
:1063D000C0C084E80F00C4E9026C204607F1340114
:1063E000F9F74EFF0A20FEF797FB03460021052030
:1063F000D3F801B0BB60FEF7CDF80A2398F819A0D6
:1064000007F1380101F8383D0AF1070303F4FC7382
:10641000ADEB030D02ABF86001207B60FEF72CFBB7
:10642000DBF8043045F00105587844F001048001A0
:1064300006F032F8DBF808207B6851894FEA8A06BB
:10644000CDE90045524600F033FE06F10A0303F49D
:10645000FF63ADEB030D02ACD7E9025398F81510BA
:10646000D8F804007A68CDE900352346FEF7B2FD7E
:10647000B9F1000F04D032462146484613F070F9B6
:106480003C37BD46BDE8F08F58990100914F0000A0
:106490004156000070B582B009F0CAF901210446E6
:1064A0000320FEF777F8002106460320FEF772F876
:1064B0000546627E3146920013F052F96168637EB0
:1064C000627D284600912946FFF74CFC02B070BD62
:1064D00038B509F0ADF9012105460320FEF75AF859
:1064E000044600210320FEF755F86A7E2146BDE8E8
:1064F0003840920013F034B970B582B009F098F9C1
:10650000012104460520FEF745F800210646052036
:10651000FEF740F80546627E3146920013F020F9FE
:106520006168637E627D284600912946FFF71AFC68
:1065300002B070BD38B509F07BF94FF04053054605
:1065400093F8414101210220FEF724F8E4B2AA7E2B
:106550000349240421449200BDE8384013F000B9F7
:106560007009016038B509F063F94FF040530546F2
:1065700093F8414101210320FEF70CF86A7E04499B
:10658000E4B201EB04419200BDE8384013F0E8B8F2
:106590000809016038B509F04BF94FF04053054642
:1065A00093F8414101210420FDF7F4FFE4B2AA7EF3
:1065B0000349240421449200BDE8384013F0D0B8C8
:1065C0007009016010B509F033F94FF04053012113
:1065D00093F841410520FDF7DDFF0449E4B201EBEA
:1065E00004415022BDE8104013F0BAB80809016018
:1065F00038B509F01DF9012105460520FDF7CAFF50
:10660000044600210520FDF7C5FF6A7E2146BDE84E
:106610003840920013F0A4B808B5FEF7DBFABDE8E5
:10662000084000210220FDF7B5BF00BF08B5FEF706
:10663000D1FABDE8084000210420FDF7ABBF00BF40
:1066400008B5FEF7C7FABDE8084000210320FDF7B2
:10665000A1BF00BF08B5FEF7BDFABDE808400021A4
:106660000520FDF797BF00BF704700BFF0B5B5B07C
:106670003A9E0546F8B1421E022A01D935B0F0BD56
:106680006427194602A8442213F06AF8306871683A
:10669000B268F36813AC0FC430697169B269F36909
:1066A000184E0FC4009702AB2A463468002101201F
:1066B000A04735B0F0BD0F4614460146C82202A8D7
:1066C00013F059F8396802A8882213F049F82468B1
:1066D00024AE04F14007354620686168A268E3688B
:1066E0001034BC4206F110060FC5F4D10022C821B7
:1066F00004480091046802AB11460120A04735B060
:10670000F0BD00BF04D50100F8B50023114C1946B7
:10671000236063603C22104813F02DF800F0EAF982
:106720004FF480620D4B0E490E4E0F4C9B688860F3
:1067300030689A606368851C9847A3680746984745
:1067400039460246284613F00BF823693468984707
:10675000E080F8BD60250020BC2700203006002026
:10676000F4190020D805002004D50100F0B51E4C16
:1067700085B02678174686421946DDE90A23054684
:10678000DDF830C018D0A378AB4201D005B0F0BD21
:10679000E378002BFAD0CDB94FF4086001210A90BC
:1067A0002A460846114B1B680393039C104BA446D2
:1067B00005B0BDE8F04060476678002EE3D0CDF824
:1067C00000C010321031FFF751FFDCE76B1E022BC7
:1067D000DCD84FF488600121044C0A9024683B46C1
:1067E0002A4608460394E2E76025002004D501000C
:1067F000980004602DE9F04F5A4C85B00E9D6479E5
:106800000295DDE90F56019614B905B0BDE8F08F89
:10681000914600240090A0228846534800219A46C1
:10682000DFF850B112F0A7FFA646504A4E4805F1D6
:10683000FF3CCDF80C904FE0002B0CBF012302234E
:106840004FF487664370009B047033F91430029D47
:1068500006FB03F38BFB03761E44DB17C3EBE62337
:106860004FF4166655F82450438038F91430C5F3B8
:10687000072706FB03F38BFB03961E44DB17C3EBD2
:10688000E6238380039B33F81460EBB2FF1AC5F351
:106890000743C3EB1565AF42C6804FF04D034BDD98
:1068A00003FB07F7BF1107814581019B3AF814509C
:1068B0001B5D85818373009B0EF1010E33F914304B
:1068C000138038F91430538001340A2C117100F10F
:1068D000100002F1060235D01CF8011F13790029BF
:1068E000AAD1002BF0D04FF48766B2F90050B2F96C
:1068F000023006FB05F54FF4166606FB03F38BFB2F
:1069000005678BFB03964FF003091E44DB17C3EBAF
:10691000E623019E047080F80190365D2F44ED1748
:10692000C5EBE725C1800181418181810EF1010E16
:10693000458083808673C7E703FB05F5AB110381B0
:106940004781B2E70A4B03221B6802210093009C97
:106950000120A446044BCDF838E005B0BDE8F04F67
:10696000604700BF60250020A4100020BC27002045
:1069700004D501008100088010B584B003F044FF05
:106980000E4A4379117899420CD043790C49DBB215
:1069900013700A6803923BB90221009308461A4615
:1069A000039CA04704B010BD0023022100930846B9
:1069B0000122039CA04704B010BD00BF9810002026
:1069C00004D5010010B582B003F01EFF437F43B130
:1069D0000023054C43771A46009319462468022089
:1069E000A04702B010BD00BF04D5010030B583B090
:1069F00003F00AFF084CC37F22789A420AD0002392
:106A0000C07F0649C0B202460D682070009306217F
:106A10000220A84703B030BD9A10002004D5010021
:106A200030B583B091B1838B028B19491A44782A0F
:106A30000B781FDDB0F924001BB30024154A146045
:106A4000013BDBB202200B70106004E00846114AE3
:106A50000F4B11601970104C2378834208D000232B
:106A60000E49024600930D68207007210220A847B6
:106A700003B030BD0020074A1060002BE0D1106841
:106A8000E9E70123034AA0281360F8DD2323D9E7AF
:106A9000A01000209C1000209910002004D50100B7
:106AA000002300B583B0019300F024F80378054A71
:106AB0008DF80430019BC3F30013137003B05DF82D
:106AC00004FB00BF9B10002010B582B0FFF77AFFD7
:106AD000FFF752FFFFF78AFFFFF7E2FF00230449A9
:106AE00000930C681A4604210120A04702B010BD93
:106AF00004D5010000487047441100204FF4806025
:106B0000704700BFF9F7BEBB12F02ABE12F033BEC9
:106B10000C2330B5012583B0054C00930022054BB2
:106B2000054964202570FCF7EFF803B030BD00BFC5
:106B300022230020E8A60100F8A601002B23F0B5CF
:106B400005460E461446144F8BB0009300223B4678
:106B5000124964200994CDE90756FCF7D5F84FF0A7
:106B60002E0C0121002004220D4BCDE901100092D2
:106B70000393CDE9047C07AB03226420FCF772F891
:106B8000003418BF0124074B03EB450203F81560DE
:106B900054700BB0F0BD00BFE8A601008CA6010048
:106BA000C0A6010060250020132330B583B0044641
:106BB000009300220B4B0C496420FCF7A5F80B4A0C
:106BC00040F2F1211346104623F8021B0C212568E0
:106BD0006468C2F802505C6003B0BDE8304003F066
:106BE00047BE00BFE8A601006CA60100582E002099
:106BF0000048704714A701001EF0040F0CBFEFF30C
:106C00000880EFF309808169004A1047E9FE00001F
:106C1000684620F007018D4601B401BC85467047E7
:106C200072B61EF0040F0CBFEFF30880EFF309807B
:106C3000004A1047B96D000072B61EF0040F0CBF79
:106C4000EFF30880EFF30980004A1047BD6D0000A4
:106C500072B61EF0040F0CBFEFF30880EFF309804B
:106C6000004A1047C16D000072B61EF0040F0CBF41
:106C7000EFF30880EFF30980004A1047C56D00006C
:106C8000684620F007018D4601B401BC8546704777
:106C9000684620F007018D4601B401BC8546704767
:106CA000684620F007018D4601B401BC8546704757
:106CB000684620F007018D4619B507232B4CB020FC
:106CC000237309F0C7F80021294A2A4BA1709A4280
:106CD0000CD2111D03335B1A23F0030326480B4427
:106CE00050F8041B42F8041B9A42F9D1234A244B62
:106CF0009A420CD2111D03335B1A23F0030321487F
:106D00000B4450F8041B42F8041B9A42F9D11E4A66
:106D10001E4B9A420AD20020111D03335B1A23F046
:106D200003030B4442F8040B9342FBD1EFF30882B8
:106D3000174B9A4205D94FF0CD3143F8041B9A42C4
:106D4000FBD84FF6FF72094B1A8708F037FF08F09F
:106D500041FF1049002008F0DDFE044600F05EF817
:106D6000844200D0FEE70AF031FEFBE7000010503D
:106D70000056002080560020800000000000002007
:106D8000E40F0020E8D50100E40F00200C250020CE
:106D9000942F0020FCFB0100684620F007018D467F
:106DA000002201B5034B1A6009F00EFCBDE801405A
:106DB0008546704710E000E0704700BF704700BF95
:106DC000704700BF704700BF014B93F82100704728
:106DD000C0FB0100014B187E704700BFC0FB0100E3
:106DE000014B587E704700BFC0FB0100014B987EED
:106DF000704700BFC0FB0100014BD87E704700BF49
:106E0000C0FB0100014B986A704700BFC0FB010046
:106E1000014BD86A704700BFC0FB0100014B1868E6
:106E2000704700BFFCFB01002DE9F04F4FEA820BD9
:106E300083B00BF10A0525F0070500AFADEB050D9A
:106E40006D463B604B68D1F80080064614468A4682
:106E50007B60C0475A462846002112F08CFC012274
:106E600002FA06FB1BF1FF3B17D37B68984781466C
:106E7000BBF1000F00D0C047002CF3DDAC46002171
:106E80005CF8043B59F8042B013113448C424CF854
:106E9000043CF5D11BF1FF3BE7D2002C09DD29466C
:106EA000002251F8043B01323341944241F8043C42
:106EB000F7D1DAF808302946204698473A68DAF8D8
:106EC0000C302946204698470C37BD46BDE8F08F68
:106ED00001322DE9F04191FBF2F404FB121282B071
:106EE000DDE90A67DDE90C4512B102B0BDE8F081C9
:106EF0002022804600921846DDE90812012305F0A1
:106F000031FAB8F1000FF0DD04EB48020FFA87FE0A
:106F10000FFA86FC08E0634655F8041B944203FB15
:106F2000101345F8043CE0D034F9023BB342F2DCE4
:106F3000BB42B8BF7346EFE72DE9F04F14469846C1
:106F4000D31D85B023F0070300AFADEB030D950013
:106F500079608346002168463A6012F00CFC05F126
:106F60000A0323F0070341462046EA46ADEB030D32
:106F7000BB6B9847FB6B9847E94601462A46484653
:106F800012F0EEFB002C40F38880434608EB04012E
:106F900013F8012B01328B4203F8012CF8D1414642
:106FA0003868BB6B9847FB6B9847043D04384D44E9
:106FB000A9F10403514642464FF0FF0C4FF0010E79
:106FC00008E0AB4281F800E01C6001F1010102F130
:106FD000010211D050F8044F53F8046FA642F0DBC1
:106FE0001478AB4204F1FF3481F800C0147001F151
:106FF000010102F10102EDD13B685E1E56440AF127
:10700000FF334FF0000A1D46C4461C46012209E02A
:10701000786888420FDB00228CF80010B4420CF133
:10702000010C0ED014F9011F0029F7D09CF80000C4
:1070300001448B45ECDDB44284F800A00CF1010C56
:10704000F0D182BBC7E9023241463868BB6B984732
:10705000FB6B9847D7E9023284469E4605E049F823
:107060002200AC4202F1010215D015F9011F0029DE
:10707000F7D05CF8220059F822308342EFDB18F891
:107080000200AC42A0EB010108F8021085F800A054
:1070900002F10102E9D17346B5E7BB6B414638689E
:1070A0009847FB6B98471437BD46BDE8F08F00BF8B
:1070B0002DE9F04F012683B00138B2F100080D46EA
:1070C00000AF9B4606FA00F640F39880013B03EBC5
:1070D0000800F1B203F8011F8342FBD1761000F0E3
:1070E0009D804FEA880AAAF10409C7F804A07C6BC6
:1070F000D7F830A059464046D047A047B8F1000F16
:1071000013DD5B465FFA86FC011F00EB090E51F8A8
:10711000040F1A78A842A2EB0C00D6BF6244187084
:107120001A70714503F10103F1D17610E2D159468D
:1071300040463B6BD7F804A098477B6B98470AF111
:107140000A0323F00703ADEB030DB8F1000F02466D
:107150006C465CDD043C161F20463146AAF1040A49
:1071600002EB0A0C51F8043F5B1B8C4540F8043FCE
:10717000F8D1D9465B46304602EB0A0E50F804CFF0
:107180001978AC4501F1FF3CD6BF013183F800C04E
:107190001970704503F10103F0D1594640463B6B2D
:1071A0007A6098477B6B98477A68924456F8043F18
:1071B00054F8042F5B1B002A83EAE371A1EBE3710F
:1071C000B8BF52428A420ADA99F80020002B02F135
:1071D000FF31D6BF013289F8001089F80020B2458E
:1071E000236009F10109E1D1594640463B6B9847BC
:1071F0007B6B98470C37BD46BDE8F08F76107FF467
:1072000070AF3B6B5946404698477B6B98473B6B4A
:107210005946404698477B6B9847E5E759464046B4
:107220003B6B98477B6B98474FEA880A0AF10A0341
:1072300023F00703ADEB030D02466C468AE700BF5F
:107240002DE9F04F83B00D9EDDE90F9C002E40DD4F
:10725000DFF88480DF021D0388FB073B88FB0538CD
:107260000E9BFF17ED17013B5200C5EB681500247C
:1072700000EB01084FF47A7E41F2301AA7EB6B174E
:107280001E44411A01921AE008FB00FB59F8240041
:10729000019A381890FBF2F00EFB00F090FBF5F02D
:1072A0000EFB0BFB0AFB00F00C9A9E4202FB10B097
:1072B00090FBF1F04CF8240004F1010409D013F81C
:1072C000010F0028E0D19E424CF8240004F1010493
:1072D000F5D103B0BDE8F08F1F85EB512DE9F04FDC
:1072E00017469A460646850097B02A46DDE92149A9
:1072F00008468846002112F03EFA2A460021384608
:1073000012F039FA72000021504612F034FA324677
:107310000021209812F02FFA2A464846002112F048
:107320002AFA002E40F39980209BCE460993002331
:107330000193249B221FC3EBC3730F925B002A446B
:10734000CDF814A00B9711920E93CDF818800F9BD7
:1073500053F8041F0F934FEA116BC1F307435B45CA
:107360000C9156D80123249A26989A400BFB0202CE
:107370000292DDE924200BFB02020792019A93405E
:107380000A93CBB20093C1F307230D930D99009B91
:1073900099422FDB079B4FF0010C5E18DDF82C8023
:1073A00005E090065CD4009B01398B4222DC16F884
:1073B0000129019B9A42F4D1029B069C33F91120CA
:1073C0002368059D01FB023328882360D8F800302C
:1073D00010440BFB0233C8F800302880099803786A
:1073E0009342E0DAFF2AA8BFFF22009B01398B42BB
:1073F0000270DCDD029A0E990C9B0A4402922499D9
:10740000079A0BF1FF3BC3F30743521A5B45079200
:10741000BCDD059BB3F900205AB106990B685B02ED
:1074200093FBF2F30B600B990B685B0293FBF2F298
:107430000A60019B0F9A01330193059B0233059368
:10744000069B043306930B9B04330B93099B013378
:107450000993119B93427FF47AAF17B0BDE8F08F88
:1074600000234FF601701C464A4D16AF2D7847F8A1
:10747000040D03952598484D0493149500EB010ADB
:1074800002F00F05089245FA03F0C2071AD514AAB4
:10749000D056249A584402FB00A013F90790039A8F
:1074A00010F809900CFA09F0914540EA040009D25D
:1074B000A04207D0049A044616A81044013200F8EE
:1074C0000C9C04920133042BDDD10A9B089A1C42C8
:1074D0003FF469AF029B33F911300893D30613D4FC
:1074E0009DF804307370069D08982B68059F01FB7A
:1074F00000333A882B60D8F8003002440BFB00338D
:10750000C8F800303A804EE74FF00009049B0DF1B7
:107510004B005A1E914500EB03070DF14C0A18462B
:10752000CDF840B01CDA09F10109484514DD544694
:107530009AF800B0039214F8013F9B452ABF1D46FC
:107540005D465B465EF825200CFA03F31343A74221
:107550004EF82530EFD1039A91450AF1010AE2DB9A
:10756000049BDDF840B0032B0BD0042B05D0022B7D
:10757000B9D1089B5B100893B5E7089B9B10089353
:10758000B1E74AF6AB23089A03FB02F35B140893B6
:10759000A9E700BF2CA70100000001FF0288014BF2
:1075A0001A807047441500202DE9F0414DF6301C3B
:1075B0004EF23437184C069E94F8008094F801E09F
:1075C00006EB410611F1FF3123D336F9024D002CB1
:1075D000F8D032F9114033F9115068B905F58075CA
:1075E00004F58074B8F1000F01D0C5F50055BEF167
:1075F000000F01D0C4F588440CFB05F507FB04F42B
:107600002D14241422F8115023F8114011F1FF31E8
:10761000DBD2BDE8F08100BF441500202DE9F04F1A
:1076200040F6FF7CDDE9097640F6FE7849F2D6693E
:1076300044F2DA3EACEB060B0344A8EB060AACEBD3
:10764000070C10F1FF3020D313F8014D002CF8D0B7
:1076500031F9105032F9104009FB05F50EFB04F426
:107660002D14BD424FEA244413DDAC4501DCA8EBE8
:107670000705B4420BDDA345D8BF544621F810508E
:1076800022F8104010F1FF30DED2BDE8F08F344612
:10769000F4E73D46EDE700BF0288014B1A807047D2
:1076A0004815002000231849184A70B41848194E8C
:1076B000194D1A4CC1E900330B81C2E90033184956
:1076C0001381184AC6E90033C6E902333361C5E9BC
:1076D0000033154EC5E902332B61C4E90033C4E918
:1076E00002332361C0E90033C0E902330361C1E919
:1076F0000033C1E902330B61C2E90033C2E902334E
:107700001361337070BC704788190020D8180020AE
:107710000C190020341900205C19002020190020C9
:10772000E4180020F8180020841900202DE9F04FFB
:107730008BB09DF854607A4CCDE90260277865786B
:10774000784C01932478029B92469C4238BF754A3C
:107750000E468DF824708DF8255038BF1370149D97
:10776000092405F081F8039B0490DFF8D091DFF83D
:10777000D081DFF8D0B12544123603F1120739E089
:1077800018F804300AAA0A4412F804CC0133DBB218
:1077900065489C4508F804304FEA440230F914006B
:1077A0003BF914E0009745D20023297808F804300B
:1077B00009F804105D4B98525D4B5B4823F802E0DA
:1077C000009BB3F900308352B6F9003059482BF8CA
:1077D00002303AF914308352019B574833F9143080
:1077E0008352013C631C05F80119A7F10207A6F1B9
:1077F00002063CD005F0E0FD58B13AF91430002BF8
:1078000007DDB6F90030B3F5007FBCBF01238DF86A
:10781000243019F804102B788B42B1D10023620078
:1078200008F80430404B3BF902E0985E039B134498
:107830000093BFE7002BBDD09DF858302BB92B78B3
:107840001BB9384B1B78012B18D038803BF902301C
:107850003380384B01989B5E2AF81430364B9B5E80
:1078600020F8143018F80430002BBAD1DAE7029B64
:107870000BB92C4A13700BB0BDE8F08F049B132B8F
:10788000E3DC2A4B9B5E0093294B33F902C0009B3B
:1078900013B9BCF1000FD8D0009BC31A002B06937C
:1078A000B8BF5B420593AEEB0C0300930793059BB7
:1078B000772B2EDD41F6941CA0F1C9039BB26345E2
:1078C000C3D86FF4C87343F6381C73449BB2634546
:1078D000BBD841F6243C069B03EB430303EBD37375
:1078E00000EB63030093013B6345AED8079B03EBBA
:1078F000430C0CEBDC7C0EEB6C0E43F6584C0EF19B
:10790000FF336345A1D8BDF800303B80A6F800E006
:107910009FE7009B002BB8BF5B42772B95DDC9E743
:10792000481500208419002034190020E418002094
:10793000F8180020201900200C19002088190020B8
:10794000D81800205C190020F0B40C781A4D14B33C
:1079500005EB8406B6F8446086421CDD0027661EEF
:10796000F6B21F700E702F6C013FA74206DD05EBCB
:107970008406B6F84C60B04217DC0E78B44218BFEB
:1079800014701A780132D2B21A7069698A4200DD25
:107990001970F0BC70472E6C013EA642F1DD05EB7C
:1079A0008406B6F84C60B042E7DD0020661CF6B2F3
:1079B00018700E70E2E700BF9404002001467422A4
:1079C000014811F0CDBE00BF9404002000224FF406
:1079D00080710848084B007D1A61987583F8320061
:1079E000DA759A61DA6283F833205A6399821986CC
:1079F000704700BF9404002040260020F0B49DF89A
:107A0000104024B33B4F3C4D012C18BF00272C786D
:107A1000012C21D0002C4BD1D7F800C0BCF1000FB5
:107A200064DDBE88B04247DB23463A4605E016894E
:107A30002346864202F104023EDC5C1C6445F6D11A
:107A4000DAB20A7007EB8303D888F0BC70472A4D7E
:107A50002A4F2C78012CDDD1686991F800C00028EC
:107A600016784FF0000408DD05F1140202EB8000E7
:107A700052F8041F82420C44FAD11878A0B30021B6
:107A80001F4A02EB800052F8043F90421944FAD199
:107A900007EB8603B44507EB8C07D888FB881BD916
:107AA0001B1A01FB03F191FBF4F1F0BC0844704791
:107AB0004FF47A70F0BC70470A78A242134608DD92
:107AC0004FF0640C6D780CFB00F006FB05F6B0423D
:107AD000B7DCE2B22346B4E7C31A01FB03F191FB22
:107AE000F4F1F0BC401A70470146D1E72246234624
:107AF000A7E700BFF004002094040020D804002071
:107B0000A80400202DE9F04FC600351AAD008E4CB8
:107B100005F1180787B004EB0709002900F0FD8084
:107B200004EB050EDEF810100A2940F3E380D3F8C9
:107B300000C00293331A9B000492109A04EB0308CE
:107B40008346E0581168D8F80430ACEB0000C91A3D
:107B50000028B8BF40420029B8BF494204F018FCD1
:107B60004FF6FF738342A8BF034698F8172005F12C
:107B7000150A29F8123098F8173005900133DBB256
:107B8000012B88BF002388F81730DFF8C081B9F8CF
:107B90000210E35B98F800200B4405F114095B1018
:107BA0001635012A0393A144A244254400F0C58060
:107BB00000222B460092494652460398FFF71EFFCB
:107BC000A6EB0B0304EB83031A6998F80C30074605
:107BD0009A42C0F286800A22A6EB0B0304EB8303D1
:107BE0001A61012052462B46009049460398FFF740
:107BF00005FFA6EB0B0304EB83031A6998F80C301E
:107C000082469A4206DAD8F81030059A9342C8BFE5
:107C1000D8F808A0049BA6EB0B0203F1010997FB1F
:107C2000F9F7029B92001B68A11803FB07FC886808
:107C3000A358C7F57A75034405FB03C3DFF810C1E9
:107C40004FEAE37E8CFB03030298CEEBA3130360A1
:107C5000109BC8681B6803FB07F74B68184405FBBB
:107C600000778CFB075E109DFF17C7EBAE172F60E8
:107C700098F80230039DAB420FDB0023C1E90233C9
:107C8000029BA6EB0B061B68B600A351109B264473
:107C90001B68736007B0BDE8F08F9AFBF9F98D6837
:107CA000C9F57A7A029805FB0AF5A3580268D21A38
:107CB00009FB02558CFB0532CB68ED17C5EBA2150D
:107CC00003FB0AFA109B8D601B684A689B1A09FB2C
:107CD00003A98CFB093C4FEAE979C9EBAC13CB60F3
:107CE000CEE7D8F81030059A93427FF774AFD8F8F2
:107CF000047076E70131CEF810100129D3F800C0E6
:107D00007FF417AF4FF00008109944F805C00968D8
:107D1000CEF80C80CEE9011809E74FF480700B4AC9
:107D200005F1100352692544E15023449880E97518
:107D3000AA75E15107B0BDE8F08F2B46524649467F
:107D40000398FFF701FE33E740260020940400204B
:107D5000D34D6210F8B505461A4C0146B0222046B4
:107D600011F0FEFC2E1D04F15C0C0FCEACE80F00F0
:107D70000FCEACE80F0096E8030005F1300704F1E0
:107D800088068CE803000FCF0FC60FCF0FC697E809
:107D9000030086E8030005F18807261D0FCF0FC6F4
:107DA0000FCF0FC697E803005C35303486E8030038
:107DB0000FCD0FC40FCD0FC495E8030084E8030076
:107DC000F8BD00BF4C1500202DE9F84F9DF8288024
:107DD00004460E4617461D4604F046FDB8F1010F55
:107DE00043D0DFF810B1DFF8109105EB44050BF13B
:107DF000300A14F1FF3438D335F9023D002BF8D0A6
:107E000056F82400DBF8583098424EDAB8F1020FE9
:107E100000B20CBF4946344904F010FBDBF858307F
:107E200056F82420D21A00FB02F003EBA01346F808
:107E3000243057F82400DBF80030984217DAB8F104
:107E4000020F0CBF4946294900B204F0F7FADBF8EB
:107E5000003057F82420D21A00FB02F003EBA013E5
:107E600047F8243014F1FF34C6D2BDE8F88FDBF8B0
:107E70002C30C0F5F0509842BBDAB8F1020F00B2D6
:107E80000CBF4946514604F0D9FA57F82420DBF8D4
:107E90002C30C2F5F052D21A00FB02F203EBA2130F
:107EA000C3F5F05347F82430A3E7DBF88430C0F57E
:107EB00084409842BDDAB8F1020F00B20CBF4946C7
:107EC0000B4904F0BBFA56F82420DBF88430C2F5E5
:107ED0008442D21A00FB02F203EBA213C3F58443DF
:107EE00046F82430A5E700BFA81500205015002053
:107EF000D41500204C15002080050020F0B4847AB1
:107F0000464B0278012C1A7021D142884449C2EBB9
:107F10000232A1FB02120226120A5A808188414DC8
:107F2000C1EB0131A5FB0121890A9980C1888672C4
:107F3000C1EB0131A5FB0121890AD98002893A49A7
:107F4000C2EB0232A5FB0252920A1A810C70027C2B
:107F5000012A4CD012B90121334A1170827C304C75
:107F60009A74B0F81320D0F81B50C2EB0232A4FB75
:107F70000212C2F30F22A3F81320B0F815202B49E8
:107F8000C2EB0232A4FB0262C2F30F22A3F8152057
:107F9000B0F81720C2EB0232A4FB0262C2F30F2238
:107FA000A3F81720B0F81920C3F81B50987FC2EB34
:107FB0000232060900F00F073D053005A0EB062050
:107FC000A5EB0725A4FB0262A4FB0565A4FB000446
:107FD000587F1E7F00EB1424154806EB1525C2F3CD
:107FE0000F220D800480A3F81920F0BC70470025F3
:107FF00002261A7481890B4CC1EB0131A4FB0121CB
:10800000890A9981C2890674C2EB0232A4FB02126A
:108010000549920ADA810D70A0E700BFFC15002027
:10802000B5814E1B49D6B9F27C2E0020782600205F
:1080300020280020002370B4124D134A13482B60EF
:108040006B60AB60EB602B61114D124C124E1360F4
:1080500053609360D3601361036043608360C360C7
:1080600003612B606B602B8123606360A360E3601E
:108070002361336073603381194670BC282207483E
:1080800011F079BB202F0020942600200C2800201E
:10809000D8260020382F00207C2600200C25002028
:1080A00030B4C0F5FF63274C0733002B2478264BF0
:1080B000BABFC0F57F620E3202469D7C3CB11C897E
:1080C000944207DD45B384B930BC02207047DC8997
:1080D00094421EDC15B9012030BC7047B3F817205C
:1080E0008A4220D91A89002AEED0184A12888A4278
:1080F000EAD8174A12888A42E6D3DB7E012B1AD0CF
:10810000022BE1D140F2FE73984294BF022001207D
:10811000E2E71C89002DD6D1002CD5D00B4A12885D
:108120008A42E6D9D0E7B3F81920C2F57F620F3250
:108130009142D0DDD6E740F2FE7398428CBF022018
:108140000120C9E77C2E0020FC15002078260020A5
:10815000202800202DE9F04F8FB0834605A8CDE9F7
:1081600000238A46189F02F0BBF89DF81D30022BB1
:1081700000F0B0805C4B1B78002B00F0AB8000243B
:10818000A146DFF88081594AABF1020BAAF1020A3D
:1081900039783BF9025F3AF9026F18F8013B002980
:1081A00040D0B1B2A8B2CDE90232FFF779FF009B0F
:1081B000012833F914E0019B33F914C0DDE90232E0
:1081C0007CD0022824D1115D19BB4FF0010111555B
:1081D0005BBB4749474851F8241020F81450481C0D
:1081E0000121454D25F81460444D25F814E0444D17
:1081F00025F814C03B703E4B43F8240001340A2C90
:1082000008F8011C07F10107C2D10FB0BDE8F08FDB
:10821000115D0129DCD0012B07D0354B115D43F8EE
:108220002490EBE7012B1155F7D1334B33F91410A0
:10823000304B761A2E4906FB06F651F8240045F617
:10824000111133F91430ED1A05FB05658D424FEA23
:1082500044034FEA84062ADD4FF0020111552449F8
:108260002F2841F824904FF00201C7DC214D224E07
:10827000E85E009DABF80000F05EAAF800001F4821
:10828000185E25F814001E48019D185E25F814009C
:108290004FF0010519483D7023F80090154D18481E
:1082A00025F8039026F8039023F80090A6E72F28DE
:1082B000115D07DC31B90E488151D7E74FF002015B
:1082C0001155A8E701290AD1094B013087F8009020
:1082D000985193E70FB0BDE8F04FFFF7ABBE044BEA
:1082E00043F806908AE700BFFC150020D82600203E
:1082F0000C250020202F0020382F0020942600205D
:108300000C2800207C260020C0F5FF630733002BDB
:10831000344B30B41D78BABFC0F57F640E340446C8
:108320002DB99A7C002A39D1104630BC70472E4AAC
:10833000127862B364295A8843D9914243D89A8803
:10834000A24243DC9A7C002A35D0B3F813208A423B
:1083500006D8B3F81520C2F57F620F3291422ADDAC
:108360002522224D2D888D4228D8214D2D888D42E1
:1083700024D3A24222DADB7E012B2BD0022B1DD18B
:1083800040F2FE73984294BF02200120CDE79A8903
:10839000A242E5DC9A7C002AD7D10CE0B3F8132086
:1083A0008A42DDD8B3F81520C2F57F620F329142C0
:1083B000D6DC2846B9E7012030BC7047022030BC2B
:1083C00070479142BED9DA88A242BBDD252A28BF78
:1083D0002522C6E740F2FE7398428CBF022001209E
:1083E000A3E700BFFC1500207C2E0020782600208B
:1083F000202800202DE9F04F8BB0064601A80F463B
:1084000001F06EFF9DF80D30022B38D0204B1B7809
:1084100073B300244FF00209A0464FF0010A149BE9
:10842000DFF870B05D1E15F8013FDBB137F81410AE
:1084300036F81400FFF768FF012816D0022805D18E
:108440001BF8043023B90BF804A003E01BF8043038
:10845000012B01D185F8008001340A2CE3D10BB047
:10846000BDE8F08F0BF80430F6E70BF80490F3E763
:10847000084A1360536013810BB0BDE8F08F0022EF
:10848000044B1A605A601A810BB0BDE8F08F00BF30
:10849000FC150020882600202DE9F04105460E46F7
:1084A0001746984682B0089C0094FFF753FE434657
:1084B0003A4631462846089402B0BDE8F041FFF73D
:1084C00099BF00BF01465422014811F049B900BFCD
:1084D000080500200021044B03F1780299600C3359
:1084E0009342FBD1704700BFA82E00202DE9F04F2A
:1084F0003F4F85B03C68DDF83880012C08BF002272
:1085000000295AD04FEA400A0AEB0001394D890090
:108510006E18B4680A2C59DDD3F800C00AEB0001CC
:1085200005EB810149680AEB00094FEA8909044615
:1085300055F809001E46D8F80030ACEB0000591A77
:108540000028B8BF40420029B8BF4942039203F057
:108550001FFF039A834607EB0217D7E902237968C6
:108560003F69009703F0FEFE05EB090700283BD0AA
:10857000326855F8093002FB0BF203FB00230BEBCA
:10858000000251100B4493FBF2F33360D8F8003033
:108590007F6803FB0BFB07FB00B0084490FBF2F085
:1085A000C8F8000033685444A4002B51D8F80030B8
:1085B0002C44636005B0BDE8F08F0E4B00EB40002B
:1085C00003EB8000816005B0BDE8F08F0134B4603A
:1085D000012CD3F800C0A1D145F801C0D8F8001093
:1085E0007160D3F800C09EE7D8F80000D8E700BF5C
:1085F00008050020A82E002030B40546064C696806
:10860000AA68EB6800680FC428696969AA69EB6900
:108610000FC430BC704700BF1C1600202DE9F04F7E
:10862000DFF828A1C5B0DAF80420002192008146C5
:1086300011F0A1F8DAF80430DAF81020581EA0EB97
:1086400063009047DAF814309847DAF80430002BCA
:1086500065D0DAF8006003F1FF3B09EB8309A3F171
:10866000020843AD88224FF0FF31684611F083F8CD
:10867000882200210DEB020011F07DF816F1FF3683
:1086800033D3DAF8183098470446BBF1000F53D0C3
:10869000DAF80400DAF81030A8EB6000984716EB1F
:1086A0000B0F02D0DAF8143098472046694621AA09
:1086B00003680F68BB4202D20B601F46036852F882
:1086C000044F04309C423CBF1C461360D0F88430F9
:1086D0000431BB4238BF41F8043CA34288BF136059
:1086E0009542E5D116F1FF36CBD2002321AAADF198
:1086F000040152F8044F51F8040F23449542A3EBB0
:108700000003F6D1DAF800600BF1FF3B93FBF6F3C0
:10871000BBF1FF3F08F1FF3849F8043DA2D1DAF878
:108720000430DAF8102003EBD3705B10C3EB600069
:10873000904745B0BDE8F08FDAF80430DAF8102041
:10874000581EA0EB63009047A9E700BF1C1600204D
:108750000E4BF0B45F68022F15DD00EB87070C3F6E
:108760000438024600230A4900F10C0652F8045F5F
:1087700011F9014B964205FB0433F7D11B1140F868
:10878000043F8742EDD1F0BC704700BF1C160020AB
:1087900028160020DFF868C0F0B4DCF8046000247C
:1087A000002E0ADD01EB8606043E0B1F53F8045F22
:1087B000AC42B8BF2C469E42F8D1DCF808304610D7
:1087C000A34214DA002818DD00236FF000450439B5
:1087D00051F8044FAC42B8BF1F4603F10103B8BFC4
:1087E00025469842F4D1B81B1560F0BC704751F88B
:1087F00026300020F0BC136070476FF00045F2E7B0
:108800001C160020F0B40446074E00F13007354630
:1088100020686168A268E3681034BC4206F1100663
:108820000FC5F4D1F0BC70473C1600202DE9F0478D
:10883000DFF8E89002EB400599F82C3099F82D20EC
:1088400082B0441E0F468DF804208DF805304E4648
:108850004FF0000A4FF0640800E0013C631C17D0A1
:1088600035F9023D002BF8D0314637F9140003F0FA
:10887000E5FDB5F9003098423EDBD9F8282008FB29
:1088800003F302FB00F29342C8BF4FF0020AE4E791
:108890001F4B1878BAF1000F13D11E4AC2F800A07E
:1088A00060B91D4999F82E400A680132A2420A6057
:1088B00004DD01221046C1F800A01A7002B0BDE824
:1088C000F0870546AAF10200B0FA80F0400985421F
:1088D00017D0104C02A92268014411F8041C01327F
:1088E0008A42226011DD00221870226000220A4BA9
:1088F0001A6002B0BDE8F0870020054B1D78854264
:10890000E7D10022034B1A60F0E72846EEE700BFEC
:10891000A0190020941900209C1900203C1600206A
:10892000014B1870704700BFA0190020014B187848
:10893000704700BFA0190020034B1B781BB9034AE6
:108940001368013313607047A01900209C190020A0
:108950000278014B1A7070475C0500200022034B1F
:1089600083F8F02083F8E421704700BF302800200E
:108970002DE9F04F614D97B02C78002C69D000297B
:108980006BD0F42404FB00F4DFF874811E4608EB7E
:10899000040C9CF8F0301746FF2B68D00133DBB293
:1089A0008CF8F030D2F800E0D6F8009004F1D00B4B
:1089B000012BCDE904E9C34461D00DF11009002376
:1089C0004FF4807A5A460EA808EB040B4946CDE9CD
:1089D0000633039300F096F80EAA06A9584600F055
:1089E00037F9039B59461A46CDF800A001234846A3
:1089F00000F084FA012304F134011A460A9041443C
:108A0000CDF800A0484600F079FA04F168010B9017
:108A100041444FF4C8730222CDF800A0484600F04C
:108A20006DFA04F19C010C90414449F64043012247
:108A3000CDF800A0484600F061FA06AA0D900AABF6
:108A4000594608A800F018FADDE908232C783A60A6
:108A50003360204617B0BDE8F08FF422284B02FBAC
:108A60000033204683F8F01017B0BDE8F08F12688D
:108A7000336804F1D00BCDE90423C3449DE74FF0E4
:108A8000000A6146524653468CF8F1A08CF8F2A0D9
:108A90000132042AC1F800E0C1F80C904B600B6170
:108AA0008B60C1E90533C1E90733C1E90933CB6202
:108AB00001F13401ECD1F4214FF4C863FA2201FB37
:108AC00000800DF1100902634266C0F89820C0F8DA
:108AD000CC208361C3648365C0F88030C0F88C30DB
:108AE000C0F89430C0F8B430C0F8C030C0F8C83016
:108AF0004946584600F098F861E700BF5C05002041
:108B000030280020F0B4D1E90057D2E900134E1B01
:108B1000DB1B002EB8BF7642002BB8BF5B421E4461
:108B2000C82E84B004DC4EF6602113898B4266D9CE
:108B30000124C2E900571346002123F8084F02F12F
:108B40001C0533F8024FA142B8BF21469D42F8D11F
:108B5000937FB142B8BF3146082B02EB43048CBF70
:108B60000023013305296681937722DD27294BDC19
:108B7000294B4A1F03FB02F2284BD41783FB0253F5
:108B80001344C4EB631303F2CA341429009413DDB5
:108B900031293EDC6FF0D102143902FB01F1204A89
:108BA000CB1782FB01520A44C3EB221303F28E332C
:108BB00004E040F2CA34009440F28E3301934FF443
:108BC0002F730146CDE90233164F00F1280601AD9F
:108BD000C4F57A7287FB02C3A3EBE2739BB200F188
:108BE000080220F8023B8242FBD121F80A4B8E4258
:108BF00002D055F8044BEBE704B0F0BC70470133EA
:108C00009CB296FBF4F696E74FF42F74312900944A
:108C1000C0DD4FF42F73D1E7F2FEFFFFEBA00EEAA9
:108C2000898888885655555570B4D1E90062034645
:108C300000256424C0E9006200F11C0223F8085FEB
:108C400023F8024F9342FBD170BC00238377704717
:108C50002DE9F04F0C469246CFB003900146D0224A
:108C60001AA8A4F1020B10F07BFD5D46D6465046D3
:108C7000A046804F0AF10806002213461AA930F8D0
:108C800033C00C6B0133042B04FB0C2201F13401C3
:108C9000F5D1B2F5FA6F34BF0122A7FB023200F121
:108CA000020028BFC2F38F12864225F8022FE3D1BB
:108CB00044460023A11D8C46CDE90633CDE9083397
:108CC0000AF1200A0DF124090DF1680806AA1546DB
:108CD0004F465C467646D8F83010029236F8022BA2
:108CE00034F8020F01FB02F2B2FBF0F2A445134488
:108CF00045F8043B47F8042F01D02B68EEE70EF14E
:108D0000080EF24508F1340809F11009069BDDD17F
:108D1000002108460C461AAD05F1D00C2A6B2F68CD
:108D2000EE683435AC45114407FB024406FB0200F3
:108D3000F4D194FBF1F490FBF1F1039A1046146026
:108D4000D160934604229046CDE9040300218C466D
:108D50000F460E460C4608460AAB019303EB080E7D
:108D60001AAA00915EF8103B1168D2F8089001FB36
:108D70000300D168D2F814A001FB0344516809FB39
:108D800003CC01FB03661169343201FB03770099C0
:108D900095420AFB03130093E4D1194606AB53F83E
:108DA000083008F1040890FBF3F094FBF3F496FB11
:108DB000F3F697FBF3F79CFBF3FC91FBF3F1B8F1AF
:108DC000100FCBF83400CBF84040CBF83860CBF82C
:108DD0004470CBF83CC0CBF848100BF1340BB5D144
:108DE000DDE904430399D03103910025A846AE463E
:108DF000AC462F462E46DDF804901AA9009359F888
:108E0000100B8B69D1F82CB003FB0066CB690BFB10
:108E1000005503FB00770B6A03FB00CCD1E9093A4C
:108E200034318A4203FB00EE0AFB0088E7D1009B45
:108E300096FBF3F697FBF3F79EFBF3F09CFBF3FC3A
:108E400098FBF3F195FBF3F5019BC4E90667043346
:108E50000193039BC4E908C0C4E90A153434A34252
:108E600004D0029951F8043F0291BEE74FB0BDE82B
:108E7000F08F00BFD34D62102DE9F0438C460C46B5
:108E80000026DFF87480971E043B063237F802EFA5
:108E900053F8045FBA4205FB0EF5A8FB059ECCF81B
:108EA000305006EB9E160CF1340CEFD101250A462A
:108EB000D031136B3432B3FBF6F3002B08BF2B46D3
:108EC00042F8043C9142F4D100210D460E46236B3A
:108ED000D4F800C0E7683434A24219440CFB03669E
:108EE00007FB0355F3D196FBF1F695FBF1F1C0E9D1
:108EF0000061BDE8F08300BFD34D62102DE9F04F53
:108F0000D2B28BB0012A0192044600F05881C0F021
:108F10002881022A00F09D8000234FF480629C4645
:108F20001F461D469E469B461E46984699469A46B3
:108F3000CDE90733059203930293069304930093BC
:108F4000039AD4E90004A4EB090406FB04290BFBF3
:108F50000433A0EB0A0043F3951308FB00EE06FB75
:108F600000550BFB007708FB04CC49F39519C1E9C8
:108F70000493029B4FEAAE2E8B61019B45F395153E
:108F800047F395174FEAAC2CC1E900E5C1E9027C33
:108F9000002B00F0E080009A059B764203FB02F371
:108FA000069A002B4FEA822A009AB8BF03F2FF33D9
:108FB00006FB02AABAF1000F4FEAA323B8BF0AF2D8
:108FC000FF3ACB614FEAAA234B62019B022B00F0D0
:108FD00037810023C1E90A330B6204FB04F400FB70
:108FE0000040A94B984200F3AE80642404FB00F0DB
:108FF000149BA64A90FBF3F46310934200F3A38002
:1090000042F21071A24AE41782FB0302C4EB22323F
:1090100001FB12309F4D561C80EAE07401FB1633B1
:10902000A4EBE07435F81600002B00FB04F035F8D3
:109030001220B8BF5B4202FB0300974FA7FB003032
:10904000400B01FB00F0149B90FBF3F00BB0BDE86C
:10905000F08FD1F82090D1E906073D1809EBD970BF
:10906000D1E90ACED1F824A005EB60050EEBDE783D
:1090700009EB0C064FEA68080CEBDC7B3D4406EB81
:1090800008024FEA6B0B5744554404925F445D4419
:1090900002EBD27B8A684F4403924A696744099283
:1090A0000A687344914605EB6B05079307EB0803C9
:1090B00000932B4648680AEB4C0A0290029AF2444D
:1090C00009EB2219039ACDF818A009EB621A099A44
:1090D000D1E9036006EB201606EB6219002D149A05
:1090E000B8BF05F10F0302EB23134FEA851898FB75
:1090F000F3F8009A14939601049AC8F580634FEA36
:10910000821B149A059396FBF2F69BFBF2FB029AE4
:1091100003FB05F31546099F002B3844F444039ADA
:10912000B8BF03F2FF338001CDF820C0039098123E
:10913000099B1544AD01029097019B014FEA8A2ECD
:109140004FEA892CFCE642F21070149B90FBF3F07E
:109150000BB0BDE8F08FC1E90733C1E90933CB6239
:109160003BE78869149A03441846002BB8BF03F103
:109170000F0002EB20124FEA831898FBF2F81492CA
:10918000C8F5806202FB03F000230028D1F800A09C
:10919000D1F80C90B8BF00F2FF3005928212CDE9F1
:1091A00002231F461D469B461E46CDE90733069304
:1091B000049300934FEA8A2E4FEA892CC0E6486A4E
:1091C000D1E9065605EB460E8644034406937346E2
:1091D00032184D6800920A680F6902EB251ACA68B6
:1091E000BEF1000F02EB2719149AB8BF0EF10F035E
:1091F00002EB23134FEA8E1898FBF3F81493C8F58B
:10920000806303FB0EFE0593009BBEF1000F4FEA47
:109210008316149BB8BF0EF2FF3E96FBF3F60023B5
:109220004FEAAE220292BA01AD0103921F469B465D
:10923000CDE9073304934FEA8A2E4FEA892C7FE663
:10924000DDE9042303FB02F3089A002BB8BF03F205
:10925000FF334FEA822C9B12049A0B62079B06FB9A
:1092600002C6049A9B020BFB123B002EB8BF06F20B
:10927000FF36BBF1000FB8BF0BF2FF3BB6124FEA4F
:10928000AB238E62CB62A8E614AE47016F110100DA
:10929000AD8BDB6838A701005917B7D10268014BC5
:1092A0001A6070476C1600200146B822014810F081
:1092B00057BA00BF701600202DE9F043074603227D
:1092C00000204FF0010803FB07F6079D104C2944CE
:1092D0008E5D94F80090DFF83CE0DFF83CC006F0CB
:1092E0000F0646FA02F4E4070CD512F90E4012F903
:1092F0000C503C4403FB0414645D4C453CBF08FA2D
:1093000004F4204312F1FF32EBD2BDE8F08300BF3A
:1093100030A7010048A7010050A701002DE9F04F38
:109320008DB0189F0546059097F802B0F8788846EA
:109330008345CDE90832DDF870A04DDC0123B84645
:109340001E9C0BFA03F20AFB024204921D9A97F844
:1093500001900BFB0A2603FA05F28B40134303939B
:109360004FEA4A030693EBB2CDE90A13079298F845
:1093700000404C450CDD23E0FA0606D4079B8342EF
:1093800000F09780002800F0B1800134A14515DB82
:10939000375DB906F9D51D9B1B9A009321465346AC
:1093A0005846FFF789FF039B8342E5D19DF81430AF
:1093B000335598F801900134A145E9DA98F8030093
:1093C000049B069A0BF1010B134458455644049331
:1093D000CDDA4746DDF8288019993B680846059A9A
:1093E00040F8223050F828309400C3F30741B1EB25
:1093F000136F4FEA88003B6019DC94461D9B97F879
:1094000001900AFB01353B7899450BD32B4413F8A7
:10941000016B464504BF03F801CC97F801905A1B35
:109420009145F4DAFB7801318B425544EBDA1A9B13
:1094300008F101011844099B8B420FDD01279C466E
:109440001A9A059D161952F82550026807FA01F379
:10945000134001311D438C453560F6D100231A9A23
:10946000984542F8283040F383800122059F1A98DE
:1094700002FA08F10444BC4602FA07F0CD4316464E
:109480001A9F06E002432A4047F8232001339845FB
:109490006ED057F823200A42F8D09C45F2DCF2DA6D
:1094A000226806FA03FE42EA0E02226057F82320E1
:1094B000E9E79DF8143008983355049B98F801901B
:1094C00033F91420036804FB02F103EB412303602A
:1094D0000BFB02F1169B1B6803EB412316990B60F3
:1094E000179B1B681344179A13604EE707F00F038E
:1094F000CDF860800325984648FA05F3DB072FD5A1
:109500001D4B1B9AEF561D4B5F4415F903901D9B95
:10951000A1440093384653464946FFF7CDFE039BCE
:1095200083421DD11D9B0B9A0AFB0737049B07F84A
:109530000920325533F91420089804FB02F103681E
:1095400003EB412303600BFB02F1169B1B6803EB4B
:10955000412316990B60179B1B681344179A1360DD
:1095600015F1FF35C8D2DDF8608098F801900CE75E
:109570000DB0BDE8F08F00BF48A7010050A7010063
:109580002DE9F04F814291B00546DDE91A760C468F
:10959000984601DB04460D4636F9149058F824B07D
:1095A00057F824A009FB0BFE0AFB09FC36F915301D
:1095B00058F8250057F8251003FB00EE01FB03CCFB
:1095C000ABEB00004B44AAEB0101CDE90DC30A92BD
:1095D000CDF830E002F0DCFE1D9B0B9053F8241018
:1095E00053F825308C46D8B25FFA81FE864588BF95
:1095F00060F3070CC1F3072EC3F30720864538BF7D
:1096000060F30F2CC1F3074EC3F3074086454FEAC2
:10961000136388BF60F3174CB3EB116F88BF63F31C
:109620001F6C239B0FA80893229B0EA90793219BD5
:109630000DF1340E0693209B0A9A05931F9BCDE9EA
:1096400000E104931D9B2946CDE902030CAB2046A3
:10965000CDF83CC0FFF762FE0CA90EC991FBF3F1F7
:1096600092FBF3F24FEA840A4FEA440948F80A10E1
:1096700047F80A2026F809301E9B4FEA450B43B1F4
:1096800033F909300B9A9342B8BF13461E9A22F859
:1096900009301C9A1C9B115D5B5D00228B4238BF18
:1096A0000B461C990B5526F80B2011B0BDE8F08F26
:1096B0002DE9F04FDFF8CCB08BB09BF80C40002CBC
:1096C0005DD000285BDD00251F4637F9153005F118
:1096D000010A002B91468846064654464DDD564504
:1096E00003DC4CE00134A6423FD037F91430002BA4
:1096F000F8DD59F8243059F8250058F82510C01A1B
:109700004EF2343358F82420891A0029B8BF494250
:1097100003FB01F14DF630130028B8BF404203FBB4
:1097200000F00914001402F033FEDBF81430834219
:10973000D8DD1B9B214609931A9BCDF80090089316
:10974000199B32460793189B28460693179B0134B2
:109750000593169B0493159B0393149BCDE901730A
:109760004346FFF70DFFA642BFD1554637F91530E6
:1097700005F1010A002B5446B1DC5645F5DC0BB06F
:10978000BDE8F08F701600202DE9F04F654C93B0C6
:10979000247C34B3002824DD1F4690468A46814647
:1097A0004FF0000B37F91B30BBB158F82B20219933
:1097B00002F58072521201FB02F65AF82B30229900
:1097C00003F5807331445B12C95C574859450578ED
:1097D00024D0A94209D3880671D40BF1010BD945D5
:1097E000E0D113B0BDE8F08F7746239BCDF8008021
:1097F0000993229B4A460893219B58460793209B36
:1098000006931F9B05931E9B04931D9B03931C9B18
:10981000CDE901735346FFF7B3FEDEE74FF0FF30AB
:109820006FF0FE1E844603243E49CDE90A5789683D
:10983000CDF844E00E913D490DF1400E1091239971
:1098400001EB46010D9159000C9111AE1CEB020C7D
:1098500018442CD400282ADB2099614527DD219962
:10986000814224DD01FB0CFC22990A9D6144095CC4
:10987000A9421CD20C9F8B4507EB4C0C17D06427D8
:10988000239D35F90C500F950D9D35F913C00F9D93
:1098900007FB05F50E9F07FB0CFC654507DD6425FE
:1098A0000D9F37F9100005FB00F0604537DC24B14F
:1098B000013C14F90EC0A057C8E70B9F8DE71D9817
:1098C00050F82B00C0F307249C4224D0C0B2984229
:1098D0000BBF032401244FF0020C4FF0000CBE46D6
:1098E00001F00F0022990B4440FA04F1C9070DD58D
:1098F0000F49219F61560F4E114407FB0131A657B6
:10990000895DA94202D259457FF46EAF013C64459E
:10991000EADA774661E703244FF0020CDFE70B9F9A
:1099200063E700BF7016002030A701000101FFFFB0
:1099300048A7010050A701002DE9F04F83B0DDE9F1
:109940000D4704FB02FE07EB0E04E65C864245D0A1
:109950008E4243D016F0200549D000250324AA46A4
:109960004FF0010BDFF8A4C006F00F069CF8009042
:10997000019307EB030C46FA04F7FB0715D5214FBB
:10998000214BE75714F903800D9B174403FB07C7CE
:1099900017F808800BFA08F7C84547EA050704D20C
:1099A000AF421CBF3D460AF1010A14F1FF34E2D276
:1099B000012202FA00F002FA01F10843A842019BD9
:1099C00019D0284010D05B0003EB4E0E0F9B33F9EB
:1099D0000E0090FBFAF003B0BDE8F08F5B0003EBE4
:1099E0004E0E0F9B33F90E0003B0BDE8F08F2846F2
:1099F00003B0BDE8F08F934003EB4E0E0F9B33F99D
:109A00000E00F1E748A7010050A7010030A70100B0
:109A10002DE9F04FB64CABB0E47B1C94002C00F069
:109A20000E81002800F0038118930023CDE91A125B
:109A30001093431E14901F93109B1F9A934280F221
:109A4000FE80379B109A194651F82230511CCB40AA
:109A50004FEA82021D9115920F9300F05781149BDB
:109A600019461D9B994240F351810E930023109A91
:109A70001E93189B03EB420319930BE00E9B0F9A66
:109A8000013352080E930F9200F03C81149A9A42CF
:109A900000F038810F9BDB07F0D51A9B15991C4607
:109AA00058581B9B0E9A1D4654F82240595855F899
:109AB0002230051B0C940D93CC1A85EAE573A3EBB9
:109AC000E573169384EAE473A3EBE4731793189E8B
:109AD000199B36F91220B3F90030002C40F0FD80BC
:109AE000002D40F016814FF4007BDDF870800C9E55
:109AF0000D9F34463D4604FB03F402FB004405FB86
:109B000003F5134494FBF3F402FB015595FBF3F5C5
:109B1000359B159A9C469A5822941446CDE92361A8
:109B200000260E9B21905CF82330D0B2D9B281423E
:109B300038BF61F30704C2F30720C3F3072188424B
:109B400038BF61F30F24C2F30740C3F307418842D3
:109B50004FEA136388BF61F31744B3EB126F88BFFA
:109B600063F31F642595230EC4F307459D42269792
:109B7000CDE92766299600F3D28001331193E3B231
:109B80001293C4F30723139327AF129C139A9442A2
:109B90005CDC9DF840306E020B9333464646984697
:109BA0009DF838A002F101093B9B2A4603933A9B9A
:109BB00051460293399B0B980193389B009323469F
:109BC000FFF7BAFE00283DDDDDE90C324FEA442CF8
:109BD0000221ACEB030E0EB30BFB0EF3A2EB6323DF
:109BE000A3EB0803002BB8BF5B42B3F5007F09DA93
:109BF000C3F5007300FB03F357F8212002EB632346
:109C000047F82130F1B1013921AB53F8213024AAB2
:109C100052F82120ACEB030E002EDDD1A8EB02029E
:109C20000BFB02F2A3EB6223A3EB0C03DAE76FF06A
:109C30000043304C3049314A23600B6010602BB038
:109C4000BDE8F08F01344C45AED1B046119B0135D3
:109C50009D429AD1DDE92842DDE91601279B642562
:109C60009A42A8BF1A4605FB04F4154602F0C8FB49
:109C70002D2801DDC0F15A001D4A0CCA03FB00F378
:109C8000C0F12D0002FB00321D4B83FB0231D317C4
:109C90000A44C3EB621305FB03F3A342BFF6EEAE27
:109CA0003B9B149A09933A9B0E990893399B109801
:109CB0000793389B0693379B0593369B0493359BFC
:109CC0000393349B0293189B01931B9B00931A9B55
:109CD000FFF756FC1C9B1E93D0E6DDE91667BE42DB
:109CE00017DA6D0295FBF4FBDDF87080FFE600BF2C
:109CF00070160020A8050020AC050020BC1900202B
:109D0000B7600BB61E9B002B7FF496AE1D9B109385
:109D100092E6640294FBF5FB4FF00008E7E6DDE90C
:109D2000160102F06DFB2D287FF7A8AE00252C460A
:109D3000A0E700BF2DE9F04FB84CABB0A47B002CDE
:109D400000F03281002800F02F8191461393023BEE
:109D5000159303EB40030D934B464FF0000B8946E0
:109D60009A460A901E2200211AA80FF004FD002135
:109D70001E2222A80FF0FFFCA94B4FEA4B0133F93A
:109D80001B301091002B40F32281A64B33F91B307E
:109D9000C3EBC3139B1211930A9B002B40F3178153
:109DA0000027A14A159B8A180C92A04A0F978A187F
:109DB0000B921D46CDF850B003E00D9B01379D423C
:109DC00072D035F9022F002AF7DD0B9B0C98B3F9FE
:109DD000004059F827205AF82710B0F90000611AFE
:109DE000801A02F0D5FA6624359E914904FB00F4EE
:109DF000F05D51F8046C02F021FBA41280468D49FD
:109E000020B202F01BFB0B9A12900C98B2F900C022
:109E10005AF82710B0F9002059F82700ACEB0101DF
:109E20007E4B101A00299A6FB8BF49420028B8BF6C
:109E30004042D3F87CB00E9202F0E2FA2D28C8BF5F
:109E4000C0F15A0000FB0BFB0E9AC0F12D0002FB83
:109E500000B2794B794983FB023C109B9444595ED4
:109E6000D2170E44C2EB6C1208FB04F806FB02F694
:109E7000B04580F29C806420684BD3F8802000FBC2
:109E800002F2424540F39380129B8B420F9B03F1F9
:109E9000010280F28C800121D3B20F931AABD95505
:109EA0000D9B01379D428CD10F9BDDF850B0012BEB
:109EB00040F28D809DF86820002A40F091811AA917
:109EC00013460A9C04E011F8010F002840F07B8142
:109ED00001339C42F7D1169B9F004FEA430809EBE0
:109EE00007030C930AEB07030E93369B1F44139B47
:109EF00043440F93349B98440026CDF840B0CDF8EE
:109F00002C80DDF828B0DDF8588019AD18AC002A97
:109F10003BD0B04539D022AB9B5D3C9A002B379BA0
:109F200018BF002309923B9A049308923A9A4B4631
:109F30000792399A31460692389A40460592369AE7
:109F40000392359A0292139ACDE900A25A46FFF77E
:109F500017FB38680F9B0E9A0C99B3F90030126802
:109F6000096802903C98CDE9004506903B98059021
:109F70003A98049039980390404601F079F9DDE968
:109F8000180102F005FA0B9B18800136B3451CD06E
:109F90001AAB9A5DBBE73C460D9B0BF1010B0233FC
:109FA0000D930A9B5B4526D12BB0BDE8F08F119B2A
:109FB000A3427FF702AF01220F991144CBB20F9356
:109FC00022ABDA551AABDA55F7E6DDF840B00BF103
:109FD000010BBBF10A0F7FF4C5AE5346CA46994642
:109FE0000A9B002BE0DD349B4FF0000B0D934B469A
:109FF000D1469A46139C34F91B3004EB4B02002BDC
:10A000001492C9DD4FEA8B0309EB03021793534403
:10A010004FF0000816921593274651E07016002065
:10A020006827002068250020682E00202C260020AC
:10A0300098160020C0160020B7600BB6942E0020A2
:10A040002546594644463C9B0A9A09933B9B204629
:10A0500008933A9BCDF800A00793399B0693389B51
:10A060000593379B0493369B0393359BCDE901738E
:10A070004B46FFF785FA36980B9E0C9B8059129A37
:10A080001399B3F900301268096802903C98069061
:10A090003B9805903A9804903998039022A8019033
:10A0A0001AA80090204601F0E3F822991A9802F0CD
:10A0B0006FF928800A9B08F1010843453FF46BAF14
:10A0C00037F918304FEA48043A19002B0C92F1DDA9
:10A0D000C345EFD05AF8282059F828305AF82B10E9
:10A0E00059F82B00891AC01A02F052F959F82B308E
:10A0F0000E9059F828005AF828101B1A5AF82B20ED
:10A1000083EAE375A5EBE375359B521A82EAE276A2
:10A11000394913F80B00A6EBE27602F08FF9359B74
:10A120000F90354913F8080002F088F9334A314698
:10A13000D2F8B030109028461193D2F8B45002F003
:10A140005FF942F2107C4FEA88032D280B934B44B1
:10A15000C8BFC0F15A0013930B9B00FB05F5534495
:10A160001293119BC0F12D0003FB0053234A0D9D58
:10A170002348D2F88460B5F9001080FB03200F9AC1
:10A18000184402FB016E3499109A31F91810DB174C
:10A1900002FB01E2C3EB60100E9B02FB00F20CFB22
:10A1A00003FC349B94451C4484DAC345FFF648AF56
:10A1B000149B41460C93159B5C461293169B13937C
:10A1C000179B0B933FE79F0009EB07010C910AEBEC
:10A1D00007010E9136994FEA43080F44169386E61D
:10A1E000139BDDF8D080CDE90EA30023369FCDF878
:10A1F0003090169380E600BFF816002070160020FD
:10A20000B7600BB684B038B5174D04AC84E80F00C6
:10A21000212240F21461154804AC00F0B9F80FCCCB
:10A2200028606960AA6003CC182228616961284609
:10A230004FF4B871EB6000F0ABF80D494FF460607B
:10A2400000F0F4F80B494FF4905000F0EFF8642060
:10A2500000F0F0FC632000F0EDFCBDE83840602029
:10A2600004B000F0E7BC00BF34250020B405002096
:10A27000100600202006002084B030B402AC84E830
:10A280000F000A4B9DF808209DF80A109DF8125007
:10A290009DF813401A7099709D72DC7230BC18469C
:10A2A00018224FF4B87104B000F09CB83425002097
:10A2B000F8B500F0A9FA0446084E00F1200735462B
:10A2C00020686168A268E3681034BC4206F1100699
:10A2D0000FC5F4D123783370F8BD00BFB40500205A
:10A2E000F0B4074605460A4E06F1200C34460FCC62
:10A2F000644528606960AA60EB6006F1100605F10C
:10A300001005F3D1337838462B70F0BC704700BF8E
:10A31000B405002070B40446174D00686168A26857
:10A32000E368164E0FC520696169154A03C5736855
:10A33000A569207F51692B4373600870A37F657FF7
:10A34000CB71E17F93680F480570197094F8200075
:10A350000D49587094F821500C489D7094F8225083
:10A36000DD70D368A28DD4E909651A811E605D6035
:10A37000086070BC704700BFA42700206008002060
:10A38000E80700200C1A00202826002049A9000018
:10A39000F8B5134B0C0A53F824606EB1F468CFB2D1
:10A3A000013C05E073681B5DFB1A002B05DA2C46A7
:10A3B000631C04F1FF35F5D1F8BD1546B36832686A
:10A3C00033F81430014652F824002A4618440FF09E
:10A3D000C7F9B36833F814202A4423F81420F8BDD1
:10A3E00040060020104BF0B40C0A53F824706FB1F3
:10A3F000FB68CEB2013B05E07C68E45C341B002CBA
:10A4000006DA2B46591C03F1FF35F5D1F0BC704735
:10A41000BC68396834F8134051F82350A41A014637
:10A420002819F0BC0FF09CB940060020044B000A2C
:10A4300053F820201AB9142898BF43F82010704709
:10A440004006002000232DE9F043036069B3CE6885
:10A45000D2B206F1804C06F100470CF1FF3C013FFF
:10A4600006F1FF3EB342A7EB0308AEEB0305ACEBEE
:10A47000030915D04C680133645D141BF2D40D68D8
:10A4800055F82990B9F1000F07D08D6835F81850AC
:10A490002D1B002DE6DD0560A1444846BDE8F08394
:10A4A0004FF000094846BDE8F0838946F5E700BF54
:10A4B0000023B1F5704F70B4C1F30724036028DAAC
:10A4C000132C1FD9144D06466A68E86889B2431EEA
:10A4D00002EB400204E032F8020D081A07D52346C9
:10A4E000581C03F1FF34F6D1002070BC7047AA68F5
:10A4F000296852F8232051F82330121A3260184488
:10A5000070BC7047054B8AB253F8241070BCFFF73B
:10A5100099BF1846E9E700BF30060020400600203A
:10A5200000B583B0014601A8FFF7C2FF044B1860D5
:10A5300008B1019B1844034B186003B05DF804FB9D
:10A54000001A0020041A002070B50E4E024635682D
:10A550001DB10D4B1C68A54206D3144608460021C8
:10A560000FF009F9204670BD641B8442A8BF044661
:10A5700008462246294625440FF0F2F83560204669
:10A5800070BD00BF001A0020041A002070B50B4EE9
:10A5900035681DB10A4B1C68A54202D30024204631
:10A5A00070BD641B8442A8BF044628462246254449
:10A5B0000FF0D6F83560204670BD00BF001A0020AD
:10A5C000041A0020B0F5C06F16D0B0F5047F03DC8C
:10A5D0000F4B5B69B3B118470E4B1B7803F07F0339
:10A5E00003F504738342F3DB42189342F0DA10B5AB
:10A5F00000F036F8012010BD0029E9DB064B1A787F
:10A60000A02A01D000207047052201201A7070474F
:10A61000A42700207C1B0020E0060020024B1B69C1
:10A6200003B1184718467047A4270020084B094A71
:10A630005B78DBB2012B137006D0022B03D1012211
:10A64000054B5A7070477047044B1B68184700BF92
:10A65000F40600204C1A0020E0060020A427002069
:10A6600008B50A4B1B78012B0CD0022B02D100221B
:10A67000074B5A70074A137803F080036FF3C71330
:10A68000137008BD044B5B689847F3E74C1A002031
:10A69000E00600207C1B0020A42700202DE9F843C1
:10A6A000254EDFF8A8903378244DDFF89C80244FA6
:10A6B000012B06D0022B1BD06A78934238D1BDE81B
:10A6C000F883D8F8083098470446B9F1000F28D12C
:10A6D000D8F804309847D8F800309847DFF87090E1
:10A6E0006B783278DBB2934209D1002CE0D1E6E7F7
:10A6F0001A467C786B78E4B2DBB29342F5D0012A3B
:10A7000012D0022A02D100220D4B5A700D4A6978EC
:10A710001378317003F080036FF3C7131370BDE833
:10A72000F88309F1FF39DBE7074B5B689847EDE7F2
:10A730001A46012AE5D1F7E74C1A0020F40600205A
:10A74000E00600207C1B0020A4270020FF2C010035
:10A75000FE2C010038B5194C2378012B17D0022BA1
:10A760000CD0174A5278934206D0164A137803F059
:10A7700080036FF3C7131370002038BD124B104ACB
:10A7800059785278022AF7D000225A70EDE70F4D1F
:10A79000AB68984718B16B6898472B6898470A4B85
:10A7A00007492278587849789142E5D0012A02D1A8
:10A7B0006B689847D9E7022AE6D0D6E74C1A002002
:10A7C000F40600207C1B0020E0060020A4270020C7
:10A7D000A023034A13701378A02BFCD0704700BF4E
:10A7E000E0060020014B1878704700BFF4060020F7
:10A7F000014BD878704700BFF4060020014BD87099
:10A80000704700BFF406002000487047F80600209B
:10A81000014B9878704700BFF4060020014B9870F8
:10A82000704700BFF406002008B5FFF793FF08B992
:10A83000014B186008BD00BF781B00200A46F8B520
:10A84000094F0A4C3B6826689B79B51803EB8301D6
:10A8500003EB41039D4200D9FFDE0146B868304456
:10A860000EF07EFF2560F8BD34070020781B002025
:10A8700070B50D460646FFF711FF094A094C1378DB
:10A88000094963F07F0365F306038D80A5681370A3
:10A89000A660FFF7CBFEFFF701FFA56070BD00BF0C
:10A8A0007C1B00203407002040070020F0B50D4637
:10A8B000002185B02E79CDE9011103919DF828C0C2
:10A8C000044638B35EB31F4E3178814224D09DF8E0
:10A8D0000510600860F300019DF80470C4F3800E59
:10A8E00064F382016EF3C30162F303070A466CF35B
:10A8F00007176EF3041201A80C21ADF809308DF88A
:10A9000005208DF80470FFF799FF012334702B7137
:10A9100005B0F0BD2EB90B4E347005B0F0BD094E38
:10A92000D5E79DF8043001A862F303036CF3071325
:10A930000C218DF80430FFF781FF024E2C7134702A
:10A9400005B0F0BDCA1B00202DE9F04F89B0994633
:10A950009DF85C409DF8603006460F469046029395
:10A960003CB1FFF761FF002800F0E18009B0BDE8CD
:10A97000F08F734B1D460393FFF790FE2C6000246D
:10A98000CDE905440794FDF7D1FFA642824640F386
:10A99000B280DDF850B06B4D6BE037F914E038F958
:10A9A000140021B1B5F90030734500F0C3800122D5
:10A9B0009DF816104FEA2E2C9DF814306CF303010D
:10A9C00004F1010C6CF303039DF815C062F3071347
:10A9D0004CEA020C159A8DF817E08DF8180012F861
:10A9E00004E00012129A60F307118DF8161032F984
:10A9F00014108DF81430FE29C8BFFF2339F8140055
:10AA0000C8BF8DF81B30139BADF8190053F8240014
:10AA10006EF3410CD8BF8DF81B108DF815C0C1B274
:10AA2000C0F3072CC0F30743ACEB0101C3EB106389
:10AA300099428DF81DA04FF04D0252DD02FB01F14D
:10AA400089118DF81E108DF81F300C2105A8FFF715
:10AA5000F5FE37F914309BF800102B8038F91430CC
:10AA60006B800134A64229710BF1010B05F106053B
:10AA700041D09BF800302979002B8ED10029F0D0ED
:10AA8000B5F900109DF815C09DF816009DF814E06A
:10AA900063F3000C0B1263F30300631C63F3030EF8
:10AAA00073460122B5F902E062F30713159A8DF897
:10AAB00017108DF818E0115D4FEA2E2E6EF3071077
:10AAC00061F3410C8DF816000C2105A88DF81DA02E
:10AAD0008DF815C08DF81430FFF7B0FE9BF800100C
:10AAE000BFE702FB03F3ACEB00009B118DF81E30B7
:10AAF0008DF81F00A9E70222B9F8143002980092DD
:10AB000011490B22FFF7D2FE039B1B68002B3FF479
:10AB10002DAF0E490E480A78838002F07F0263F35E
:10AB200006020A70FFF782FD09B0BDE8F08F044B02
:10AB3000039324E7B5F9023083427FF438AF90E7FE
:10AB4000781B0020801B0020C41B00207C1B0020E1
:10AB500040070020092300B583B08DF805000221CD
:10AB600001A88DF80430FFF783FE03B05DF804FB05
:10AB7000F0B4224C82B025788DF80720854202D0AF
:10AB800002B0F0BC7047FF261D4802AD076B15F8F8
:10AB9000012DBF681B4892000361C0E902151A4BE2
:10ABA0003A81069A26701A608A7822B30B7908785F
:10ABB0004E7902FB003006F07F06144B06FB00F0D6
:10ABC0009F6838608B795BB10022013B01EB830504
:10ABD0006D89013B2A445D1CF8D102FB06023A60F4
:10ABE000A0230B4A13702378FF2BFCD0052313708E
:10ABF00002B0F0BC70474A78D8E700BFCC1B0020F9
:10AC00004006002060070020F419002030060020D4
:10AC1000E0060020014BDB6858817047E807002000
:10AC2000034B1879A0F10100B0FA80F04009704799
:10AC3000DC1B002000B583B00146202268460EF0E0
:10AC40006BFD01230099064A019802EB8102D2F8BC
:10AC5000051083400B43C2F8053003B05DF804FBD8
:10AC6000DC1B0020014B1878704700BF5C080020F7
:10AC700070B4184A184B90601960827802B9427813
:10AC800003790178457902FB013105F07F05134B0B
:10AC900005FB01F19E68316083795BB10022013BC5
:10ACA00000EB83046489013B22445C1CF8D102FB65
:10ACB00005123260A024FF2309480A4A04700A4999
:10ACC000137002E00B78022B02D11378FF2BF9D01E
:10ACD00070BC704750080020F41900203006002096
:10ACE000E00600205C080020F40600200246024B2B
:10ACF0000068516803C370472817002000230B49E0
:10AD00000B4A0C4810B4C1E90033C1E90233C2E96F
:10AD10000033C2E90233C0E90033074C0B61136111
:10AD20000381C4E90033238110BC70474819002017
:10AD300070190020B0190020F41B002009232DE910
:10AD4000F04F324C85B065682468864603953048DC
:10AD50000294304FDFF8C090DFF8C0A01A44009191
:10AD600037E006784FEA430C3EF91350002E36D0F8
:10AD700039F913B0FC5CA5EB0B01019102998846EF
:10AD80000399002C18BF884644460199E4B2002973
:10AD9000B8BF49428C422ADD009931F913803AF953
:10ADA0001310A8EB0108B8F1000FB8BFC8F10008F4
:10ADB00044451CDD34462EF813B03AF90C50009986
:10ADC00021F81350013B591C00F8014902F1FF32F0
:10ADD00019D01478002CC4D1DC551478F2E700990E
:10ADE00029F8135031F913502AF81350EAE7009963
:10ADF00029F80C5031F913404FF00101F9542AF8A9
:10AE00000C401478DEE705B0BDE8F08F281700206D
:10AE1000B9190020F41B00204819002070190020E7
:10AE200030B40546044C00686968AA68EB680FC432
:10AE30002869206030BC704730170020014B18781B
:10AE4000704700BFFE1B00204FF0000C2DE9F04FB3
:10AE5000E0464FF0010B1646304F83B0D7E9034967
:10AE600000910194D7E901EA10F1FF303DD33A781F
:10AE7000002AF9D033F9104074453DDD0C9D35F9B9
:10AE80001050554538DD94460D9D05F800B07A7890
:10AE9000002AE9D04C45E7DD009A56F8204052F8E8
:10AEA0002020A2F5007292B2B2F5804F28D90E9AF6
:10AEB00052F82050C5F307221446C5F30741EAB201
:10AEC000A21AC1EB156401320134A2421FDA6425D3
:10AED00005FB02F292FBF4F4019AA242C4BF0D9A60
:10AEE00002F800B010F1FF30C1D260460C4B83F87D
:10AEF00000C003B0BDE8F08F0D9A02F80080C6E7ED
:10AF0000A4F50074A4B2B4F5E05FD0D8ACE7642532
:10AF100005FB04F494FBF2F4DEE700BF30170020D9
:10AF2000FE1B00202DE9F04FC3F307461C0E8BB02B
:10AF3000A642DDF85090DDE917E856DC06FB09FC77
:10AF400012B2A2EB46220292621CDDB209920AB250
:10AF5000079505926544159AC3F307276B1ED3180E
:10AF60000193169B089703EB4C0C4FEA49030137FA
:10AF70000693079B08998B422ADC029A019D002ABE
:10AF8000B8BF5242039204E08A0631D40133BB4277
:10AF90001ED015F8011F8142F6D13CF91340002C58
:10AFA000F4DD059AA2EB432181EAE172A2EBE172A2
:10AFB000DEF80010013304FB0211CEF80010D8F8BF
:10AFC00000200399BB4201FB0422C8F80020E0D115
:10AFD000069B01369C44019B4B440193029BA3F5C5
:10AFE00000730293099B9E42C3D10BB0BDE8F08F62
:10AFF0000022159C01F00F0104EB030B049341FAAE
:10B0000002F4E3070BD5094C094B145712F903A0BE
:10B01000344409FB04B414F80A40A04204D00132BD
:10B02000042AECD1049BB1E7049BB6E74CA70100CE
:10B0300054A70100F0B404460F46124E00F1300C44
:10B04000354620686168A268E3681034644506F1FB
:10B0500010060FC5F4D13D46206861680A4F03C64B
:10B0600005F130063C4628686968AA68EB68103527
:10B07000B54207F110070FC4F4D12868696803C707
:10B08000F0BC7047001C0020381C00202DE9F04F58
:10B09000824693B01F46BDF98C30840007939DF81B
:10B0A000903088469146002122461C9806930EF067
:10B0B00062FB22461D9800210EF05DFBBAF1000FE5
:10B0C00072DD0024DFF8A4B102E00134A2456BD0A8
:10B0D00037F91430002BF8DD0025229E1E9B12A8A4
:10B0E00053F8243059F8242058F8241040F8245DEF
:10B0F0000296219E04900196209E08A80390009637
:10B1000020460895FFF70EFFDDE9083237F91410E5
:10B1100093FBF1F392FBF1F11C9A42F824301D9B52
:10B1200043F82410069B012B41D058F824005946BF
:10B13000C0F30800B0F5807FC8BFC0F5007001F013
:10B140007DF9064659F824004549C0F30800B0F5DA
:10B15000807FC8BFC0F5007001F070F91D9B0546E7
:10B1600053F824101C9B53F8240001F011F9DBF86C
:10B170002C3083424FDC4020064637F914C0DDE90D
:10B18000082302FB06F603FB00F34FEA8C1C96FB38
:10B19000FCF693FBFCF31C9A42F824601D9A42F8DB
:10B1A00024300134A24593D113B0BDE8F08F1C9B2D
:10B1B00058F8242053F8240059F82430C2F3080228
:10B1C000C3F30803B2F5807FC8BFC2F50072B3F5C0
:10B1D000807FC8BFC3F50073CDE90B010D920E93BC
:10B1E0000A9401F0D5F8B3250026012104220F901E
:10B1F0001C481D4BCDE9040537F91450CDE9011663
:10B20000079E0092039308220AAB6420CDE91065E3
:10B21000F7F728FD59E7DBF82830079A37F914C00B
:10B220009A4202DC40200646A9E7C6F14003DBE96A
:10B230000C1260460093002301F094F8084B37F994
:10B2400014C0D3E90C12C5F1400300930644002357
:10B25000604601F087F837F914C028448FE700BF33
:10B26000381C002058A7010060A70100001C002026
:10B270002DE9F047002688B01C1EDDE91087C8F8CC
:10B2800000603E604FDD8A46169D08AB43F8046DB2
:10B290000295159D0DF1180C0195149DCDE903C380
:10B2A0000095129B91460696FFF73CFE1F4ECAF38F
:10B2B0000800B0F5807FC8BFC0F50070314601F0CE
:10B2C000BDF8DFF86CA0C0F14003316BDAF8342030
:10B2D000054600932046002301F044F8C9F308090D
:10B2E000B9F5807FC8BFC9F50079054410494846C3
:10B2F00001F0A4F8DAE90C12C0F14003064600930D
:10B300002046002301F02EF8DDE90623304403FB3C
:10B3100000F302FB05F0A40193FBF4F390FBF4F4BB
:10B32000C8F800403B6008B0BDE8F087001C002072
:10B33000381C0020F0B40446094E00F130073546B1
:10B3400020686168A268E3681034BC4206F1100608
:10B350000FC5F4D12068616803C6F0BC704700BF18
:10B36000441700202DE9F04F061E83B026DD9946D4
:10B370009046019100244FF0640ADFF84CB0114F61
:10B3800002E00134A64219D01BF80450002DF8D079
:10B3900038F914000B4901F051F8019BFD6A33F9AB
:10B3A000142005FB00F00AFB02F28242B4BF002029
:10B3B000012009F804000134A642E5D103B0BDE83C
:10B3C000F08F00BF44170020A82600202DE9F04789
:10B3D000061E1FDDDFF840A04FF064085746941E9C
:10B3E00004EB4606A1F102095D1E34F9020F39464D
:10B3F00001F024F8DAF8282039F9023F02FB00F0C6
:10B4000008FB03F38342B4BF00230123B44205F8D1
:10B41000013FEAD1BDE8F0874417002000283BDD5A
:10B420002DE9F043002637468C1E04EB4008951E9C
:10B4300034F902EF35F902CF7745B8BF7746664554
:10B44000B8BF66464445F3D100254FF06408A946CD
:10B45000124CD4E90CC404FB06F60CFB07F7079C5E
:10B46000013C04EB000E14F8010F78B131F915C05E
:10B4700008FB0CFCBC4505DB32F9150008FB00F0AD
:10B48000B04203DA84F8009003F80590A64505F170
:10B490000105E8D1BDE8F083704700BF44170020E4
:10B4A000034610B4034C59689A680068DB680FC4FF
:10B4B00010BC70477C1700200023F0B4344A354D8F
:10B4C000354C3648364F3749C2E90033364EC2E96B
:10B4D00002331361C5E90033344AC5E902332B61F5
:10B4E000C4E90033324DC4E902332361314CC0E971
:10B4F0000033C0E9023303613B602F487B603B812E
:10B50000C1E90033C1E902330B61C2E900332B49C1
:10B51000C2E90233C6E9003313613381284A294E58
:10B52000C5E90033C5E902332B612360264D636012
:10B53000A360E3602361254C036043608360C360C4
:10B5400003610B6022484B608B60CB600B61136022
:10B55000204953609360D360136133601E4A736067
:10B5600033812B60C4E900336B602B81036043603F
:10B570008360C36003610B604B608B60CB600B61C9
:10B580002381136053609360D3601361F0BC7047F4
:10B59000C41C0020D81C0020001D0020B01C00206E
:10B5A000A8260020EC1C0020841C00209C1C0020ED
:10B5B000701C0020942E0020F8270020802E0020F0
:10B5C000682700209425002024280020901C0020BB
:10B5D000682E00202C260020682500202DE9F04F41
:10B5E000460006F108058BB0044625F00705073034
:10B5F00020F0070000AFADEB050DE846D7E91FAB23
:10B60000ADEB000D6846BD6FF961E91D21F0070142
:10B610007B61D7F89430ADEB010DBA610021224671
:10B620007B62C7F8088078600EF0A5F82A464FF0D4
:10B63000FF3168460EF09FF83246396F4046C7F832
:10B6400010D00EF08DF8002C7B6A6FDD7A6E00262C
:10B6500002F1FF3909EB04027A62C7F894305A46C6
:10B66000D34603E07B6A013699455BD019F8011F88
:10B670000029F7D03B6F002D33F916A05D4B5968B8
:10B6800001EB4A0AEEDD4FF0FF333B62D7F884301E
:10B69000C7F80C900024A3F10208914602E001349F
:10B6A000A54220D038F9023F002BF8D0FB6E59F8A4
:10B6B000241033F916C0BB6EA1EB0C0133F9160050
:10B6C0005BF82430181A00F063FE4DF6301303FBCC
:10B6D00000F000145045B8BF3C6204F10104B8BF4B
:10B6E0008246A542DED13B6A4A46591CD7F80C90E7
:10B6F000B8D03969C9564B1C71D0BB6833F91100F9
:10B700008245AFDA00244FF0010C23F816A0386A06
:10B710003B691E547B685C5403F806C07B6A0136A3
:10B720009945A3D1DA469346D7F89430002D52DDDF
:10B73000D7E9226C002210463969013D0D44D7F843
:10B7400090E04C1E7D6214F9011F4D1C3FD05AF849
:10B7500022505BF82280A946FD6925F81190BD6949
:10B7600025F81180D7F884501CF8028035F9129022
:10B770007D6925F8119036F912903D6D25F81190EC
:10B780007D6D05F801801EF80280BD6D05F8018011
:10B790007D6F6A54D7F8985035F91280FD6DA9462F
:10B7A00053F8225049F821503D6E25F81180D7F802
:10B7B00084104AF822004BF8220021F8120026F8E3
:10B7C00012000CF802000EF8020043F82200796A19
:10B7D0000132A142B7D12C37BD46BDE8F08F01211F
:10B7E000BB68386A23F816A03B691E547B689955DC
:10B7F00038E700BF7C1700202DE9F04F04469DB0CC
:10B800000AAFF962D7F88410BA62073121F0070154
:10B81000ADEB010D0AA939610846D7F884204FF035
:10B82000FF319846FB600DF0A6FFE31D23F00703F0
:10B83000ADEB030D0DF1280B2246002158460DF00B
:10B840009AFF0022D7F88410FA63914256DDD34E56
:10B85000C7F824B006E0FA6BD7F8843001329A4278
:10B86000FA6349DAD7F8903033F91230002BF2DD61
:10B870000023D7F8C0209C42C7E91023FA6B40F39D
:10B88000D5814FF0FF3904E07B6C0133A3427B6428
:10B8900024DA38F913100029F6DDF86AB96A31F9AB
:10B8A000131030F91330D7F88C0050F82250D7F825
:10B8B0008800691A50F822004DF63015C01A00F0C1
:10B8C00067FD05FB00F53B6C2D14AB4200F36A816C
:10B8D0007B6CFA6B0133A3427B64DADB4FFA89F3AA
:10B8E0000121386983547B6A013203F80910D7F8C3
:10B8F0008430FA639A42B5DBD7F824B0002C40F3C9
:10B900004981013C0BEB0403D7F870904FF000081D
:10B910007B610BF1FF3A07E07B6908F101089A456A
:10B9200009F1020900F036811AF8013F002BF3D02B
:10B93000FB6833F91820FB6AFA6333F91800BB6A15
:10B9400002FB00F033F91850BB6F02FB05F513F84A
:10B9500008303B627B6F13F808307B62D7F8BC304D
:10B9600013F80830FB61FB6F53F82860D7F8843078
:10B97000002B40F35F81002494463B69C7E901A98D
:10B98000D7E9219A03F1FF3B07F14403BB611BF99F
:10B99000013F434540F09880D7F890305AF8242072
:10B9A00033F91410D7F88C3002FB0100324653F8FB
:10B9B000243003FB0155D7F8A030614453F82430FC
:10B9C000F9635FFA83FEF1B2C3F3072C7145C6F346
:10B9D000072188BF6EF30702C7E90D056145C3F370
:10B9E0000740C6F3074138BF6CF30F221B0E81429C
:10B9F00088BF60F31742B3EB166F88BF63F31F6213
:10BA00001546D1B27145C2F3072188BF6EF3070511
:10BA10006145C2F3074138BF6CF30F25814288BFEF
:10BA200060F31745B3EB126F88BF63F31F65D7F858
:10BA3000B83021460893D7F8B430F8690793D7F89F
:10BA4000B03016460693D7F8AC304A460593D7F87F
:10BA5000A8307D640493D7F8A0300393BB690293A8
:10BA600007F13C03019307F13803009307F1340316
:10BA7000FDF754FCBB6F396A1A5D00239142B8BFD1
:10BA80001146D7F898203962115D7A6A4AF8243055
:10BA90000A437A62D7F88C2007F1340042F8243048
:10BAA000D7F8902090E8211022F81430D7F894208D
:10BAB00022F81430D7F898201355D7F89C20135546
:10BAC000D7F8A02042F824300134A1457FF45FAFBD
:10BAD000D7E901A9624690FBF2FB95FBF2F5D7F896
:10BAE000B83014B20693D7F8B4302A460593D7F885
:10BAF000B030F8690493D7F8AC305946CDE9026309
:10BB0000BB69C7E90DB5019307F1400300932346D4
:10BB1000FFF7AEFBD7E9100100F03AFC66230122E3
:10BB200040F2A23E00214FF0020C00B203FB00F3F2
:10BB30001A489B1204901A480390A9F80030742008
:10BB4000CDE901214B461146CDF814E0CDF800C0F7
:10BB5000F7F788F8FB6809F1020923F81840FB6A37
:10BB600023F818B0BB6A23F818507B6F1A4697F871
:10BB7000243002F80830BB6F1A4697F8203002F8DC
:10BB80000830FB6F43F828607B6908F101089A458B
:10BB90007FF4CAAE4C37BD46BDE8F08F6CA70100FC
:10BBA00098A7010040F2493200920022334623490F
:10BBB0006D2093464FF0040A3D64D7F84490012568
:10BBC000F7F7A2F840F24A331D4A0593039229463B
:10BBD0002A4607F13C030496CDE9015BCDF800A0AD
:10BBE0006420F7F73FF840F24B33164A2946039298
:10BBF00005932A4607F14403CDE9015BCDF800A087
:10BC000004966420F7F72EF84FF453700E4B05900E
:10BC10000393CDE9015BCDF800A004962A4629469E
:10BC200007F140036420F7F71DF851E64FF0FF33AA
:10BC3000994655E607F14403BB614CE778A701003C
:10BC400084A7010088A701008CA701002DE9F04F0F
:10BC5000B0F1000B8DB066DD9A4616460D46002405
:10BC60003AF91430002B5BDD4FF0FF394FF000083C
:10BC7000229F444513D03AF91830002B0FDD56F8B7
:10BC8000241056F8282055F8240055F82830891A31
:10BC9000C01A00F07DFBB842BCBF0746C14608F1A0
:10BCA0000108C345E5D1B9F1FF3F39D0209B00968B
:10BCB00009931F9B5A4608931E9B494607931D9B59
:10BCC000204606931C9B05931B9B0493199B03938F
:10BCD000189BCDE901A32B46FDF752FCA14525DDBC
:10BCE00019983AF9143050F8240056F8242055F8E1
:10BCF0002410029020980AAF06901F9805901E9875
:10BD000004901D9803900BA8CDE900702046FFF722
:10BD1000AFFADDE90A0100F03BFB169B23F81400A3
:10BD20000134A3459CD10DB0BDE8F08F19983AF9C4
:10BD3000193050F8290056F8292055F8291002909A
:10BD400020980AAF06901F9805901E9804901D98A1
:10BD500003900BA8CDE900704846FFF789FADDE9AA
:10BD60000A0100F015FB169B23F81900D8E700BF65
:10BD70002DE9F04FB0F1000B83B0DDE912C9DDF819
:10BD800064A0DDF86C804ADD00264FF0FF34DFF858
:10BD900094E0019302E00136B34540D01EF806005E
:10BDA0000028F8D1013408EB0400019B02E00134C3
:10BDB000A44534DD077805460130002FF7D06445EF
:10BDC00001932CDA149859F8247050F8240021F8C3
:10BDD000167022F81600159830F914701798005D47
:10BDE00023F81670169F0C9B37F9147023F8167001
:10BDF0000D9B9855189B185D0E9B98551A9B28789B
:10BE00005AF8247033F914500F9B43F82670109B96
:10BE100023F81650119B98550136B345BED103B097
:10BE2000BDE8F08FA82600202DE9F04F04461D46FE
:10BE30004FF01F339DB016AF7960CDE90A41D7E9C5
:10BE4000139A0E46396FC7E903330491F96EBB822A
:10BE500003913B6CB96E0E9302917B6C796EDFF8A7
:10BE600098E1DFF898C10F930191BB6C396ECDE971
:10BE70000C25904607F10C025D48CDE91039099276
:10BE8000FB6DBA6DCDF848A00091CDE907CEDFF883
:10BE900070C1796DCDE905C00A20FFF79FFB554AB7
:10BEA000D7F88C00D2E9023200210092642200F01F
:10BEB00059FA00285BD0BB6F002B58D0D7F88430DC
:10BEC000002B54D083467B6CCDE906680A933B6C0B
:10BED00007F10C06CDE9085313963B6FD7F888603D
:10BEE00004931296FB6ED7F8846003931196BB6E91
:10BEF000D7F88060029310967B6EFE6F01930F96C9
:10BF00003B6EBE6F0093796DD7E916230594CDF88B
:10BF100050B0CDE90DA6BE6C0A20CDF830900B963E
:10BF2000FFF76AFCD7F88C300BB3002307F10C0243
:10BF30000B92D7F8882005930A92D7F88420CDE990
:10BF4000039A0992D7F880202B460892FA6F7968F5
:10BF50000792BA6F20460692BA6CCDF830B00292C2
:10BF60007A6C01923A6C00924246FFF76FFEE31D35
:10BF700023F00703ADEB030D002C0DF1580C10DD81
:10BF8000AA1E7E6802EB44000DF1570132F9023F10
:10BF9000002BD4BF00230123824201F8013FF5D1D9
:10BFA0007E60BB6C796D0C937B6C0A200B933B6CB1
:10BFB000CDE90EACCDE909537B68CDF83490CDE9DD
:10BFC00006437B6FCDF8208005933B6F0493FB6E97
:10BFD0000393BB6E02937B6E01933B6E0093D7E994
:10BFE0001623FFF7C5FE1C37BD46BDE8F08F00BF26
:10BFF000EC1C00207C170020701C0020001D00207D
:10C00000A82600202DE9F04F4FF0000883B00192E0
:10C010008246894644460E9D574E584ADFF878B10D
:10C020002BE000232354002963D13AF91430544FF4
:10C0300022F8143039F91400524927F814003AF95B
:10C040001400514B2BF8140039F91400371921F85A
:10C0500014000199287831F9141023F814100D9B5D
:10C0600033F91410494B387023F8141008F1010803
:10C0700001340A2C05F1010537D02B7831190091D4
:10C080004348315D002BCCD14148DFF8F8C0DFF8E0
:10C090000CE10029ECD0215C3BF81470013149B26D
:10C0A000DEF800E0215422F814703CF81400344FFC
:10C0B000714527F81400DBDD31192CF814303548B0
:10C0C000DFF8C4C00B70314922F8143027F814305F
:10C0D0002BF8143020F814302CF8143021F81430D8
:10C0E00001340A2C05F10105C7D1404603B0BDE873
:10C0F000F08F234F32F9143039F914C037F9141086
:10C100003AF91400ACEB0101C01A009200F040F9BA
:10C11000204B3BF914C023F814003AF91430009A6C
:10C12000A3EB0C0C174903EB6C0322F8143039F91C
:10C13000143031F914C01448A3EB0C0C03EB6C035E
:10C1400027F814303AF9143095F800C02BF8143061
:10C1500039F9143021F81430019B311933F91430B6
:10C1600081F800C020F814300D9B33F91410074BF0
:10C1700023F814107AE700BFA8260020EC1C00204A
:10C18000001D0020D81C0020B01C00209C1C00209A
:10C19000841C0020701C0020C41C00207C17002080
:10C1A0002DE9F04F4FF0000983B0CDE90012984619
:10C1B0005F4D604B824695E8070003C34C460E9ED8
:10C1C000DFF89CB11A803BE000215A4F9E42DFF815
:10C1D00080E1DFF884C15848584A395565DB3AF99F
:10C1E0001430574FA15CEB53009B564F33F914307A
:10C1F000EB533AF91430544F25F80B30009B33F9C8
:10C20000143025F80E30019B33F914E04F4B25F81C
:10C210000CE038F914C027F805C00C9F17F804C0CB
:10C2200004F800C0385D814238BF0146A1540D9A20
:10C2300032F91420EA5209F1010901340A2C30D0F4
:10C2400038F91420404BB2424FEA440533F9143018
:10C25000BADC9E423E4A3F49EFDA364F35F80B00D2
:10C260003B5D096801335BB23B55354F35F802C081
:10C27000E85334488B4225F800C0DEDD0023364900
:10C28000AB526B522C4A2D492B52A3542E482F4AA5
:10C29000635401340A2C25F80B30EB534353AB5253
:10C2A000CED1484603B0BDE8F08F264B009FEA5E32
:10C2B000234B37F91410EB5E3AF91400891AC01AAF
:10C2C00000F066F8254B35F90B1058533AF9143045
:10C2D0001F4A591A03EB61031949A85E6B5237F9DB
:10C2E00014301D49181A03EB600316482B523AF913
:10C2F0001430114825F80B3037F91430124FAB5277
:10C30000019B0E4A33F914306B5238F91410A35CB8
:10C3100079530C99095D21540C99085D0B498342AE
:10C3200038BF0346A3540D9B33F914306B5282E798
:10C33000841C0020901C002024280020942500202C
:10C34000682E00202C260020682700206825002069
:10C35000802E00207C170020942E0020701C0020CE
:10C36000F8270020884210DB904210B40ADA441A01
:10C370000198521AC01A04FB00F494FBF2F210BCAC
:10C38000D0187047019810BC70471846704700BF1E
:10C3900081EAE173A3EBE17318B30028B8BF404210
:10C3A000F1B198421FDA820192FBF3F2402AA8BF52
:10C3B000402211498A5CC2F15A028AB10F4910B475
:10C3C000C2F15A0431F8122031F8141003FB02F3C1
:10C3D00000FB01F01B1403EB2043184610BC704710
:10C3E0000346184670479A0192FBF0F2402AA8BF14
:10C3F000402201498A5CE0E784A80100C8A8010046
:10C4000088420ADB40B1890191FBF0F04028A8BFC7
:10C410004020094B185C7047704751B1800190FB78
:10C42000F1F14029A8BF4021034B595CC1F15A00EA
:10C4300070470846704700BF84A8010070B40E68BA
:10C440000C89022E25DDA04223DB0B460125013E8F
:10C4500002E0844206DC15466A1C96429C8903F180
:10C460000403F6D101EB8505AE88ED88A6420DD018
:10C4700001EB8201CB88001B5D1B00FB05F0A41BB8
:10C4800090FBF4F41C4420B270BC704728B270BC1E
:10C49000704700250122E5E77F280CDC402824DADC
:10C4A0000F2824DC082827DA022829DB0428B4BF57
:10C4B000012002207047B0F5806F08DAB0F5007FE8
:10C4C0001CDAB0F5807FB4BF072008207047B0F5B4
:10C4D000805F05DAB0F5006FACBF0B200A20704713
:10C4E000B0F5005F0CDA0C2070470620704720285A
:10C4F000B4BF04200520704703207047092070470F
:10C50000002070472DE9F04F056889B01446ADB1A1
:10C51000394D3A4F3A4E4FF480722B4600923946CD
:10C5200000226020F6F7F0FB40F201122B46009249
:10C53000314622466420F6F7E7FBECE7314A8146B4
:10C540001368084601338A4613600DF0F9F8C9F8FC
:10C55000000020B12C4B00EB0A029A423CD9264F36
:10C560000025B846DFF8B0B040F20B124346009207
:10C57000264900226420F6F7C7FB0426012240F278
:10C580000F13D9F80000114600EB0A0C0593069032
:10C5900006ABCDE903B7CDE9015500966420CDF88F
:10C5A0001CC0F6F75FFB01224FF48873184905930E
:10C5B000CDE9025107AB114600960497019564201E
:10C5C000F6F750FB40F2111243460092214600223A
:10C5D0006420F6F799FBC7E70E4A2B46114602E0A6
:10C5E0000133322B05D051F8044B002CF8D142F81E
:10C5F000230009B0BDE8F08F2CA8010034A8010089
:10C6000038A80100DC1D0020943F002058A801003C
:10C6100078A80100141D00206CA801002DE9F04F3E
:10C620008046006889B08946C0B12F4D00232A4654
:10C6300002E00133322B1DD052F8041B8142F8D1A5
:10C64000002445F823400DF083F8284AC8F800403C
:10C650001368013B136009B0BDE8F08F4FF491738C
:10C660000A4600932249234B6420F6F74DFB09B09C
:10C67000BDE8F08F1F4E00243746DFF880B0DFF8AA
:10C6800080A04FF497723B4600921B490022642021
:10C69000F6F73AFB042501224FF49873D8F80010FE
:10C6A000642007910593114607ABCDE903B6CDE9A8
:10C6B00001440095F6F7D6FA40F231123B4600925B
:10C6C000494600226420F6F71FFB4FF499730A22B3
:10C6D00005930095CDE903A6CDE901441146024B2F
:10C6E0000020F6F7BFFACCE7141D0020DC1D002067
:10C6F000D0A701002CA80100F0A701007CA8010030
:10C7000018A80100134B1B68002B22DD2DE9F04116
:10C71000114C4FF000082746104E114D86B040F2E4
:10C720003F123B460092294600226420F6F7ECFABD
:10C7300001224FF4A071042305910093CDE9036415
:10C74000CDF8088001921146024B6420F6F78AFA70
:10C75000E5E77047DC1D00202CA801009CA9010022
:10C7600080A9010010B50446FCF79EFD04F1F0011C
:10C7700004F1B800FEF75EFC04F59470FBF7EAFAEA
:10C7800004F5EC70FAF70AFF04F5EE70FEF748FBCB
:10C7900004F5F870FCF736F804F51670FEF7CAFDDC
:10C7A00004F52470FEF77CFE04F52870FCF776FD96
:10C7B00004F2793001F042FC04F2A620FCF7C8F83C
:10C7C00094F8A6320BB9FCF7C9F804F52A70FBF708
:10C7D00079FE04F53F70FBF7F1F804F55C70FEF7A5
:10C7E00085FA04F55F7000F0DFFD0023044C194664
:10C7F00023604FF48862BDE8104002480CF0BBBFD4
:10C8000098190020182A002038B9064A1368013305
:10C810008B4205DD10600120704700231846014A55
:10C82000136070479819002008B5FAF73BFFFEF730
:10C8300065FAFEF741FEFCF791F8FBF74BFEFBF7BC
:10C84000C5F8BDE8084001F0F1BB00BF0022014B74
:10C850001A607047E01D0020024A1368013313601C
:10C86000704700BFE01D0020014B1868704700BFF3
:10C87000E01D00206E20704738B500240A4B0B4D98
:10C8800021464FF42A72C3E90044C3E902441C6103
:10C8900007482C600CF06FFF2146BDE838404FF48C
:10C8A000A07204480CF067BF4C250020E81D002052
:10C8B000EC1D0020942000202DE9F04F00279A461F
:10C8C0000D4695B00BAC0DF11C0881461646394655
:10C8D000222220460797C8E90177C8F80C700CF0AF
:10C8E0004AFF4FEAAA034D4A142BB8BF1423BD4296
:10C8F000C2E90077C2E90277176174DDC446C9EB6B
:10C90000C9714900CDE901774FEA490E0091691ECE
:10C910000597039706EB0E0208EB050A0491B9F19F
:10C92000000F16DD00210098ACEB080B101830F951
:10C93000025B9D4207DD9CF800700E5D01370136F9
:10C940008CF800700E55212938DD904201F101016B
:10C95000EDD10CF1010CD4457244E0D1019B002BC8
:10C960004AD1059A9DF82C609DF81C30002A50D1C0
:10C97000002528462F4629460DF11D020BB1012541
:10C9800028448B42C4BF19460127944202D012F8B2
:10C99000013BF3E7002F39D1002D34D100210B46A4
:10C9A0000DF131020EB101210B44944202D014F872
:10C9B000016FF7E721BB15B0BDE8F08F029EBBF118
:10C9C000000F2E4402960BDD049E5E4508DD039F9A
:10C9D0000126AF42B8BF2F46059603970196B4E7EC
:10C9E00001250195B1E700253B463E4628462F46E6
:10C9F00029460DF11D02C1E7084B029ADA60B0E743
:10CA0000064A9360D7E7054B1860C7E7034B5960A8
:10CA1000C2E7024A03991161AAE700BF7C25002002
:10CA20002DE9F04F95B000AF7B61D7F89430002826
:10CA3000BB60D7F89830C7E90621D7E91ECED7E901
:10CA40002C51D7F8B8407B60386240F37D81914625
:10CA5000DFF83083C44ED8F80020400002EB021209
:10CA600006EB8202A9F10203B246F860023A1E18F0
:10CA700033F9020F9E4222F8020FF9D123683B617D
:10CA8000FB69002B17DD7B69D8F800809E1E3346BA
:10CA9000B64AF86902EB481206EB4000023A33F955
:10CAA000028F834222F8028FF9D13B6A002B40F3B8
:10CAB0006D81AD4B9A460022C7F8B84047F6FF7625
:10CAC0005446C7F8B410DFF8C082B9697A6200230F
:10CAD0004FEA420B786A04EB0B09C34439F944ABC3
:10CAE000CB455344FAD182467862A14880FB0309C2
:10CAF000DB17C3EBA9031BB2002B21F812309946B8
:10CB000002DD5046184478629E42A8BF1E469C45EE
:10CB10000CDAB5F808902B6809F10109A5F808901E
:10CB200031F91290A9EB0C0A53442B60CE450CDD71
:10CB3000B5F80A906B6809F10109A5F80A9031F976
:10CB40001290A9EB0E094B446B60022A40F32D8131
:10CB50003B6A01329342BADCD7E92D143A69AE81BF
:10CB60001546844B786A83FB0553A3EBE27323607D
:10CB7000E3683A6A3B61FB6990FBF2F0002B40F3FB
:10CB8000EE807B699E1E6FF001054FF0000E47F6A8
:10CB9000FF7CFB69754A03EB0508C7F82480D7F8CA
:10CBA0000490D7F8088078611046002302F5A07B36
:10CBB00030F920AB83455344FAD16D4880FB03A084
:10CBC000DB17C3EBA0031BB29E45B8BF9E469C4536
:10CBD000A8BF9C46434526F8023F09DD0B8908683B
:10CBE00001330B81B6F90030A3EB080A504408600A
:10CBF000994509DD4B89486801334B81B6F900300E
:10CC0000A3EB090A504448600B2D23EAE37000F2BD
:10CC100091803B69013503443B61E3607B6A0232EA
:10CC2000AB42C1D178690FFA8EFE0FFA8CFCFD6819
:10CC3000A1F80EC02B46083323F00703ADEB030D1C
:10CC4000FB69A1F80CE0A3F1040C3B6A6946002BD8
:10CC500038DDBB6900269A1E154440F24458A946A7
:10CC6000A1F1020E32F902AF256AAAEB000323EA12
:10CC7000E3731BB2AAF1970AAB421FFA8AFAC8BF44
:10CC8000C4E90763C2452EF8023F06F1010602D847
:10CC9000A3690133A3619145E4D1B1F90030002BC0
:10CCA00010DDA36A3A6A1A441046013304E031F9F0
:10CCB000022F002A40F39C8098421D4603F1010395
:10CCC000F5D1A06247F6FF703B690326984293FBBB
:10CCD000FCF1B8BF18460023274AC7E90E33C7E95D
:10CCE0001033C7E91233254D254BA16000B207F17F
:10CCF0002801C7E90C23C7E90A65FFF79FFBE26833
:10CD00006369012A1146B8BF01219B0193FBF1F32E
:10CD100023EAE373984209DAE369B34206DD41F29C
:10CD200087339A4202DC012384F824305437BD460D
:10CD3000BDE8F08F63690135034463617B6A0232A9
:10CD4000AB427FF431AF6DE723683B61FB69002B99
:10CD50003CDD3B6ADFF82C805B00FB6093E647F626
:10CD6000FF7C4FF0000E62E7EC1D002094200020B5
:10CD70006766666656555555E8034000F401320073
:10CD8000D0074000E81D00209420002047F6FF72E5
:10CD9000AA813A69174B104683FB0003A3EBE273A9
:10CDA0002360E36800203B61EDE631F912903869B9
:10CDB000D7F8B830B9F1000FA8BF48445B683861B4
:10CDC0009944D7F8B830C3E90009C1E647F6FF70C7
:10CDD000FA69084BA2F1040C3A69A88183FB02634B
:10CDE000E068A3EBE273044A23603861CA6069E734
:10CDF000A56267E7565555550000FF7F002347F6AB
:10CE0000FF7C18462DE9F043584CDFF86C818F1EEB
:10CE1000136053609360D36013610431A2F1040E78
:10CE200037F9023F002B44DD9DB26E1E092E43D818
:10CE30001E4618449C42B8BF1C469C45A8BF9C4651
:10CE4000B9424EF8046FEBD1494F3D7945BB61467D
:10CE50000129B8BF012128461646DFF820C1DFF8B6
:10CE600020E109B202F10C08B4F57A7F33680BDADD
:10CE700094FBF1F5032D07DD312B05DD8EFB0395CA
:10CE8000DB17C3EBA50333605CF8045F2B445B1036
:10CE900046F8043B46451844CCF80030E4D13D79CF
:10CEA000344B156183FB0013A3EBE070D060BDE849
:10CEB000F08300263346BDE7A5F10B06092E11D9F4
:10CEC000A5F11509B9F1090F1E4612D803EB43036A
:10CED0005B00A8FB0353DB0803339BB21E461BB267
:10CEE0003044A7E75B1005339BB21E461BB23044AB
:10CEF000A0E7A5F11F09B9F1090F0ED9A5F129097C
:10CF0000B9F1090F11D8DB00A8FB0353DB08043B80
:10CF10009BB21E461BB230448CE7C3EBC303A8FB95
:10CF20000336F608304433B284E7A5F13309B9F18A
:10CF3000090F04D93D3D272D0CD918447AE703EB9E
:10CF4000C303A8FB0353DB08093B9BB21E461BB27D
:10CF500030446FE7C3EBC3035B00A8FB0353DB085C
:10CF6000263B9BB21E461BB2304463E70080FFFFA6
:10CF70004C25002056555555CDCCCCCCD021002089
:10CF80006766666684B02DE9F047002482B081466A
:10CF90000BA880E80E00524D9DF85070DFF86C81B0
:10CFA000504EDFF86CA115F8013BD3B9119B122B41
:10CFB00002DCB9F1000F34D04FB340F2B312334664
:10CFC0000092494900224920F5F79EFE002305F80A
:10CFD000043C0134032CE6D102B0BDE8F04704B0B4
:10CFE000704708EB4403DB880B9A9A4202DD0D9BE5
:10CFF0001E2B3BDC4FF4E372334600925146002275
:10D000004920F5F781FE002305F8043CE1E740F2F2
:10D01000B7123346009235493A464920F5F774FE77
:10D02000D7E74FF4CD722F4B009231494A46492041
:10D03000F5F76AFE129B062BCBDD002F44D1109B27
:10D04000B3F57A7F36DD159B052B33DC139BB3F5E7
:10D05000FA7F2FDA4FF4D3723346009225493A46CD
:10D060004920F5F751FE05F8047CB2E74FF4DE7273
:10D070001C4B0092204900224920F5F745FE012370
:10D0800005F8043C67B14FF4E072334600921B4947
:10D0900000224920F5F738FE002305F8043C98E704
:10D0A00040F2C3123346009215493A464920F5F73B
:10D0B0002BFE8EE740F2AB1233460092114900225C
:10D0C0004920F5F721FE84E740F29F123346009293
:10D0D0000D494A464920F5F717FE05F8049C78E704
:10D0E0004F250020D0A9010090AA0100CCAA010080
:10D0F000E4A9010034AA010000AB01001CAB01004F
:10D100004CAB010058AA01000CAA0100ACA9010017
:10D110005CAB010082B010B401A981E80C00DDE92C
:10D120000234012B17D098B1511001EB4201994202
:10D1300002DCD11E032907D9023B032B08D8012C9E
:10D1400006DD023A042A03D80022064B5A709A7070
:10D1500010BC02B07047042AE5DC0022014B5A7073
:10D160009A70F5E74C25002030B400250124104BBF
:10D17000D81CDA7819786AB979B199790131C9B2CC
:10D180000A29997101D9DC709A7101338342F0D177
:10D1900030BC704719B15D72F7E79971F5E75A7ABB
:10D1A0000132D2B20A2A5A7284BFD9705972ECE79E
:10D1B0004C25002000212DE9F043984601250B461F
:10D1C0002B4E89B0129F149C2A4891463180B17031
:10D1D000F21C12F8011B31B930F813108F4202DD36
:10D1E0001E2CC8BFF5540133032BF2D16C4615AD8C
:10D1F0000FCD0FC495E80F0084E80F0012AD95E83D
:10D200000E004046FFF7BEFE1FAB93E807008DE817
:10D2100007001DAC94E80C0041464846FFF77AFF32
:10D22000002342F210741A4620993078A3B1022BE1
:10D2300001D00133FAE7C2B940F2DC539F4206DC69
:10D2400043F698239942CCBF01230023B37009B061
:10D25000BDE8F043FFF788BF0028EAD1A1424FF0B4
:10D260000103E6DD18461A46E3E73070E4E700BF45
:10D270004C250020ACA901002DE9F04FA3B00025FA
:10D28000DDE93C876E4681468B4617AC14922046FA
:10D290002C22002115939DF800A10CF06CFACDE929
:10D2A0000F74CDF838800DF1D40C0DF11C0EBCE8D4
:10D2B0000F00AEE80F009CE807008EE807000DF1B4
:10D2C000B80CBCE80F00C8F80050C8F80450C8F803
:10D2D0000850C8F80C50C8F810503D607D60BD6023
:10D2E000FD603D610FC69CE807002D9B86E80700A6
:10D2F00059462C9A4846214EFFF792FB0DAFCDF8C8
:10D3000048A00FCE0FC736680FCC3E6002AE0FC6E6
:10D310000FCC0FC694E80700159B86E807002D99EF
:10D32000174C01912C99149A009148465946FFF7E1
:10D3300041FF23683E9A01330A2B08BF2B462C99E4
:10D3400048462360FFF75AFD3E9B3F9ADB68938275
:10D35000BAF1000F09D10B4B5A7952B9D878401B5A
:10D3600018BF012023B0BDE8F08F284623B0BDE8E8
:10D37000F08F042023B0BDE8F08F00BF7C25002093
:10D38000E81D00204C25002030B9064B187810B15C
:10D390000138C0B2187070471423024A184613703F
:10D3A000704700BFE41D002001464FF4A4720148FD
:10D3B0000CF0D6B98C170020014B1878704700BFCD
:10D3C000E92100202DE9F04FB1B0074605A8CDE9CD
:10D3D0000223DDF80081FCF783FF0EA888220021DC
:10D3E0000CF0C9F900204FF0420C2126804BDFF8E9
:10D3F000109293F902A001900DF1BC0ECDF80081BE
:10D400000F2302E013F1FF3324D303EB031209EBE4
:10D41000820232F90C20BA4204BF34461D465245FE
:10D4200002F10508EEDADEF80010013000914099B3
:10D4300011F803B00099BBF11F0F4144CEF8001062
:10D44000E0D13F990029DDDD019913F1FF3311444B
:10D450000191DAD2013E731CAEF1040EACF1020C64
:10D46000CED12122624BDDF80480B3F804E0B3F999
:10D470000660B3F908C03A9B03F19C0131F8023D04
:10D480004BB1734507D20EAB53F82230B34202DAE8
:10D49000C445C0F2A18012F1FF32EFD200261E2C4B
:10D4A000C8BFC4F12103A5F1030ECCBF5BB20323B7
:10D4B000BEF1090F01D8022C58DC0022029BB3F503
:10D4C0007A6F51D93A9B198B5A2994BF00210121B7
:10D4D00040F2EE243A9B1B8EA34243D93A9BB3F809
:10D4E0004C30A34294BF002301236EB13A9C248B9D
:10D4F000142C09D91E2807DD0398052804DD19B965
:10D5000013B99DF81A30C3B13A4BB3F90A30BB4294
:10D5100021DA3A9B3A98452F93F82A1093F82B403A
:10D5200090F8290093F8283013DC091B052912D83C
:10D530001B1A052B0FD8052A0DDD2D4B2E4A197805
:10D5400041981368014499424DDD01331360002076
:10D5500005E0592F42DD00231846274A136031B0F9
:10D56000BDE8F08F0023C0E70021B1E7C3F122023C
:10D57000A242A2DD033575454FF000029EDB1F4D30
:10D580000EEB0E1E04F100414FEA4E0E0339B5F8C2
:10D5900004807144DFF86CC00EF1660E09EB4101A6
:10D5A000A6445D00C8F1000A02390CEB4E0C0835A8
:10D5B00003EB0408A4F10309C84509DB0B4605EB9E
:10D5C000010E33F9024FA245A8BF01327345F8D1CD
:10D5D00044316145F0D171E7012660E73A9DAD8B9A
:10D5E000142DB8D9A1E7002301201360B7E700BFCD
:10D5F0008C1700208C0D0020E021002058D2010063
:10D60000182A0020202B002070B58AB09DF8785091
:10D610009DF87C60C0B9B9B9374C2178C9B1132ADB
:10D620004BDC0F9A632A48DC133346DB0E9B092B35
:10D6300043D8324B324AD9691368994255DD0121EA
:10D640000B44136021701FE000222B4B1A700AB0AC
:10D6500070BD1D99104606911B99CDE9075605919D
:10D660001A990491199903911799029116990191A8
:10D67000189900911946DDE90E23FFF7A3FE2070EB
:10D6800010B12048F9F78AFFFDF7BEF82478054667
:10D69000FCB11D4C1D4E2388327801331BB2238010
:10D6A000002AD4D1632BD2DD0220FDF753FA0123E7
:10D6B0006422AB7733702280C9E7104B0F99B3F91E
:10D6C00018209142B6DC002201210D4B21701A6016
:10D6D000DAE70E4E0C4A33781480002BB7D00320C3
:10D6E000FDF738FAAC773470B1E7002308481360CF
:10D6F0002370F9F753FFC7E7E92100208C170020BA
:10D70000E4210020ECD00100EA210020E8210020E3
:10D71000F8CE0100054A92F84E30834204DA8B427B
:10D72000B4BF002001207047012070478C170020F3
:10D730003228CCBF00200120704700BF2DE9F04FF8
:10D74000013883B0002801916CDD012872D04FF0C0
:10D7500000094FF0010C09EB000303EBD3735B10DE
:10D7600032F9131032F910404500A14204DD22F8CD
:10D7700013400C4622F8101032F919104FEA490BE9
:10D78000A14202EB0B0A04DD22F81940515332F991
:10D79000191032F913408C4205DD22F8131022F8DB
:10D7A0000B4032F9134006460BF10201555E02EBC5
:10D7B0004C0E22F81350545232F90B503EF9028F9E
:10D7C0000CF1010CA845F9DB711E02EB410301E0ED
:10D7D0000E4601391F4633F90249AC42F8DC8C454C
:10D7E00007DCAEF80040A7F800800E46BAF90050FA
:10D7F000E4E7019B22F80B408B423D8018DBE146B9
:10D8000016DD48450EDD09F1010C8445A3D102EB7C
:10D8100049094000B9F90030115E8B42C4BFA9F834
:10D8200000101352019B32F9130003B0BDE8F08FD2
:10D83000B01EE6E791460220ECE700BF2DE9F04F6D
:10D84000013800EBD07383B05B10002801936CDDCE
:10D85000012872D04FF000094FF0010C09EB0003D2
:10D8600003EBD3735B1031F9132031F910404500FD
:10D87000A24204DD21F81340144621F8102031F9AA
:10D8800019204FEA490BA24201EB0B0A04DD21F8F3
:10D8900019404A5331F9192031F91340944205DDFA
:10D8A00021F8132021F80B4031F9134006460BF103
:10D8B00002028D5E01EB4C0E21F813508C5231F9AF
:10D8C0000B503EF9028F0CF1010CA845F9DB721EDA
:10D8D00001EB420301E01646013A1F4633F90249C3
:10D8E000AC42F8DC944507DCAEF80040A7F80080B5
:10D8F0001646BAF90050E4E7019B21F80B40934229
:10D900003D8018DBE14616DD48450EDD09F1010CCE
:10D910008445A3D101EB49094000B9F900300A5E02
:10D920009342C4BFA9F800200B52019B31F91300A8
:10D9300003B0BDE8F08FB01EE6E789460220ECE7B1
:10D94000831A042B10B413DDDC1EB1F90430002A55
:10D950000B804B8031F9143008DD4000A0EB42020F
:10D960000A44014421F8023D8A42FBD110BC7047B1
:10D970005C1E032C08BF9C1EE7E700BFF0B4044602
:10D98000049E0846DDE90551A642DDF81CC019DDFC
:10D9900004F10044AF1E013C07EB460705EB4405CC
:10D9A0008E1C06E09C42B8BF1C46BD4226F8024FC2
:10D9B00008D035F9024F9442F4DD1446BD4226F8F2
:10D9C000024FF6D1F0BC6246FFF7BABFF0B40028B0
:10D9D0000F46DDE90561DDF81CC014DB013006EB04
:10D9E00040048D1C06E09842B8BF1846B44225F8A2
:10D9F000020F08D034F9020D9042F4DD1046B44213
:10DA000025F8020FF6D13846F0BC6246FFF798BF02
:10DA10002DE9F043B1F9009002284FEA4918DDE9F9
:10DA20000767C2E90088DDE909CE21DD8C1E5B01B4
:10DA300076017F01043204EB4000023103E0A84686
:10DA400031F9029C0432B1F90050B1F9024006FBF1
:10DA500005F503FB0454156802310CFB054407FB74
:10DA6000094408FB0E4481424FEAA4245460E6D1E5
:10DA7000BDE8F0832DE9F041884684B04C000834BD
:10DA800004AFBD6B24F00704ADEB040DBE69039534
:10DA9000FD6904AC0195009602947D6BFFF76EFF63
:10DAA0003B6B21460293FB6A03950193BB6A404698
:10DAB0000093D7E90823FFF7ABFFBD46BDE8F0812F
:10DAC0002DE9F041884684B04C00083404AFBD6BAA
:10DAD00024F00704ADEB040DBE690395FD6904ACA9
:10DAE0000195009602947D6BFFF770FF3B6B21461A
:10DAF0000293FB6A03950193BB6A40460093D7E902
:10DB00000823FFF785FFBD46BDE8F0812DE9F04F02
:10DB10008FB00AAF7D6D9A461B1A023300F10308DD
:10DB20008B465919FB6B18EB050804461646FB603B
:10DB300000F0AA804FEA8809002934D109F10A09C6
:10DB400029F00709C7F808D0ADEB090D08953E6D1F
:10DB50000DF128090796FE6C13460696BE6C5A46D0
:10DB600005967E6C414604963E6C0396BE6BCDF8DE
:10DB70000890CDE900A6FFF7A3FF002C0DDBFE689F
:10DB80000235013409EB850906EB440459F8043BDE
:10DB90005B1124F8023DA642F8D1D7F808D014371B
:10DBA000BD46BDE8F08F8B000A3323F00703C7F8AA
:10DBB00004D0ADEB030D08953A6D0AAB0792FA6CF1
:10DBC00009F10A090692BA6C29F0070905927A6CE4
:10DBD00004923A6C0392BA6BCDE900A2BB605A463C
:10DBE00002933346FFF746FFADEB090D0895396DFB
:10DBF0000DF128090791F96C33460691B96C5A4624
:10DC00000591796C20460491396C0391B96BCDF87C
:10DC10000890CDE900A14146FFF752FF631C9A45E9
:10DC200011DDFE68BA68E91CB31E02EB810103EB4B
:10DC30004A0A06EB440251F8043B5B1122F8023F0A
:10DC40005245F8D1FE60002C0DDDFE68E91C09EBA1
:10DC5000810106EB440251F8043B5B1122F8023DBE
:10DC60009642F8D1FE60BB68023559F8252053F87A
:10DC700025301344FA689B1122F81430D7F804D0E9
:10DC80001437BD46BDE8F08F8B000A3323F007033D
:10DC9000E946ADEB030D08953E6D0DF1280807969A
:10DCA000FE6C13460696BE6C5A4605967E6C04962C
:10DCB0003E6C0396BE6BCDF80880CDE900A6FFF759
:10DCC000D9FE544512DAFA6804F10044013C0335E8
:10DCD000931E02EB440608EB850803EB4A0A58F84A
:10DCE000043B5B1126F8023FB245F8D1CD4614370C
:10DCF000BD46BDE8F08F00BF2DE9F04788B09946DA
:10DD00004FEA430808F1080424F0070408AFADEB1C
:10DD1000040DD7E90D563C6BCDE90656BD6AFE6A87
:10DD2000059403953C6A7D6A049608AECDE90165C9
:10DD30000094FD6BFFF7EAFEB9F1000F10DD023C25
:10DD4000A044A6F1020A34F9023F3AF9022F9B1AC5
:10DD5000AB42CCBF5B1B03EAE37344452380F2D1A3
:10DD6000BD46BDE8F08700BF1F232DE9F043274ED5
:10DD700087B00D46804600932549334664201446FB
:10DD80000022F4F7C1FF4FF02009012200270421EF
:10DD900020482B4600910390114664200496CDF84C
:10DDA0001490CDE90177F4F75DFF4FF0250E4FF0A9
:10DDB000010C1948A5EB0801490903900496CDE927
:10DDC00001774A464346CDF814E0CDF800C0642000
:10DDD000F4F748FF294651F8043BA342FBD02B2718
:10DDE00000220124C5F11F030C481944CDE901228A
:10DDF0000390049649092B4605970094202264203D
:10DE0000F4F730FF07B0BDE8F08300BF88AB010036
:10DE100094AB0100A8AB0100B4AB0100CCAB010096
:10DE20000B68934209D070B50D461446064622464B
:10DE300029463046FFF798FFF9E770472DE9F04390
:10DE400000248FB00990081ACDE9072127460693D0
:10DE500082100B94169E06E00134B2EB840F4FF053
:10DE60000107C0F2AB8051F80439B342F4D0002F5F
:10DE700040F0C68000244FF0040901224321624D86
:10DE8000624BC71B0591CDE90335114609AB6420F0
:10DE9000CDE90144CDF800900C97F4F7E3FE0122A0
:10DEA00044215B4B05910393114608AB6420049514
:10DEB000CDE90144CDF80090F4F7D4FE4FF001080D
:10DEC0004523544F0593424641460BAB64200495CD
:10DED0000294CDF80090CDF804800397F4F7C2FEC9
:10DEE00046204D4B42460590039364200CAB0495AD
:10DEF000CDE90184CDF800904146F4F7B3FE069BCE
:10DF0000DDF81CC09E46ACEB030022460B9480104B
:10DF1000043B05E00134B0EB840F4FF001025CDB01
:10DF200053F8041FB142F5D0002A66D114460026EA
:10DF30004FF0040801225421384BACEB0E0CC4EB1B
:10DF4000AC04CDE904510393114607ABCDE901665A
:10DF5000CDF8008064200D94F4F784FE0122552151
:10DF60002F4BCDE904510393114606ABCDE9016671
:10DF7000CDF800806420F4F775FE012456220BAB27
:10DF80000592214622460296CDF80080CDE9037520
:10DF900001946420F4F766FE5720224B059003930A
:10DFA000CDE90146CDF800800495224621460DAB0F
:10DFB0006420F4F757FE0FB0BDE8F0833B226420E5
:10DFC0000092114B002218490B94F4F79DFEDDE9F5
:10DFD00008500B9C281AA7004CE74D220A4B0092D0
:10DFE0001149002264200B94F4F78EFE0B9ADDF8A1
:10DFF0001CC09400DDF818E099E70B94A40096E7A4
:10E000000B94A70036E700BF88AB0100ECAB010022
:10E01000F8AB010084A7010004AC010018AC0100BA
:10E0200024AC010030AC0100E0AB01000022024B47
:10E03000C3E900221A817047642200200278014B54
:10E040001A707047D4180020314B1B78002B5AD01F
:10E050002DE9F04F16462F4A87B0894680460024A6
:10E060002D4F1368DFF8B4B0DFF8B4A0013E14E020
:10E070003D5D38F91410022D2BF8101005F1010E3A
:10E0800039F914109CBF5FFA8EF53D55032D2AF81F
:10E09000101017D001340A2C0CD04FEA440C0CEBB2
:10E0A0000401C81816F8011F0029E1D139550134BF
:10E0B0000A2CF2D10133022BC8BF0023136007B032
:10E0C000BDE8F08F0CEB04035B000BEB0301086869
:10E0D000534402901868B1F804C09B88049002A9C8
:10E0E00028460192ADF81430ADF80CC0FFF7A6FB3E
:10E0F00004A928F814002846FFF7A0FB019A29F884
:10E1000014001368C6E7044AC2E90033138170475C
:10E11000D41800207022002064220020EC2100206E
:10E1200028220020F0B483000A3323F007030028DC
:10E1300000AFADEB030D30DD6B4600260439B200B5
:10E1400002F1804292F880C292F8815292F88242A3
:10E1500092F883225FFA8CFCEDB2E4B2D2B20136BF
:10E1600083F800C05D709C70DA70BCF1000F03D0C2
:10E170000CF1FF3C83F800C0202D9CBF01355D7081
:10E180000CB1013C9C700E2A9CBF0132DA7053F82E
:10E19000042BB04241F8042FD1D1BD46F0BC7047EA
:10E1A00092F82230002B42D1F0B500288BB00E46F9
:10E1B000054614460FDD936942189A420FDB00238F
:10E1C0001A4684F82130237D93429CBF012384F8B2
:10E1D00020300BB0F0BDF2D1D3698B42EFDD362297
:10E1E00094F82130124F013384F8213011493B4615
:10E1F000009264200022F4F787FD4FF03C0C0020D1
:10E20000012104220C4B049794F82170CDE90110F0
:10E21000009203930322CDF814C007AB6420CDE92C
:10E2200008650797F4F71EFD94F82120CBE77047A7
:10E2300050AC010064AC01008CAC01002DE9F04F42
:10E2400098468DB0DDE91653012DA946B8BF4FF0B1
:10E250000109012B9C464FF00004B8BF4FF0010CA0
:10E26000189E09923788B6F804E01268D8F8006062
:10E2700005FB072503FB0E66002895FBF9F596FBC9
:10E28000FCF6CDE90A442ADDA446A146A24602399D
:10E2900001EB40000894CEF1000B079031F9023FEA
:10E2A0005A1B22EAE272334403EAE37397420EEB0D
:10E2B000030403DC0120D21B089092445B4505DC7B
:10E2C0004FF0010C002CB8BF6442A144079B994257
:10E2D000E4D1089B002B53D1BCF1000F53D1012492
:10E2E000642500270426DFF8B490DDF824A0274B2E
:10E2F000284622462146CDE9033905955346CDE906
:10E3000001470096F4F7AEFC4FF0650C204B224617
:10E3100021462846CDF814C00393CDF8109043460B
:10E32000CDE901470096F4F79DFC4FF0670C194BBF
:10E33000224621462846CDF814C00393CDF810900C
:10E340000AABCDE901470096F4F78CFC4FF0680C5E
:10E35000114B22460393CDF810900BABCDE901474A
:10E36000009628462146CDF814C0F4F77BFCDDE981
:10E370000A23CAF80020C8F800300DB0BDE8F08FBD
:10E38000CDF828A0A8E7CDF82C90A8E79CAC010018
:10E39000ACAC0100BCAC0100D0AC010050AC010041
:10E3A00070B19A4215DC0F4A1368C72B01DC0133A8
:10E3B00013600D4B187808B181F001001970704797
:10E3C000084B1A68C72AF4DD1860074B0120197042
:10E3D00070470022034B1A60034B18780028EDD0D9
:10E3E000EAE700BF782200207E22002090B130B4FE
:10E3F00041F674146FF4D97CA1F1D905A5426144AA
:10E40000187808D9B1F5BE5F0ED908B901221A7083
:10E4100030BC70477047E22A18DCB1F5BE5FF4D813
:10E420000028F5D1014609E06FF4E37443F6CC010E
:10E4300022448A428CBF0021012108B901221A70AE
:10E440000029E5D030BC00221A707047B1F5BE5FDC
:10E4500006D90028DCD143F677318A42D8DDD5E7EA
:10E460006FF4E37143F6CC045118A1428CBF002134
:10E4700001210028E4D143F677308242C8DDDDE790
:10E4800010B401299DF8044008D900B924B11378CB
:10E49000022B01D80133137010BC7047002BF4D14C
:10E4A0000028F3D013781CB1022BF3D910BC7047AD
:10E4B000002BF1D0013B1370EEE700BF2DE9F04FC8
:10E4C000BC4DADF2E44DCDE91423DDF820452B78A9
:10E4D00034A81693231C18BF01238B461993FBF70E
:10E4E000FFFE1E22002124A80BF045F93C2200214A
:10E4F00047A80BF040F978220021DEA80BF03BF989
:10E500001E2200212CA80BF036F956A83C2200212F
:10E510000BF031F90023DDF82005CDE91C33ADF80F
:10E520007830CDE91F33CDE921332393002840F023
:10E53000E4834FF022081027DDF81835A2AA0693CD
:10E54000DDF81C3584A90593DEAB01932CAB009359
:10E55000C0AB0293CDE9037847ABF8F7BFFE0123C8
:10E56000002440F26B100093DFF854A2924B424615
:10E570003946059003936C20DDF81C35CDE9014444
:10E58000CDF810A0F4F76EFBC0AB0393DDF818359F
:10E59000DDF820050793DDF81C35A2AA069356ABDB
:10E5A0000293DEAB01932CAB009384A947ABCDE97A
:10E5B0000478FBF7E9F8C0AB0393DDF81835DDF814
:10E5C00020050793DDF81C35A2AA069356AB0293EB
:10E5D000DEAB01932CAB009384A947ABCDE9047863
:10E5E000FBF716FAC0AB0393DDF81835DDF820050C
:10E5F0000793DDF81C35A2AA069356AB0293DEAB57
:10E6000001932CAB009384A947ABFCAECDE9047811
:10E61000FBF74EF80DF58D652146782230460BF05C
:10E62000AAF82146782228460BF0A5F8634BDDF8BE
:10E6300020051A68DDF844355278B3F92430089281
:10E64000DDF8182507930692DDF81C2547AB0592E7
:10E65000DEAA0292CDF810800397CDE90065A2AA48
:10E6600084A9FCF713FDDDF820350DF5CA79A34226
:10E670000DDD4F4655F8041B56F8040BFDF788FED8
:10E68000DDF820350134A34227F8020BF2DC102418
:10E690002225DDF84425DDF81815B2F924201846A6
:10E6A000CDE90812DDF81C25CDE905450792C0AA81
:10E6B000049256AA0392DEAA02922CAACDE90092F5
:10E6C00047ABA2AA84A9FBF735FB4FF4DF76002302
:10E6D00001202146384C2A46CDE901330090DDF86F
:10E6E0001C356C20CDF810A003940596F4F7BAFA07
:10E6F0009DF8D930DDF820050093A2AA47AB84A984
:10E70000F9F762FBDDF8200500280CDD4A46662497
:10E7100009EB4001B2F9003004FB03F39B1222F82D
:10E72000023B8A42F6D1DEAB029324ABCDE90093E3
:10E73000A2AA47AB84A9FCF787FBFEF73DFE0028A1
:10E740004FD19DF8D63003F0FF01002B3AD1169B34
:10E75000012B40F0C8829DF8EF30002B00F0C382FF
:10E76000242275A80BF007F81E2074ACFA214FF490
:10E77000167211254FF496774FF0320C4FF03C0E85
:10E78000A081462005264FF064080223E06225811F
:10E79000E781A4F810C0A4F814E02046E18061816C
:10E7A0006282E2822660C4F82880C4E90C33FCF758
:10E7B000C1FD17E0E70F0020E4AC01000C060020CB
:10E7C00050AC010047AA4946DDF82005FAF72EF8BB
:10E7D000002800F08882DDF84C3503F50870FCF75E
:10E7E000A9FD74AC0026DDF820352660B34249DD72
:10E7F000DFF8788140F20522434600925549002215
:10E800007020F4F781FA012540F2062204235249D0
:10E810000592CDE902612A462946009370202346DD
:10E82000CDF810A00195F4F71DFA022740F2072059
:10E8300023684A4A2946CDE9026205902A4609EB37
:10E84000430370200195CDF810A00097F4F70AFA61
:10E850004FF402702368424A059047A800EB430337
:10E86000CDE90262CDE900752A46CDF810A029460F
:10E870007020F4F7F7F92368DDF820252B44934244
:10E880002360B7DB0126002540F20A220420354B25
:10E890003146CDE904A2CDE90165324600900393EB
:10E8A0006D200DF5A463F4F7DDF9DDF860754FF028
:10E8B00022081397DDF81875149A1297DDF81C7565
:10E8C0001CAB1197C0AF0E97DDF80C750A930D972E
:10E8D0001FAF0C97DDF81475DDF810350B97102776
:10E8E000CDE905B256AA09930492DDF80835DEAAEF
:10E8F00003922CAA08930292159B24AACDE90092B8
:10E9000047AADDF82005079384A91346A2AACDF8EB
:10E9100040800F97FDF788FA40F226200096124EAD
:10E9200039460590CDE901554246CDF810A0039631
:10E93000DDF81C356C20F4F795F9DDF82015A942B7
:10E9400034DDDDF80825159B40F22A28A946971EDC
:10E950009E1E0FE0ECAC010084A7010004AD010095
:10E9600010AD01001CAD0100E4AC010050AC010091
:10E97000A9421BDD37F9022F36F9023F2560C4E9B1
:10E9800001230135002BF3D001210423C54ACDE931
:10E990000031CDE90292CDE904A8234603224120AB
:10E9A000F4F760F9DDF82015A942E3DC1423159D86
:10E9B000149E1FAA01921CAA314600920293DDF810
:10E9C00008252B465846FDF7EBFB2946DDF80C35AC
:10E9D000DDF808250A20FCF7F9FC2946DDF80C359E
:10E9E000DDF808250A20FCF7BDFCDDF80C352A46C9
:10E9F0000093DDF80815DDF810350A20FCF70EFD50
:10EA0000DDF80C352A4602931FAB01931CAB31464F
:10EA100000935846DDF80835FDF7F4FA3346814691
:10EA200000955A460A210020F8F7BEFD3146DDF870
:10EA30000C255846FFF708FBFEF7BEFC169B002688
:10EA4000022B08BF40F001005FFA89F31793DDF84D
:10EA50000C75C3B2DFF858A2DFF8588216933DADAB
:10EA6000149B3BF9160033F916C08F4B0146334413
:10EA70001A90286062463878CDF86CC0C4F800C09F
:10EA8000FFF7B4FC1AF806301897002B40F0058108
:10EA9000DDF84C153A7891F8A63222B1824A925D9F
:10EAA000002A40F0E480002B00F0E58018F80630E2
:10EAB000022B00F2018123462A4639783046F9F7C5
:10EAC00057FF002800F01F811BAB3978002200930C
:10EAD00030461AABF9F70AFD18F806201A9B296888
:10EAE00003FB02F3C2F1030201FB02336F4880FB18
:10EAF0000312A2EBE3732BF8163018F806201B9BC9
:10EB0000216803FB02F3C2F1030201FB023380FB25
:10EB10000312A2EBE373149A22F81630169A624B92
:10EB200038789B5D1799009208EB0602FFF7A8FC66
:10EB300017F8013B0AF80630B9F1000F03D108F8C5
:10EB400006900AF80690002E00F08F800226149B93
:10EB50000BEB06089F19DDF80C3503F1010A38F9B3
:10EB6000020F37F902CF1AF8011F2B46009400223A
:10EB70002860C4F800C03046F9F7B8FC01362A68AE
:10EB800023680A2EA8F800203B80E8D1B9F1000FD5
:10EB900040F3B1802822002128460AF0ECFDDDF880
:10EBA0002005002840F3B7800026DDF80C35013839
:10EBB000DDF814251844013B13F8011F19B1116841
:10EBC00045F826100136834202F10402F4D1F6B270
:10EBD0003E2200210DF5E9700AF0CDFD822742F2B8
:10EBE00010204FF0220CDDF81835214600933246F4
:10EBF00020802B46032084F802C06771FBF7B8FF22
:10EC0000149C9DF8D530DDF80C25159D00920293DB
:10EC10002A46DDF80835214658460196F8F786FD64
:10EC2000DDF80C2521465846FCF788F800229DF8AF
:10EC3000D9305946022B0CBF13460D230A20CDE9CB
:10EC40000023DDF80C352246F8F7E8FCDDF80C353A
:10EC5000584600932A46DDF808352146F9F71CFC92
:10EC600019980DF2E44DBDE8F08F0126F8E6032275
:10EC700008F8062003BB169B7BBB18F806203978E2
:10EC80002B4600943046F8F73DFF2A6823682BF89E
:10EC90001620149A22F8163040E7DDF84C3593F828
:10ECA000A63200E728AD01007422002056555555C4
:10ECB0007C2200208022002023462A460021304664
:10ECC000F9F756FE00287FF4FFAE02460146009495
:10ECD0002B463046F8F716FFF6E64FF00003002209
:10ECE00008F80630CBE7DDF84C3574AC03F5167048
:10ECF000FCF720FB76E5002682E7DEA9FFF712FA93
:10ED0000DDF8200515E43978024600942B4630469C
:10ED1000F8F7F8FED8E600265AE700BF2DE9F04FD5
:10ED2000C7B2C0F3072883B0474501900C992BDC8C
:10ED30009DF806A052000AF100499DF807B009F1BC
:10ED4000FF390AFB023301EB490901EB4B0C0D992A
:10ED500008F1010801EB470EDA4518D849461C4670
:10ED60000C4D34F9170031F9026F8542B8BF0546E2
:10ED70008642B8BF08808C451444F2D12DB20137C9
:10ED800047452EF8025BE7D103B0BDE8F08F014D97
:10ED9000F5E700BF0080FFFF2DE9F04F05468FB07B
:10EDA0004FEA410A08AF18463A60884652460021A9
:10EDB0006C007B60D7F844900AF0DDFC2246386C8A
:10EDC00000210AF0D8FC002D67DD0AF108033E6C33
:10EDD00023F0070B4FEAA803FB603B683119B960C9
:10EDE0009C1EC7F814D0ADEB0B0D08ABA51C184644
:10EDF000294652460AF0B4FCF96802464046FEF73E
:10EE00009DFCB8F1000F014653DD00202246034669
:10EE100032F902CF8C4508BF184601339845F7D127
:10EE20000522ADEB0B0D15234FF0290E07926FF461
:10EE3000247240F23E6CCDE903E3069208AA0293E5
:10EE40000095CDF814C03A610192BD6CFA6C43464E
:10EE50008A1A2944FEF75AFE3B697A689D1E0AEB1E
:10EE6000040134F9023F35F9020F1B1AA3EB090321
:10EE7000002B238006DD10889BB218441080308858
:10EE8000034433808C4202F10202EAD1BB680236AD
:10EE90009E42D7F814D00C46A3D100233A68C8EBA1
:10EEA000C8084FEA48081C3722F80830BD46BDE8BC
:10EEB000F08F6FF424724FF0050E152340F23E6C74
:10EEC0002920ADEB0B0DCDE9062E08AA0493029381
:10EED0000095CDF814C003900192B86CFA6C4346CB
:10EEE0008A1A01440020FEF711FE04EB0A01CDE767
:10EEF0002DE9F04F9FB08A0008AF7A61083222F006
:10EF00000702ADEB020DB8614E0008A80029796335
:10EF1000B860FE6119DD4FF4004E47F6FF7C002516
:10EF2000B11ED7F884200144D7F88C00023A961914
:10EF30000DF11E04023822F8025FB24221F802EFFE
:10EF400020F8025F24F802CFF5D1B969786B4A0046
:10EF500000FB02F2083222F00702ADEB020D08AA14
:10EF600000297A6040F3E3807A6400223A6300EB80
:10EF7000D07222F00102043B0A32D7F88010BB6342
:10EF800022F007033B617B690439CB18F9603B65CC
:10EF90003B69C7F82CD0ADEB030D08AAADEB030D10
:10EFA00008ABBB647B6BFA64002B40F33981D7F864
:10EFB00090200023013A144647F6FF797A62904682
:10EFC000D7F88C209A46951E7A6CC7E90F33CB464A
:10EFD000FE68D7F838E0A2F1020C3C620BE0FC6C52
:10EFE0004A4524F8130002DA01468146FB633A6D74
:10EFF0000133964221D056F8040F5EF8042F35F8FD
:10F00000021FC2EBA0121144298018F8014F10B260
:10F01000E4072CF8020F4946C7F854B0DFD4BC6CA3
:10F020005A4524F81A0003DA83467865C7F840A0E9
:10F030003A6D0AF1010A9642DDD1C7F828A01525DC
:10F040004FF0000B05266FF4247840F23E694FF034
:10F05000290AFA6C3C6A0092F86B6431CDE9066BC0
:10F060000395CDE9015A4FF00042CDE90498FEF72F
:10F0700043FECDE902A5CDE9066BCDE904980195E3
:10F08000BE6C4FF000420096796DBB6A6431386CFB
:10F09000FEF732FE796B7B6AFD6C0B4459461846CD
:10F0A0007B6C14F8012F0233D2074BBF35F81B20BD
:10F0B00036F811200BF1010B0131844223F8022CA8
:10F0C000EFD17A6CF9693B6B0A447A647969BA6B5F
:10F0D00001330A44BA63BA693B639A42D7F82CD029
:10F0E0007FF456AFD7E90C897A68FB69A2F1020C6C
:10F0F000BA6800269E4692469D1E1544B9F1000F3F
:10F1000011DD29466046AAF1020230F9023F31F9C9
:10F11000024F9C42B8BF0B8032F9024F9C42C8BFDD
:10F120001380AA42F1D101364645F444E6D17B6B07
:10F13000002B71DDBB68D7F888109C1E2646FA6943
:10F14000881ED7F88C10A2F1020CD7F8188002396B
:10F1500003EB0C0500EB020E35F8023F36F8022FE8
:10F160009B1A20F8023F31F9023F704593FBF8F3F8
:10F170000B80F1D1D7F88430991E0A46BB6803EBA7
:10F180000C0534F9023F32F9020F002BB8BF5B4285
:10F19000984200DA1380A542F3D1BB680846634465
:10F1A0009C46FB690B441A463CF9023F30F9024F7A
:10F1B000002BB8BF5B429C42B8BF03809042F3D1A2
:10F1C0006FF00044D7F890302646581E7B6B0344FE
:10F1D0009C46034604E09442A8BF14469C450AD0CE
:10F1E00013F8015F31F9022FED07F4D49642A8BF5E
:10F1F00016469C45F4D1D7F8842010F8015F118899
:10F2000015F0010FA1EB04050ABF891B15801180C1
:10F21000834202F10202F0D15C37BD46BDE8F08FB7
:10F220000024152505266FF4247840F23E694FF03E
:10F23000290AFB6C2046009307942346CDE90586F6
:10F24000CDE90359CDE9015A4FF0004248F263017C
:10F25000FEF752FDCDE90664CDE90498CDE902A59B
:10F260000195BB6C204600934FF00042234648F2C4
:10F270006301FEF741FD24E7002824DDF0B40025FA
:10F280008E1EAC464FF0FF3700E01D4636F9024FA8
:10F290006B1C944203DD6445C4BFA4462F469842CC
:10F2A000F3D17B1C11D07B0031F917001FB1CA18B4
:10F2B00032F9022C1044AF4203DA1944B1F902309A
:10F2C0001844F0BC7047002070470020F0BC704725
:10F2D00070B40024061E1C6020460EDD023901EBCE
:10F2E000460631F9024F944202DD1D6801351D606A
:10F2F000A042B8BF2046B142F3D170BC704700BFF6
:10F3000070B40024061E1C6020460CDD023901EB9F
:10F31000460631F9024F944203DD1D682044013551
:10F320001D60B142F5D170BC704700BF2DE9F04FB0
:10F3300082461646524600258BB000AF8846386D8F
:10F34000520000213C6E9946BB61C7F808A00AF044
:10F3500012FA0AEBDA7323F001030A3323F00703EE
:10F36000ADEB030DC7F820D0AA45ADEB030D256129
:10F37000C7F81CD025606560A560E56084F811A021
:10F38000257440F3F980504647F6FF7E7A6DCC46EF
:10F39000013A7A609246321F02EB80037B613B6D3B
:10F3A000AB467146A8F10408A3F102097D623C66F0
:10F3B00011E07345A8BF7346D7E9084524F8150046
:10F3C000A8BF18467C6A86467869013490427C6200
:10F3D0000CF1010C31D0B86952F8043F20B19CF80F
:10F3E000000000FB0333DB1158F8040FBD6DC3EBC5
:10F3F000A01347F6FF708342A8BF034661480E463C
:10F400008342B8BF034618B229F8020F1AF8014F19
:10F410002C57002CCDD18B42A8BF0B46FC691E4651
:10F4200024F81B00A8BF184601467869734690422D
:10F430000BF1010B0CF1010CCDD1D7E9184293422D
:10F44000A8BF13469642A8BF16461BB2524236B218
:10F450009342B8BF13469642B8BF164632464FF0A5
:10F46000000C4FF00040FE60FE6D7968D6E900E9BF
:10F47000BE683B610E44B346B7F9106012B27E61BC
:10F48000E0464E4663466FF00045BA617862D7F8B1
:10F49000509041E03A6A786932F91820002A5ADB24
:10F4A000002802DB3869121A12B229F8132008F179
:10F4B0000108724518DDB4F808A022680AF1010AB3
:10F4C000A4F808A039F913A094F91100AAEB0E0AC8
:10F4D0005244226094F910209842C8BF63749A4243
:10F4E000B8BF237439F9132096420ADD6289606837
:10F4F0000132628139F91320A2EB060A8244C4F872
:10F5000004A0786A01339042B8BF10469542A8BF64
:10F5100015468B45786227D011F8012FB86D8256B9
:10F52000002AB7D1FA69B86932F91C20002A09DB30
:10F53000002802DBF868121A12B229F813200CF125
:10F54000010CB6E70028F5DA121A02EAE27212B2EA
:10F5500029F81320F3E70028A4DA121A02EAE2726B
:10F5600012B229F81320A2E72DB203B22C37A381DF
:10F57000E581BD46BDE8F08F2B464FF000404FF0CF
:10F58000FF35F3E70080FFFF2DE9F047824686B0A4
:10F590000620DDE912981C460E4617461425F5F79D
:10F5A000BBFAF5F763FE159B3A460493149B31466C
:10F5B00003930F9B0290CDE9004305950E9B5046A7
:10F5C000FFF7B4FE00254FF02E0C0121022718484A
:10F5D000184E2346CDE9030652466920CDF814C0E3
:10F5E000CDE901150097F3F73DFBAA4528460FDD4D
:10F5F000A31E03EB4A0A33F9021FA1EB0902002AFA
:10F60000C8BFAD18B1EB080148BF40185345F2D14F
:10F61000109BAB4207DB119B8342D4BF002001202B
:10F6200006B0BDE8F087012006B0BDE8F08700BF56
:10F6300008B0010040AD0100002820DDF0B48E1EAE
:10F6400006EB4006B14218D0571C38460B46B1F9BC
:10F65000004033F9025FAC4207DD0D801C8092F957
:10F66000004090F9005015700470B34200F10100A1
:10F67000EDD10231B1423A46E6D1F0BC7047704755
:10F680002DE9F04F8046450005F1080485B000EBF8
:10F69000D07A24F0070407302AF0010A00AF20F0E6
:10F6A0000700ADEB040D08F1090424F00704EB4654
:10F6B000ADEB000D0AF10A0020F007006E46ADEB3D
:10F6C000040D6C46ADEB000DE946C7E902210AF1D5
:10F6D000020A08F102021F2120467B600AF04BF863
:10F6E0005246484600210AF046F8B8F1000F7B6800
:10F6F00007DD324606EB0800911B02F8011B82422F
:10F70000FAD14FF0FF3A2A46F96858467B600AF072
:10F7100027F8594632464046FFF78EFF023D08F172
:10F72000FF3E7B6806EB0E01AB44013EB14218D0B0
:10F730003BF9025911F901299D4202F1010C10DB3C
:10F74000A05C22441F28927860D01E2860D81E2A10
:10F7500096BF4FF0FF3204F80C0004F80C20B142C1
:10F76000E6D1B8F1020F04F1010113DD0B46FF20D1
:10F77000A64402E0013373450CD05A781F2AF9D110
:10F780001A781E2AF6D89A7801331E2A98BF187064
:10F790007345F2D1B8F1000F2EDDFB6804EB0806CB
:10F7A000F96004E00134A64203F1020323D0627839
:10F7B000FF2AF7D1257894F802C039F8150039F8F6
:10F7C0001CE08346704528BFF346B3F90020B96BAF
:10F7D0000A449345E6DA704538BF70460134654502
:10F7E0008CBF29F81C0029F81500A6420AF1FF3A3F
:10F7F00003F10203DBD1F9684246B86809F0B0FFB3
:10F800000AF101001437BD46BDE8F08F1F2A06D06B
:10F810001E2A88BF6FF0690204F80C2086E70AF1FF
:10F82000010A04F80CA029F81A507FE7FFF728BF57
:10F830000048704758010020024B1A680260187D8A
:10F84000704700BF58010020024B5A680260587D83
:10F85000704700BF5801002030B44FF080430022B1
:10F860000F2121202225102483F8082183F80A2162
:10F8700083F8090183F80B111A739A735873D973BB
:10F880001D725C72DA7793F8211041F0010183F860
:10F89000211093F8211062F3410183F8211030BC4C
:10F8A000704700BF10B44FF0804485B00DF1100CCC
:10F8B0000CE90F00BDF800302382BDF802306382EE
:10F8C000BDF90430A382BDF90630E382BDF80830EB
:10F8D0002383BDF80A306383BDF80C30A38305B0E1
:10F8E00010BC70474FF08043988370474FF08043BF
:10F8F000988B70474FF0804383F82000704700BF1B
:10F900000123002110B50A4A0A4C2377917210B9DD
:10F910004FF08042D3704FF0804301229870002155
:10F920001A700A2000F098F90022024B1A7710BDD5
:10F93000842200200000105001234FF0804010214D
:10F9400010B4034A034CA372436010BC11607047AB
:10F95000580900208422002001234FF0804010210C
:10F9600010B4044A044C6372C0F8043110BC116036
:10F97000704700BF5809002084220020E0220021A7
:10F98000014809F0F8BE00BF800100402DE9F041B8
:10F9900005461E4B1E4886B06A1E13F8011B8342A3
:10F9A00002F8011FF9D101242B464FF0A50C0027C6
:10F9B00002262A681748D11780FB0202DFF8608010
:10F9C0001548C1EB222243F8242B2146CDF814C060
:10F9D0002246CDE90308CDE9014700966220F3F7FE
:10F9E00041F94FF0A60C0D48CDF810800390CDE9F9
:10F9F0000147009605F1260322462146CDF814C0A2
:10FA00006220F3F72FF906B0BDE8F081280000402E
:10FA1000540000407978787828D4010088AD01003E
:10FA200084AD010070B5E022064600210B4809F0C4
:10FA3000A2FE002401234FF08042094D09492B7793
:10FA40000A208C7293702146137000F005F92C7710
:10FA50003046BDE87040FFF799BF00BF800100400D
:10FA6000000010508422002010B50446FFF78EFFDE
:10FA700031234FF0804004F1500203F1600150F84F
:10FA80002110013B212B22F8021DF6D14FF08040BE
:10FA900004F19C0203F1600150F82110013B22F8AF
:10FAA000021D591CF6D110BD4FF0804270B503798C
:10FAB00009B201FB03F1948B8B11A342B8BF23461B
:10FAC00001250024022106889BB24380A2F80C6124
:10FAD000A2F80E31074E084B357709205C7282F888
:10FAE000035182F802112146A2F8005100F0B4F847
:10FAF000347770BD00001050842200204FF0804306
:10FB000093F81401704700BF4FF0804393F817013A
:10FB1000704700BF0023094A82F832305064916474
:10FB200072B6012382F8403000BFB2F852309BB267
:10FB3000002BFAD062B6B2F85000704700001050A7
:10FB40002DE9F047102220204FF0300A5021602488
:10FB50004FF040094FF001084FF4807E4FF4007CD5
:10FB60004FF480674FF400660825124B83F800239A
:10FB700083F8040383F808A3DFF83CA08AF8234045
:10FB800083F8032383F8059383F8091383F80A1392
:10FB900083F80B1383F80F43C3F800801A601860D2
:10FBA000C3F800E0C3F800C01F601E601D60BDE820
:10FBB000F08700BF00E100E000ED00E04FF40042FC
:10FBC000034BC3F88020BFF34F8FBFF36F8F704795
:10FBD00000E100E000220121034BA3F86E20A3F80E
:10FBE0006A20A3F8681070470000105010B5174C39
:10FBF00084B094E80300029002A88DF80C1000F085
:10FC0000ADF800F0B5F8FFF79BFF62B600F062FABE
:10FC1000A36804A840F80C3D00F056FA00F09EFAE4
:10FC200000F0AAF900F00EFB094B1A6922F0040259
:10FC30001A61BFF34F8F0721064A82F824105A69D0
:10FC400042F010025A6104B010BD00BF7899010063
:10FC500000ED00E00000105008B500BF72B6084A81
:10FC6000135C3BB900BF30BF62B600BF72B6135C15
:10FC7000002BF7D00023135401B1884762B608BDAA
:10FC80008422002000200A4B0A4913F8012B10445B
:10FC90008B42C0B2F9D1064B1A78AA2A01D00020B3
:10FCA0007047DB7B181AB0FA80F04009704700BF3C
:10FCB000800040008F0040002DE9F041142000F04A
:10FCC0004DFD0028B8BF0730C51000234FF0A040FD
:10FCD00001E08D4228DB027E0133591E002AF8D153
:10FCE0000126B046194F00234FF0A04402E0A9427C
:10FCF000267406DCA27E0133591E002AF7D0BDE827
:10FD0000F08172B6BFF34F8F4FF6FE724FF6FF735E
:10FD10003A877A877B873B87BFF34F8F01F0B2F832
:10FD200084F8118062B6DEE772B6BFF34F8F4FF6EC
:10FD3000FE714FF6FF72054B198759875A871A874C
:10FD4000BFF34F8F01F09EF862B6C9E70000105074
:10FD50004FF0A04301225A74704700BF0246034B84
:10FD60000068127918601A71704700BF9422002051
:10FD700070B5FFF787FF01220021334BD9705A720B
:10FD8000DA7200285CD0314AD278D2B21A720022DC
:10FD900001242F492C4B8D789A725A731D734D781C
:10FDA0000E781E751D77CD78097983F8215083F878
:10FDB00020105A749A741C749A7018B3234A51789C
:10FDC0001A78C9B2D2B28A4208D08A42B4BF01328C
:10FDD00002F1FF32D0B28A421870F6D11B4B1A4999
:10FDE0001A794B78D2B2DBB29A420AD09A4203F126
:10FDF000010096BF03F1FF33C3B2DBB29A424B70EE
:10FE0000F4D170BD1A78D2B2B02A08D0AF2AD4BFCC
:10FE1000013202F1FF32D1B2B02A1970F6D10A4A8A
:10FE20005378DBB2082BECD0072B03F101018ABF1A
:10FE300003F1FF33CBB2DBB2082B5370F4D1E0E710
:10FE4000E0221A72A3E700BF0000105080004000BB
:10FE50009422002007490B78DBB2834208D09842F5
:10FE6000CCBF013303F1FF33DAB283420A70F6D11B
:10FE7000704700BF0000105008B5FFF703FF18B12E
:10FE8000024B5878C0B208BDB02008BD80004000C9
:10FE9000014B1878704700BF00001050084A537893
:10FEA000DBB283420AD0984203F1010196BF03F10D
:10FEB000FF33CBB2DBB283425370F4D1704700BF43
:10FEC00000001050014B5878704700BF00001050E0
:10FED00010B50446FFF73CFF4FF0A043206861686F
:10FEE000A26807C310BD00BF38B54FF0A044E37D42
:10FEF000DBB2042B28D0082B19D0022B09D0012308
:10FF0000184A137000BF4FF0A042137300BF537321
:10FF100038BD154D15496079FAF738FB61792868C5
:10FF2000FAF77CFB62792B6813442B60E7E7104BF0
:10FF3000D0E9051259609A60236A5BBA0A4A1846EA
:10FF40001360FAF7EDFADAE7074D0A492079FAF774
:10FF5000FBFA21792868FAF735FB22792B681344DC
:10FF60002B60CCE7842200209C220020200000503F
:10FF70000C1A0020240000501021264B0020D3F83A
:10FF8000802042F00102C3F880201A6C22F00102A6
:10FF90001A641A6842F001021A60D3F8802022F035
:10FFA0000202C3F880201A6C22F002021A641A6856
:10FFB00042F002021A60D3F880200A43C3F880207E
:10FFC0001A6C0A431A641A680A431A60D3F880202C
:10FFD00022F02002C3F880201A6C22F020021A645A
:10FFE0001A6842F020021A60D3F8802022F0400202
:10FFF000C3F880201A6C22F040021A641A6842F09A
:020000021000EC
:1000000040021A60C3F80801C3F80411C3F80011D4
:10001000704700BF00000250034BD3F8C0301842B5
:100020000CBF0120002070470000025038B572B6A6
:100030004FF040540125642084F8245000F0B8FBB0
:1000400000F03CFB00234FF47A7084F8253084F8EC
:10005000815000F0ADFB00F031FB62B638BD00BF4F
:1000600010B572B64FF040540123642084F8253057
:1000700000F09EFB00F022FB002384F8243084F87B
:10008000813062B610BD00BF14200122002130B5BE
:100090000A4D89B02D780A4C05900A4808AB03F840
:1000A000015DCDE90111CDE9030400921146642000
:1000B000F2F7D8FD9DF81F0009B030BDB700400031
:1000C0009CAD0100A4AD01000268014B1A607047AD
:1000D000A022002038B5FFF7D5FD0F23F0B94FF06F
:1000E00040524FF00104D9B2013B072B82F82B108C
:1000F00082F8284082F82800F5D1042382F82F30B6
:100100004FF040530121002283F8281083F8282063
:100110004FF47A70BDE8384000F0DCBB4FF040513E
:10012000012500240C4806E081F82B20013B81F8D2
:10013000285081F82840027A0E2A8EBF0F22027AB8
:10014000D2B29342DAB2EFDA4FF04052024B5B7A0E
:10015000DBB282F82F30D3E780004000F8B5FFF71C
:1001600091FD4FF0405401250026074684F8256094
:100170004FF47A7084F8205084F8275000F0AAFBDE
:10018000642084F8255000F0A5FB84F824506420F6
:1001900000F0A0FB84F8256007BB06231C4D84F803
:1001A0002730EB7884F826302B7884F842304FF0F3
:1001B000405401230022697840F24C4084F84610F4
:1001C00084F8442084F8453084F8413084F8403085
:1001D00000F080FBAB7884F84430F8BDFFF754FFA3
:1001E0000C4B9B7A88B94FF04052DBB2084D84F833
:1001F0002730E978074B82F82610DB7A29780B4400
:100200000B3BDBB282F84230D1E7053BEBE700BFA6
:10021000A02200208000400020B9064A064B106052
:100220001860704703490548034B054A08601A6087
:10023000704700BFA8220020A42200202D0001004A
:10024000610001004FF04053F0B406240122002564
:100250000A26FF2083F8D64093F8D7100F2764F3BF
:10026000030183F8D710042183F8D86083F8402174
:1002700083F8D00083F87F5093F88C000526104354
:1002800083F88C0093F88C0040F0020083F88C0017
:1002900093F8910064F30300032483F8910083F83A
:1002A000901083F88D1083F8A02093F8A10065F3D7
:1002B000010083F8A10083F8947093F8880010433C
:1002C00083F8880093F88900104383F8890083F845
:1002D000F12083F8874083F88E4083F8D22083F89A
:1002E000D52083F8AB6083F8AD5083F8AC4002248E
:1002F000072083F8AE1083F8AF1093F88B1064F3E7
:10030000061183F88B1083F8930083F8B020F0BCBB
:10031000704700BF08B5084B1B6843B1F4F7A2FC57
:10032000F4F772FCBDE808400020F4F735BC034B3D
:100330001B68002BF2D108BD44100020481000209B
:100340000E4B5A78824211D0597A79B90C4930B49F
:100350000A7001221D780B4C5870013890422570AC
:100360004FF0020103D930BC1A7070477047187AF9
:1003700030BC002818BF0A461A7070474009002098
:1003800056090020AD220020014B5860704700BF85
:100390004009002070B404460646044D0FCD0FC43A
:1003A0002B683046236070BC704700BF40090020B6
:1003B000034B044A19781278034B59701A7070472E
:1003C00056090020AD2200204009002008B5002079
:1003D000FFF7B6FFBDE80840FFF79CBF10B572B647
:1003E0000023074C236062B6142000F0B7F900F038
:1003F00065F920680028D4BF0020012010BD00BF8F
:10040000B022002010B598B101280DD0002213466B
:100410000A4C22721846FFF793FF22786078084949
:10042000084B08701A7010BD044C03462072F1E7A7
:10043000FFF7D4FF014C03462072EBE74009002090
:1004400056090020AD22002038B5084D084C2B7A03
:1004500022789A4205D02BB90520FAF77BFB2B7A3C
:10046000237038BD0420FAF775FBF8E74009002037
:10047000AC22002070B5124C637A0BB1237A03B919
:1004800070BD00F011F90F4B1B68A3EBD302904233
:10049000F6D9A3EB13139842F2D20023637272B61B
:1004A00000F040FA62B6084D084E094B09490A4A65
:1004B000A07A2E60BDE870400B601360FFF740BF6C
:1004C00040090020B02200209410002005090100FE
:1004D0007D4400004810002044100020F0B51D4C61
:1004E0008BB0E37A0646022B154603D026732561AE
:1004F0000BB0F0BD237A002BF8D0174B53F8203007
:1005000003EBC2031F79012F16D00023637201A8E9
:10051000F9F7E6FE9DF81330A3B100219DF81330E2
:100520000E4A6172D75C6378BB42DFD03846FFF772
:1005300007FFFFF7EFFED9E76378002BE5D167727D
:10054000A772E4E7637A002BEDD0267325610BB028
:10055000F0BD00BF40090020A8AD010054090020F3
:10056000084A08B590F82030D17ADBB2994207D01A
:100570001846D372FFF7E4FEBDE80840FFF7CABE95
:1005800008BD00BF4009002010B40124094B022817
:100590001C700AD0012801D010BC70470229FBD181
:1005A000002AF9D11A7010BC7047A142F8D010BCD3
:1005B000704700BF9E250020024B1878B0FA80F0EB
:1005C000400970479E25002038B500240220FFF71F
:1005D00019FF094B5C7272B600F0A4F962B60748C5
:1005E000074D084B0849094A04600D6020461A600F
:1005F000BDE83840F4F7D0BA400900204810002088
:100600000509010044100020941000207D440000E2
:1006100070B5164C8AB0E37A022B01D00AB070BDD7
:10062000257A002DFAD16378022BF7D00120FFF74D
:10063000E9FE217B0E4B226953F8213001A803EB20
:10064000C2031E79F9F74CFE9DF813302BB12846F2
:100650000AB0BDE87040FFF773BE3046FFF770FE8A
:10066000012E04BF6672A672D8E700BF40090020C1
:10067000A8AD010000220721034B04481A6058600E
:100680009A601960704700BF10E000E0FFFF0F00A4
:100690000022044B98681A60C0F57F2000F6FF70B6
:1006A000704700BF10E000E0034B9868C0F57F2062
:1006B00000F6FF70704700BF10E000E0002382B03A
:1006C00000280193B8BF0730019BC010984206DD97
:1006D00000BF019B01330193019B8342F8DB02B011
:1006E000704700BF054A0649937CD27801335B000E
:1006F000934000FB03F091FBF0F0704700001050B6
:1007000000B4C404054A937AD27ADBB20AB1013349
:100710009840034B93FBF0F0704700BF000010506F
:1007200040420F00054A937AD27ADBB22AB1012205
:10073000134402FA03F390FBF3F0704700001050EB
:10074000054A00EB8000937CD27801335B00934034
:10075000000190FBF3F070470000105041F2883325
:10076000124A00FB03F0137B0001DBB25A1E062A7B
:100770000DD9082B12D0092B15D0A3F10B02032A97
:100780000ED90F2B0CBF01234FF0FF3300E00133D4
:10079000064AD278934090FBF3F070470A23F7E7BC
:1007A000063B9B00F4E70C23F2E700BF000010506B
:1007B000124B00EB80001B7B0001DBB25A1E062AA5
:1007C0000DD9082B12D0092B15D0A3F10B02032A47
:1007D0000ED90F2B0CBF01234FF0FF3300E0013384
:1007E000064AD278934090FBF3F070470A23F7E76C
:1007F000063B9B00F4E70C23F2E700BF000010501B
:10080000034B044A5B7C03F0010352F82330184782
:1008100000001050C0AD0100134B1B7BDBB25A1E11
:10082000062A0DD9082B18D0092B1BD0A3F10B02D7
:10083000032A14D90F2B0CBF01234FF0FF3300E024
:1008400001330949094AC9788B4000FB03F382FB55
:100850000320DB17C3EB601070470A23F1E7063B68
:100860009B00EEE70C23ECE700001050676666661D
:10087000034B044A5B7C03F0010352F82330184712
:1008800000001050B8AD010070B5012200243B21DA
:10089000042688B008AB43F8040D0B4D0B48CDE996
:1008A00001240591CDE90305114600966420F2F775
:1008B000D9F9074B07985C7100F080F821460520B4
:1008C000FFF7CAF908B070BDC8AD0100D0AD010096
:1008D0008422002008B5FFF793FFBDE80840FFF72A
:1008E000D3BF00BF08B5FFF7C3FFBDE8084000F065
:1008F0001DB800BF08B5FFF7BBFFBDE8084000F01A
:100900002DB800BF08B57A20FFF7B2FFBDE8084058
:1009100000F03CB8002000F081B800BF012000F0DA
:100920007DB800BF00F062B800F06CB8012830B4A8
:100930004FF000024FF0020438BF01200121054BA7
:10094000054D1A702A719C709860DA605A7019709F
:1009500030BC70470000085084220020012830B4C9
:100960004FF000024FF0020438BF01200121054B77
:10097000054D1A706A719C709860DA605A7019702F
:1009800030BC7047000009508422002001284FF03D
:1009900000024FF0010138BF012010B4054B064C96
:1009A0001A70227199709860DA605A70197010BCD0
:1009B000704700BF000008508422002001284FF03B
:1009C00000024FF0010138BF012010B4054B064C66
:1009D0001A70627199709860DA605A70197010BC60
:1009E000704700BF0000095084220020012000222F
:1009F0000249034B08711A70704700BF842200201F
:100A000000000850012000220249034B48711A706F
:100A1000704700BF842200200000095010B40B4A28
:100A20000B4983B0CDE9001202AB03EB800353F80E
:100A3000082C9378DBB2012B04D10021054C043043
:100A40002354117003B010BC704700BF0000095060
:100A50000000085084220020034AD2F8803023F09E
:100A60000103C2F88030704700000250034AD2F8F8
:100A7000803043F00103C2F880307047000002501C
:100A8000034BD3F88000C04300F00100704700BF63
:100A9000000002504FF48072DCF808301A61704791
:100AA000002823DDF0B5DCE9013ED3F80130002455
:100AB0001E7C0CE0DCF800703F5D07FB055503FB76
:100AC00005F35B1242F824300134A0420DD051F8F6
:100AD000045BDEF81030002EECD103FB05F39B1015
:100AE00042F824300134A042F1D1F0BD704700BF7C
:100AF0004FF48072DCF808301A617047002821DD5D
:100B0000F0B5DCE9013E00241E7C0CE0DCF800704E
:100B10003F5D07FB055503FB05F35B1242F82430EC
:100B20000134A0420DD051F8045BDEF81030002EE5
:100B3000ECD103FB05F39B1042F824300134A042B2
:100B4000F1D1F0BD704700BF4FF48072DCF808307F
:100B50001A617047002823DDF0B5DCE9013ED3F8C7
:100B6000013000241E7C0CE0DCF800703F5D07FBC8
:100B7000055503FB05F35B1242F824300134A04213
:100B80000DD051F8045BDEF81030002EECD103FBE1
:100B900005F39B1042F824300134A042F1D1F0BD9E
:100BA000704700BF4FF48072DCF808301A6170475C
:100BB000002823DDF0B5DCE9013ED3F80130002444
:100BC0001E7C0CE0DCF800703F5D07FB055503FB65
:100BD00005F35B1242F824300134A0420DD051F8E5
:100BE000045BDEF81030002EECD103FB05F39B1004
:100BF00042F824300134A042F1D1F0BD704700BF6B
:100C0000DCF80430F0B4D3F801305C7F9CB90028E4
:100C10000FDD9B68DE889D8851F8043B013403FB9F
:100C200006F393FBF5F3A0424FEA831342F8043B2B
:100C3000F2D1F0BC70470028FBDD9B68DCF8004077
:100C4000DF88013C9E88204414F8015F51F8043B82
:100C5000A04205FB033307FB03F393FBF6F34FEAD4
:100C6000630342F8043BEFD1F0BC7047704700BF0C
:100C700000280BDD10B4002451F8043B01349B0123
:100C8000A04242F8043BF7D110BC7047704700BF48
:100C90002DE9F0410E4688B0022107460120654645
:100CA000F3F778FC00231946043806F5086406F6C5
:100CB000081C079350F8046FA4F50862B60952F8AF
:100CC000883B9B1B94421944F9D10434A4450791F5
:100CD000F0D191FBF7F1AB6807911A88002A53D045
:100CE0005888121A1202091A92FBF1F1B1F5DC7F51
:100CF000A8BF4FF4DC7119616A6840F2E11ED2F8B6
:100D00000120002690684FF0020C8488012201FB2C
:100D100004F10912FF29A8BFFF211D4F1D4CC180FE
:100D2000CDF814E0CDF800C01146CDE90347CDE978
:100D300001666420F1F796FF01244FF004084FF498
:100D4000F172154B0592214622460393049707AB97
:100D500002960194CDF800806420F1F783FF40F201
:100D6000E31CAB680D4804970390CDE90146CDF82C
:100D70000080103322462146CDF814C06420F1F7DC
:100D800071FF08B0BDE8F0814FF480711961B3E7DD
:100D9000A0AE0100ACAE0100C8AE0100D4AE0100AF
:100DA000F3F7F2BE08B5F3F715FFBDE808400021E0
:100DB0000120F3F7EFBB00BF30B595B02022002132
:100DC0000CA808F0D8FC294C29492A4D2A48CDE91D
:100DD0000854CDE90A01294A294B0E9293F8812043
:100DE00002AC8DF83C2093F881308DF83D30F5F75A
:100DF000EBFF8DF83E00F5F7EDFF8DF83F00F5F7BE
:100E0000EFFF8DF84000F5F7F1FF8DF84100F5F7A1
:100E1000F3FF8DF84200F5F7F5FF1190F5F7F8FFB5
:100E20001290F5F7FBFFADF84C0008A8F9F772FA3D
:100E3000F5F7F4FFF9F7EEFE002303220293A382F5
:100E4000C4E90133C4E903338DF81D20FBF712FD1B
:100E500006ABADF81E0093E803008DE8030094E8AC
:100E60000F00F9F7CFF915B030BD00BF6D0A0100D2
:100E7000D5080100590A0100810A01006E3816FAEE
:100E80000000105070B5002301223F21482608259C
:100E9000022484B001A8CDE9013303938DF80760E3
:100EA0008DF808508DF809208DF80F208DF80A4034
:100EB0008DF80D10FFF70CF804B070BD02FB01F2C5
:100EC0001212FF2AA8BFFF22028070472DE9F043CB
:100ED0002F4E97B02F4D11AC0AAF904699460C910A
:100EE00096E80F0084E80F001EABC4E902752046A7
:100EF00015A91593EFF7C4F996E80F00264E0DAD2E
:100F000085E80F002146C5E902762846EFF7B8F9D3
:100F10000520F3F701FE0521D0F801200B90D2E95E
:100F200002309A8816AEDA8006F8401D0A903146E3
:100F30000120F3F7A1FD0221184B44F0010445F014
:100F400001050846CDE908450793CDF81890F3F759
:100F500021FB04468822002108F00DFC234631467F
:100F600040462222F5F760FFC0270121062604250E
:100F70000B480C4A2346CDE903200597CDE901161D
:100F8000009522226420F1F76DFE17B0BDE8F083D2
:100F900084990100950A0100A10A01001966000068
:100FA000A0AE01009CCA01002DE9F0432F4E97B07E
:100FB0002F4D11AC0AAF904699460C9196E80F0060
:100FC00084E80F001EABC4E90275204615A91593ED
:100FD000EFF756F996E80F00264E0DAD85E80F00A5
:100FE0002146C5E902762846EFF74AF90620F3F7CD
:100FF00093FD0627D0F8013016AE9A680B939188BE
:10100000DB68D18006F8407D314601200A93F3F772
:1010100033FD194B44F0010445F001050221032082
:10102000CDE908450793CDF81890F3F7B3FA0446D5
:101030004022002108F09FFB234631464046102203
:10104000F5F7F2FEF526012104250C480C4A02971B
:10105000CDE9032023460596CDE9005110226420F6
:10106000F1F700FE17B0BDE8F08300BF84990100DE
:10107000F10A0100FD0A010041660000A0AE010076
:101080009CCA01002DE9F042214E90B0214D0BACDD
:1010900004AF9946CDE9052196E80F0084E80F00DA
:1010A00016ABC4E9027520460FA90F93EFF7E8F8D5
:1010B00096E80F00184E07AD85E80F00C5E90276E7
:1010C00021462846EFF7DCF8059B144FD3F8013092
:1010D00044F00104D3E90223918845F00105D18051
:1010E000169A0221042004930092CDE9024501974B
:1010F000F3F750FA8822002108F03DFB2222034634
:1011000069464846F5F790FE10B0BDE8F08200BF92
:1011100084990100490B0100550B01002D66000068
:101120002DE9F042214E90B0214D0BAC04AF994611
:10113000CDE9052196E80F0084E80F0016ABC4E95D
:10114000027520460FA90F93EFF79AF896E80F0063
:10115000184E07AD85E80F00C5E9027621462846FE
:10116000EFF78EF8059B144FD3F8013044F00104DB
:10117000D3E90223918845F00105D180169A022116
:10118000052004930092CDE902450197F3F702FA96
:101190004022002108F0EFFA102203466946484633
:1011A000F5F742FE10B0BDE8F08200BF849901005F
:1011B000A50B0100B10B010055660000054B064967
:1011C000013810F8012F013303F8012C8B42F8D1BC
:1011D000704700BF00008360200283602DE9F0416A
:1011E000314E90B0314D0BAC04AF8846069096E876
:1011F0000F0084E80F0016ABC4E9027520460FA962
:101200000F93EFF73DF896E80F00294E07AD85E8FC
:101210000F002146C5E902762846EFF731F8012094
:10122000F3F77AFC05900220F3F776FC0221002008
:10123000F3F7B0F94FF408620021074608F09BFA73
:101240000122059B10AED3F8013010469B6906F8C9
:10125000402D31460493F3F70FFC059BDFF86CC07B
:10126000D3F8013031469A68124EB2F804E03B469A
:10127000A2F806E0404644F0010445F001054FF4B1
:101280000872CDE90245CDE900C6F5F7CDFD0A4B60
:101290000A4C1B690A480B490B4A236103610B6125
:1012A000136110B0BDE8F08184990100910C010038
:1012B000010C0100A14300008C0D0020E00A002079
:1012C000A80B0020700C0020540E0020894B000059
:1012D00038B505460C4601200221F3F75BF9D5F835
:1012E000013004F188059B68D9889A8854F8043B3A
:1012F00003FB01F393FBF2F3A54240F8043BF5D165
:1013000038BD00BF2DE9F041804684B00220F3F7DC
:1013100003FC022106460120F3F73CF902220546B0
:10132000D6F8013004AC9B68012099880E4FD98013
:1013300004F8102D2146F3F79FFB28468822002150
:1013400008F019FA094ADFF82CC0094E009221462C
:101350002B4640462222CDE901C70396F5F764FDEE
:1013600004B0BDE8F08100BF6D0C0100A10D0100CB
:10137000710C0100A50D010083682DE9F04F9D88D7
:10138000814602FB05F52D12FF2DA8BFFF258868B9
:10139000DD808278884601788FB0A1EB4201089108
:1013A0001A789C78B0F806B0007AA2EB4402079055
:1013B000187A91420992069000F0C8800026012216
:1013C00040F25D214FF0020A674F684806330591ED
:1013D000CDE9030711467120CDE90166CDF800A0E3
:1013E0000124F1F73FFC40F25E22D9F80830604852
:1013F0000833059221462246039004977120CDE9D7
:1014000001660094F1F72EFC4FF0040940F25F20D2
:10141000584B2246214605900393712009AB04974F
:10142000CDE90146CDF80090F1F71CFC40F2612CAB
:10143000D8F80830504822462146CDF814C006336B
:10144000039004977120CDE90166CDF800A0F1F773
:1014500009FC40F2622CD8F808304848083322468C
:101460002146CDF814C0039004977120CDE90166A0
:101470000094F1F7F7FB40F26320414B0590039392
:1014800071200497CDE90146CDF80090224621460F
:1014900008ABF1F7E7FB089800FB0BF010B90FB0B1
:1014A000BDE8F08F099BADB203FB05F4079B069ADC
:1014B0000E339B1A9C4094FBF0F451463046F3F7F0
:1014C00069F8E517A0F1040C00F67C0E5CF8040F37
:1014D000C117CDE90C01DDE90C8904FB09F7A4FB78
:1014E000080108FB0576820B314442EA81428B13E6
:1014F000CDE90C23DDE90C23F445CCF80020E5D13F
:1015000002210120F3F746F8A0F1040C00F1840E4B
:101510005CF8040FC117CDE90A01DDE90A8904FB73
:1015200009F7A4FB080108FB0576820B314442EA67
:1015300081428B13CDE90A23DDE90A23F445CCF877
:101540000020E5D101200FB0BDE8F08F40F25A2213
:10155000054B00920B4900226420F1F7D5FB0020D7
:101560000FB0BDE8F08F00BFA0AE0100F0AD0100EC
:1015700018AE01003CAE010048AE010070AE0100A3
:1015800094AE0100D4AD010070B5002482B0FFF725
:1015900013FCF5F7B9F810492346224600940E686B
:1015A000022001210D4DB047FFF76CFCFEF740F91A
:1015B000FEF71CFBFEF750F92046FEF723FF00F074
:1015C0004DFB2C68FEF764FCA0702C68FEF77AFCDB
:1015D000E07002B070BD00BF04D501000C06002011
:1015E0000246034B51680068926807C3704700BF0A
:1015F000B42200202DE9F04F964683B0544E9DF85A
:1016000034709DF830C09846009763460D46B6F991
:101610000620B6F90410044670469DF83870FAF7B3
:10162000A1FE3378800290FBF8F0002B4BD0A91C70
:1016300096F801904B002A4604EB030E03F10208D2
:10164000B9F1000F50D13EF8069C05F1FF3C24F89B
:101650000890A3F108053EF8043C254424F8113015
:101660006189238961802380531ED2B31A4602F117
:10167000010B4FEA4B0104EB010A063134F80190EB
:101680003AF8028C34F81B30C84407FB08F9BAF862
:10169000048096F903B043440BFB0398BAF8023078
:1016A00096F90290624509FB03834FEAA31300FBFE
:1016B00003F34FEA2343635246D0012AD4D1E3888F
:1016C00000226380D3E765B1A91C04EB4101043417
:1016D00031F8022D00FB02F28C424FEA22428A804E
:1016E000F6D103B0BDE8F08F00236380238024F897
:1016F000113024F80830002DF3D07F0004EB4501B1
:1017000031F802E996F90350B1F808C00B88CA888D
:101710009C4538BF9C46964538BF96460CFB07F360
:101720006A000EFB02338D8896F902208C4205FB7D
:1017300002324FEAA21200FB02F24FEA22420A8171
:10174000DED103B0BDE8F08F2B88AEF800308BE718
:10175000B4220020F0B505462C4C426994F90330C0
:1017600094F90270C3F12003E07AC7EB4307A37A30
:1017700085B0C7F34707CDE90107009305F12C00B9
:1017800022230E461021FFF735FF617A237A05F1F7
:1017900054046A692046CDE90117009322211023E1
:1017A000FFF728FFFEF7EAF8204631234FF0804488
:1017B00003F1600230F8021D013B212B44F8221096
:1017C000F6D14FF0804405F1A00232F8020D03F18A
:1017D0006001013B44F82100591CF6D10120FEF7BD
:1017E0008FF82846FEF7D2F8B4F84C301BB23360BD
:1017F00094F85030337294F85130737294F8523038
:10180000B37294F85330F37205B0F0BDB4220020E7
:1018100038B504220125124B124C1D712260FFF7CE
:1018200079F8F8F7F1FF837E2BB90F4B1B6813B1E2
:101830000E4A157098470E4BD3F80021120708D5B1
:10184000002208250B480C49C3F880510270C1F8EA
:10185000402101211023094AD160236038BD00BF17
:10186000842200205809002044100020001000208D
:1018700000E100E05709002000000250000008507D
:101880000122052138B50D4B0D4C5A712160FFF72F
:1018900045F80C4BD3F80021120708D50022082583
:1018A00009480A49C3F880510270C1F8402101215A
:1018B0001023074AD160236038BD00BF8422002076
:1018C0005809002000E100E0570900200000025004
:1018D000000009500321012238B5144B144C154D5A
:1018E000DA702160FEF794FE2B78D3B901232B70B8
:1018F000FEF7C0FE104B1B6803B19847F8F784FF52
:10190000C37E03F0FF052BB90C4B1B6813B198473E
:101910000B4B1D70002110230A4AC2F840112360AE
:1019200038BDFEF7B5FE084B1860DFE784220020C3
:10193000580900205709002094100020481000206A
:101940000010002000000250B022002001234FF0C0
:101950006050102110B4034A034CE372836210BC40
:101960001160704758090020842200200F21124A7C
:10197000124B11605B6F84B00193019B23F4FF63F2
:1019800023F007030293019B23F07F030393029B41
:10199000B3F5800F0AD0039A094B9A4206D0019AF8
:1019A000084B9A4202D20122074B1A700122034BC4
:1019B000A3F86C2004B070475809002000001050B4
:1019C00080FF010000FC0100C022002008B5FFF7E5
:1019D000DBFD00F07FFD002008BD00BF704700BFA9
:1019E00030B50A4D0A4C83B0294620464FF0CD321F
:1019F000FCF7BAF94FF0CD32204600922B46054A4B
:101A00000549FCF71BFA002003B030BD943F0020CD
:101A1000942F002000560020943F0020704700BF04
:101A200040F2071330B50C4A0C4D0D4C83B01268D0
:101A30002146009363202B46F1F766F9F2F7BCFECE
:101A400040F20910074A2B46126821460090632095
:101A5000F1F75AF903B030BD0404002014AF0100BF
:101A600004AF01000804002000210120F2F792BD1C
:101A70005B232DE9F0411D4A1D4D1E4C84B01268B8
:101A80002146009363202B46F1F73EF9F2F79CFDC7
:101A90000220F3F741F8074603A8FDF7CDFE022127
:101AA0000120F2F777FD8046134B04A91B88134EE3
:101AB00021F8083D0220F2F7DFFF0220FFF722FCA9
:101AC00030460221FFF78AFB326941463846FFF76C
:101AD000FFFB6E200A4A2B461268214600906320C5
:101AE000F1F712F904B0BDE8F08100BF0404002052
:101AF00014AF0100E4AE0100949901008C0D0020A8
:101B0000080400202DE9F0430220ABB0F3F704F8FD
:101B100002210120F2F73EFD002107460120F2F7E5
:101B200039FD064607A8FDF787FE05462D4C88229D
:101B30000021204607F01FFE079AEDB219A80DF10B
:101B4000200C0492CDE901C0039400972946334646
:101B50001A220220FDF7CCF95DB1204604EB4502C4
:101B6000B0F90030002BB8BF5B4220F8023B904236
:101B7000F6D101244FF00409A1200621DFF874807A
:101B8000194A3B460590CDE90141CDE9032821469C
:101B90002A46CDF800906220F1F764F80027A221D0
:101BA000124A33460591CDE90272CDF810802A46DB
:101BB000CDE9009402217220F1F754F8A426022006
:101BC0000B4B00900393CDF81080CDE901472146DF
:101BD0002A460596034B6920F1F744F801482BB0DB
:101BE000BDE8F083A0250020ECAF0100F8AF0100B4
:101BF00004B0010014AF0100022300B583B002A9B4
:101C000001F8043D0120F2F737FFF2F7BDFFF2F7CC
